:10000000004000209D740000DD740000DF740000DB
:1000100000000000000000000000000000000000E0
:10002000000000000000000000000000E17400007B
:100030000000000000000000E3740000E574000010
:10004000E77400008155000049780000E774000063
:10005000E774000000000000E7740000E77400008F
:10006000E77400001D7C000045340000E7740000C8
:10007000E7740000E7740000E7740000E774000014
:10008000E7740000CD780000E7740000E77400001A
:10009000E7740000E7740000E7740000E7740000F4
:1000A000E7740000E774000000000000000000009A
:1000B0000000000000000000000000000000000040
:1000C00010B5064C2378002B07D1054B002B02D02E
:1000D000044800E000BF0123237010BD6802002027
:1000E000000000001CE80000044B10B5002B03D0FA
:1000F0000349044800E000BF10BDC04600000000F6
:100100006C0200201CE80000164B002B00D1144BA1
:100110009D46402292029A1A924600218B460F4633
:100120001348144A121A0BF0ADFB0F4B002B00D0F2
:1001300098470E4B002B00D0984700200021040068
:100140000D000D48002802D00C4800E000BF0BF065
:1001500059FB2000290007F0C9FB0BF02DFBC0461E
:100160000000080000400020000000000000000027
:1001700068020020C82F00200000000000000000DE
:1001800002000120104011D1042A0ED91368180969
:1001900080B2002809D001388000031D11180979A8
:1001A000002902D001309842F8D170470020FCE7C6
:1001B0000378002B03D05AB2002A01DB01307047CC
:1001C0003F229343C03B59424B41C01803789343AD
:1001D000802BF4D10130F9E710B500240378002B0F
:1001E00001D1200010BDFFF7E3FF0134F6E770B541
:1001F000002204000D00411C092003F04DFC0028E2
:1002000006D001236200134343600023A34200DBB6
:1002100070BD9A00A958821891600133F6E770B555
:10022000012803DC1C2001F0CFF870BD01230D680C
:1002300011201D42F7D04868184206D1042804D97D
:100240000F2302681340042B01D00E20EBE703F0CC
:1002500081FA6D100400002D03DDFFF7BDFFA842F9
:1002600006DA1220DFE72000FFF7A2FF0400013DBD
:10027000012DF8D120787F2809DDDF280BDCF82359
:100280003F22DB00800118406378134018430123AC
:1002900040001843C9E7EF280BDCFC226378120109
:1002A0009B0113403F220007000C0343A07810403D
:1002B000ECE7F72812DCFC22637892021B03134060
:1002C000E0228004520310403F221843E378134099
:1002D000FC220343A07812018001E8E7012040429C
:1002E000D5E7F8B54D680F00EB0706D4042D04D907
:1002F0000F232E683340092B03D00B2001F064F844
:10030000F8BD6B683609B6B25C10731EA3420FD8F5
:100310000321200009F072F96421642803DC010044
:10032000032800DA03212800891903F0E7FB050000
:100330002B6800201B099BB2013B9C42E0D23A682B
:10034000A31C9B005A510123013464001C436C60C0
:10035000D6E7F0B585B0012803DC1C2001F034F8A5
:1003600012E001274B683A000093022806D08B6800
:100370003B4203D05F10002F00DC17000125009BDB
:100380002B4203D00120404205B0F0BD009B042B5E
:10039000F8D91B680C680F261900314004292AD1AE
:1003A0002C4205D1042C03D923681E40042E01D011
:1003B0000E20D3E70098FFF7E3FEB842E2DB009897
:1003C00003F0C8F90600200003F0C4F90100781E0C
:1003D00030180BF00DFE041ED4D03378002B01D062
:1003E000A64202D36800012521E03000FFF7E0FEBD
:1003F00001350600F1E709293ED1009B5B685B10DF
:1004000001939F42BEDC2C422ED1042C2CD92368B0
:100410003340042B28D1200003F09CF9039602906E
:100420007E1C009AB300D058844202D17800284341
:10043000AAE728420ED104280CD90368039A134076
:10044000042B07D103F086F9010002980BF09AFD06
:100450000028EBD0019B37009E42E1DD92E71F00B0
:10046000019B9F4200DD8DE77B1C00999A008A5812
:10047000A242F4D17800B6E7032900D082E71A0936
:1004800092B25B0F92000B40D31A01939F4200DDA2
:1004900078E72C4229D1042C27D922681640032E54
:1004A00019D1100980B2520F80003240251D801AE8
:1004B000019B2E181B1A0193009B781E0433019A8E
:1004C000904200DD5EE72A001918B2420FD316D120
:1004D0000130400087E7042E07D1200003F03AF9ED
:1004E00005002000FFF74CFEE2E70F2036E70C780E
:1004F000A4461478A44502D101310132E5E7013068
:10050000DDE710B503F00AF943000120184310BDE0
:10051000C30711D404280FD90F2302681340032BFB
:100520000AD119400133591AC0234907DB05194084
:10053000024B1A40114301607047C046FFFFFF9F06
:10054000F7B507000E001C20012F06DD4C680123C3
:1005500022001A40009203D10D2000F035FF53E035
:10056000022F02D08A681A42F6D0012335681D4254
:1005700000D0A9E0042D00D8A6E01C41002C00DC2E
:100580001C000F2029680840092828D16B685B10DF
:100590000093022F05D0B368009A5B109A4200DDE9
:1005A0000093009B01221D1B0135EB43DB171D400F
:1005B000691C092003F070FA071E09D001236D00A1
:1005C0001D4303003268083345600099A14201DAF7
:1005D0003800FEBD0134A100515802C3F5E70428DC
:1005E00045D1280003F0B6F8FFF7F6FD0190022F81
:1005F00004D0B3685B10984200DD0193019BA342D5
:1006000004DA002003F0BAFA0700E1E7280003F05B
:10061000A1F80700009BA34221DB2800009703F00C
:1006200099F805003800FFF7C3FD019B013407006E
:10063000A342F7DA009BC41A200003F09FFA071EBA
:10064000C6D003F087F80190306803F083F82200E9
:10065000009B591B411801980BF0F8F8B8E73800D7
:10066000FFF7A6FD009B070001330093D2E70328A4
:100670002AD10B099BB2490F9B000140591A022F46
:1006800004D0B2685210914200DD1100A14205DA97
:1006900000220320110003F0FFF9B5E703200E1B31
:1006A000331DD9170140C9188910002203F0F4F94D
:1006B000071E00D18CE7013631000334FFF728FF15
:1006C000381D29193200C7E7212046E7F8B5002870
:1006D00005DC1C2000F078FE05002800F8BD01268E
:1006E0000C6826400FD06410E343DB171C40E11C6C
:1006F00089100022032003F0CFF9051EEDD0210060
:10070000FFF706FFE9E7042C01D80025E5E70F23F2
:1007100022681340042B1BD12000FFF731FDC31CBE
:1007200007000320D9170140C9188910320003F0CF
:10073000B3F9051ED1D03900FFF7EAFE200003F01F
:1007400009F82B1D01003A0018000BF07FF8C4E7F0
:10075000092BDAD10320636832005F10FB1CD91724
:100760000140C918891003F097F9051ECDD0390052
:10077000FFF7CEFEFF20BE42AFDA0122B300E3183E
:100780009B68134208D01341FF2B00DD0300D943BF
:10079000C917AA190B4013710136ECE710B57F2970
:1007A00002DC0170013010BD1A4B99420CDC402371
:1007B0008A115B42134303703F230B40802149425F
:1007C000194341700230EEE7134B994210DC2023AD
:1007D0000A135B4213433F24802203708B11524261
:1007E0002340214013430A43437082700330DAE709
:1007F0000A4B9942D7DCF0230370603B4370113BF6
:100800008A11FF3B1A4382703F2211401943C17085
:100810000430C8E7FF070000FFFF0000FF0F0100E2
:10082000F0B50D0085B0002803DC1C2000F0CCFDE5
:100830000DE009680122080010400AD002AC114105
:100840002000FFF7ABFF011B200003F0A3F9040019
:100850001AE004293FD90F230C682340092B3AD111
:100860004B685B10019303239C46019B9A420EDD6B
:1008700003F084F9041E07D02E68012502F06AFFF8
:100880002F00019B9D421DDD200005B0F0BD01320F
:100890009300CC580123234001D10D20C6E76410FA
:1008A0007F2C0DDD0D4E0223B44209DD0C4E634654
:1008B000B44205DD00270B4EE30FA6427B419B00AF
:1008C000C018D2E70135AB00F1583942E5D04910E4
:1008D000FFF764FFD5E72120A8E7C046FF07000027
:1008E000FFFF0000FF0F010010B5040001200840C9
:1008F00010D104290DD90F230A681340042B08D105
:10090000080002F027FF010020000BF03BFB4342F0
:10091000584110BD0020FCE7F7B50F00012803DCAB
:100920001C2000F051FDFEBD01264D682E4006D171
:10093000042D04D90F222B681A40092A01D00B205C
:10094000EFE76A681B099BB25410A34200D85C1EF3
:1009500039681E48FFF7C8FF01230190002813D112
:1009600039681B48FFF7C0FF002811D0002C0DD0BC
:100970000123621C013C9C409200535123436B6055
:1009800004E00136B200AB50B442FADA0020CAE704
:100990003B680D20DA07C4D55B10002B11DD9C42AB
:1009A0000FDB9B00A200291DEB1889180433994224
:1009B00009D10123013C9C40AA181C4353606C6080
:1009C000E4E71220ADE758681860EFE717CF0000A2
:1009D0001BCF0000002310B50C000B70C30705D51A
:1009E0000D49421020000BF091FA08E00B49002855
:1009F00002D0042804D10A4920000BF0A7FA10BD48
:100A00000428FCD90F2302681340042BF7D102F00D
:100A1000A1FE04490200E5E798D9000020CF0000BC
:100A200026CF00002BCF0000F0B593B00600029156
:100A30001C20012E1DDD029B01251B681C002C4083
:100A400000D0ADE0042B00D8E6E01A680F231A406E
:100A5000092A4AD10394039A029992008A581700EE
:100A60002F4005D1042A03D910681840092806D060
:100A7000222000F0A9FC0190019813B0F0BD52684B
:100A80005210A418039A013203929642E3D1611CDA
:100A9000012203F001F80190002802D10023019304
:100AA000EAE7019B6400190025435D600831029A62
:100AB000BB00D05802684368120992B25B109A4298
:100AC00000D8531E0022934209DCDA43D2171340A8
:100AD0009B00C918039B01379F42E8DBCCE79400D9
:100AE0000519AD6801320D51EDE72700032A59D1F0
:100AF0000193029ABB00D3582B42B9D1042BB7D92A
:100B0000186801990140032939D1020992B2430FB3
:100B100092000B40D31A1C190137BE42E9D10320C1
:100B2000E31CD9170140C9188910002202F0B4FF54
:100B300001900028B2D000252100FFF7E9FC019BBD
:100B40001E1D029AAB00D45801231C421FD1042C55
:100B50001DD90F2123681940032918D1180980B223
:100B60005B0F80000B40C01A0023834213DBC3439A
:100B7000DB17184001353618BD42E2DB7CE704295B
:100B800000D075E71800FFF7FBFA2418C4E720002F
:100B9000FFF7F6FAE8E7E2181279F2540133E4E7D6
:100BA00000273C000F25029ABB00D35801221342B4
:100BB00034D1042B32D9186801002940042935D1D9
:100BC0001800FFF7DDFA24180137BE42EBD12000F0
:100BD00002F0D4FF0190002800D15FE7029FB60029
:100BE000BB19041D029301233D681D4229D1042D28
:100BF00027D90F262B681E40042E37D12800FFF777
:100C0000BFFA0600280002F0A5FD01002000320016
:100C10000AF01CFEA41922E02700C3E7180005A96A
:100C2000FFF7D8FE05A80BF0B7F9CCE7032900D0F1
:100C30001EE7020992B2430F92000B40D31A1C190F
:100C4000C2E705A92800FFF7C5FE05A80BF0A4F927
:100C500005A90500020020000AF0F8FD6419029BB6
:100C60000437BB42BFD10023237005E7032EF6D122
:100C70001A0992B25B0F92001E40961B291DC5E710
:100C8000F0B50D0097B0002806DC1C2000F09CFB9E
:100C90000700380017B0F0BD0C68012123000B409D
:100CA000009306D1042C04D922680F331A40092A74
:100CB00001D00B20EAE7626852100392002A03DC9D
:100CC000009802F05BFFE3E7504A019201280BD045
:100CD0006868084208D1042806D902681340042B2A
:100CE00002D102F037FD019001980BF055F9060092
:100CF0000F27039B0834013B05935E43039B02903F
:100D00009B00E318049301232068184273D1042840
:100D100071D901680B003B409C46042B03D1FFF7BF
:100D20002FFA861909E0032B6CD162460B099BB29E
:100D3000490F9B0011405A1A9619049B0434A34290
:100D4000E1D1300002F01AFF071EA2D02B680793F2
:100D5000029B002B03D0686802F0FCFC0190380075
:100D600002F0F8FC0400009B079A9B00D3189E68D1
:100D7000300002F0EFFC0123334005000693002B06
:100D800001D1042E04D809A93000FFF723FE09ADD4
:100D900028000BF001F9069B0490002B0ED1042EC5
:100DA0000CD90F2133681940032907D11A0992B2CF
:100DB0005B0F92000B40D31A351D04932000049A58
:100DC00029000AF043FD049BE418029B002B0AD083
:100DD000059B009A934206DD2000029A01990AF0D1
:100DE00035FD029BE418009B01330093009A039B9E
:100DF0009342B8D14DE709A9FFF7ECFD09A80BF024
:100E0000CBF88EE702F0A6FCF9E7C046B8D30000A5
:100E100010B50024A04207DD0B6801341C4003D04C
:100E20005C10E343DB171C40611C0122092002F027
:100E300033FE002803D0012364001C43446010BD2E
:100E40000A6870B510000125284034D1042A32D92F
:100E50000F24136849681C40092C17D154681B09DA
:100E60009BB22C41A34200D85C1E844205DC0220C8
:100E70000133984206DB00200FE085005519A96078
:100E80000130F2E7840011510130F2E7032C12D156
:100E9000294203D1132000F097FA70BD4910FF29B1
:100EA000F8D81B099BB204329B00D3189342E2D9B5
:100EB00011700132FAE70B2000F086FADBE7000040
:100EC000F8B5012700254E680C003740AF420ED11F
:100ED0003D00042E0BD90F2233681A40092A10D185
:100EE00072681B099BB25510AB4200D85D1E216889
:100EF000CB0716D54C10002C01DDA5421CDA1220C0
:100F000030E0042A04D13000FFF73AF90500EEE79B
:100F1000032AECD11D09ADB25B0FAD001340ED1AF1
:100F2000E5E72748FFF7E0FC002813D00AF08AFF26
:100F3000290008F049FC4C1C002F3ED1042E3CD95E
:100F40000F2332681340092B10D10134A400A45997
:100F50002000F8BD21681B48FFF7C6FC2C000028C4
:100F6000EAD1113000F030FA0400F1E7042B1CD173
:100F7000300002F0EFFB0500012C0EDCFFF718F942
:100F8000461B300002F0FAFD041EE1D002F0E2FB45
:100F9000320029000AF05AFCDAE72B78013C002BDA
:100FA000ADD02800FFF704F9E5E7032B05D134198C
:100FB000E37801245B001C43CAE70B20D2E7C0465C
:100FC00010CF00001BCF0000F7B54D680F002A00BE
:100FD00001210A402FD1042D2DD90F242B68BE6882
:100FE0001C40092C14D169681B099BB24C1001925A
:100FF000A34200D85C1E39682A48FFF775FC002818
:101000002DD00F232A681340092B1DD1012317E08F
:10101000032C10D10E4203D1132000F0D5F9FEBDF0
:1010200072100192FF2AF7D81A0992B25B0F920050
:101030001C40141BDFE70B20EFE701339A00AE5092
:101040009C42FADA0020EAE7032BFBD12B000133A4
:101050005A1BA242F6DC6A461279DA70F7E7396861
:10106000CB0706D54910002901DD8C4209DA122090
:10107000D3E70D48FFF738FC2100002801D11130DB
:10108000CBE70F232A681340092B03D101318900D4
:101090004E51D7E7032BD5D16B461B796D18EB70FA
:1010A000D0E7C04617CF00001BCF000070B5012469
:1010B0000868204207D1042805D90F2501680D4092
:1010C000092D02D14468200070BD032D08D10A0902
:1010D00092B24B0F92002B40D31A5B001C43F2E7F5
:1010E000042DF0D102F036FBFFF776F84000044300
:1010F000E9E7000010B5034A0B21034804F014FB94
:1011000010BDC046B8CE0000B0CE00000020704731
:10111000042070470120704710B5002002F02EFD1A
:1011200010BD00207047002070470020704700204D
:101130007047002070470020704700207047002053
:101140007047000010B5034A0C21034804F0ECFA84
:1011500010BDC046A0CF000000D00000704703784B
:10116000002B03D05AB2002A01DB013070473F2226
:101170009343C03B59424B41C01803789343802BA3
:10118000F4D10130F9E70000F8B50127060014009A
:101190000800394227D104293FD90F230A681A4091
:1011A000042A3AD13C4213D1042C11D922681340AD
:1011B000042B0DD102F0CEFA0500200002F0CAFA8D
:1011C000010028000AF0DEFE00282EDB1FD127E0F8
:1011D000E30722D502F0BEFA0A2200210AF0A4FF9A
:1011E0000500601010E0174015D1042A15D90F230F
:1011F00012681340042B10D120004D1002F0AAFAFF
:101200000A2239000AF090FF85420EDB08DD002E2D
:1012100009DC00200CE04D10E3E70F22054B1A70AB
:101220000136022EF5D8042002E004207617304063
:10123000F8BDC046A802002010B50124044002D029
:101240004410200010BD042810D90F230268134059
:10125000042B07D102F07EFA21000A220AF064FF73
:101260000400EEE7032B01D10430F5E70D22014B1A
:101270001A70E6E7A8020020012210B5024018D13A
:10128000042802D903681A0992B201230B4012D133
:10129000042902D90B681B099BB20024934206D192
:1012A00004309B000431C318984206D30124200067
:1012B00010BD0022E9E70023EFE704780A78002C4C
:1012C00001D1002AF2D0013001319442ECD0002447
:1012D000EDE70000F7B50700009101933049314B6D
:1012E000002A02D002220A70013A00261A601B6806
:1012F000CE54BE4200DBF7BD009AB300D058294B54
:10130000274D1C68C8239B0065191C1B012318422C
:1013100006D0254A4310210028000AF0C5FD09E047
:10132000224A002802D004281BD1214A210028008B
:101330000AF0BAFD1A4C20000AF02EFE194A019B51
:101340001060002B0BD07B1EB34208DD194B984276
:1013500005D8431C1360202222540022E254013697
:10136000C7E7042819D90F2301680B40042B04D1C7
:1013700002F0F0F9104A0300CDE7092B03D14368CE
:101380000E4A5B10C7E7032B08D10A0992B2490F36
:1013900092000B40D31A0A4ABDE70123094ABAE773
:1013A000A9020020CC05002098D9000020CF000021
:1013B00026CF00001F030000C3DF000070D2000032
:1013C0007FD200008AD20000014B187000207047C5
:1013D000A802002070B501F01DFF094C0100251D79
:1013E0001F2228000AF0F0FD28000AF0D5FD042392
:1013F00004308008000118432060200070BDC04602
:1014000084020020C368F0B59D00836889B05D192F
:101410000300183306930369069A9F00069B039006
:10142000DF19436901939B00D3180293CD4B1B78BE
:10143000002B26D17F222B68CB491C1213409B0026
:101440005B58043501929F46039B587804F0A6FD33
:101450000023039A137027E0C24B1B78002B10D196
:101460002B68019A1C121340BF4A9B009B580435FD
:10147000E9E7069B3A1DD11ABA4BD82928DD1A2272
:101480001A70039BB74C9B6821780193EA1A039B5F
:1014900092109B7812021A43039B587804F086FD41
:1014A0000023039A23701370039B069A9B68019391
:1014B000ED1A039BAD10DD60069BFE1A039BB61070
:1014C0001E61029B9B1A039A9B10536109B0F0BDE9
:1014D0001B783C60002B01D01700D2E72B680199E4
:1014E0001C120B40A0499B005B5817000435AAE76B
:1014F000069B3A1DD11A9B4BD82902DD1A221A707D
:10150000BFE728681B78291D3860002B02D0170020
:101510000D00B6E76B6801991C120B4092499B00C5
:101520005B58170008358EE7069B3A1DD11A8D4B84
:10153000D82902DD1A221A70A3E7A4001B782C19FF
:101540003C60002B01D017009BE72B6801991C120F
:101550000B4085499B005B581700043573E7069BD9
:101560003A1DD11A7F4BD82902DD1A221A7088E75A
:101570007E48A40021581B783960002B01D0170049
:101580007FE72B6801991C120B4077499B005B5841
:101590001700043557E7043F744B3A68A400E25043
:1015A000704B1B78002B00D06BE72B68019A1C1244
:1015B00013406D4A9B009B58043544E76B4BA400D5
:1015C000E058FFF739FE043F06003868FFF734FEA5
:1015D00036180120654B76000643E650614B1B78B8
:1015E000002B00D04DE72B68019A1C1213405E4A75
:1015F0009B009B58043526E7069B3A1DD11A594B90
:10160000D82902DD1A221A703BE70698029C0121B4
:10161000A04202D221000C3909681B783960002BE6
:1016200001D017002DE72B6801991C120B404E4981
:101630009B005B581700043505E7069B3A1DD11A3D
:10164000484BD82902DD1A221A701AE70699029827
:1016500081420FD203000C3B1968454B4910E41836
:10166000641AA40023583B603E4B1B78002B05D026
:10167000170006E7182119700023F4E72B68019979
:101680001C120B4038499B005B5817000435DAE602
:10169000069B029A934219D213000C3B1968344BF3
:1016A000043FE41813004910611A3A688900CA50CF
:1016B0002C4B1B78002B00D0E3E62B68019A1C1200
:1016C0001340294A9B009B580435BCE61822254B41
:1016D0001A70EDE7069B029A93422DD2244B3E1FCF
:1016E000E31814000C3C04932368049A5B10D31A8B
:1016F000029A9B009858FFF79FFD07903068FFF70C
:101700009BFD2468049B64101C1B079BA4001F18EE
:1017100001207F00029B0743E7503700114B1B78E5
:10172000002B00D0ADE62B68019A1C1213400E4A24
:101730009B009B58043586E618220A4B1A70EDE789
:10174000069B3A1DD11A074BD82902DD1A221A70BE
:1017500097E60299A40061581B783960002B09D0E4
:1017600017008EE6A802002070D00000942D002003
:10177000FDFFFF3F2B6801991C120B40CF499B00D6
:101780005B58170004355EE6043F029B3A68A400EC
:10179000E250CB4B1B78002B00D072E62B68019AED
:1017A0001C121340C54A9B009B5804354BE6029B14
:1017B000A4001C192368043F38685E10FFF73CFD45
:1017C00036180120BE4B76001B7806432660002B9E
:1017D00000D056E62B68019A1C121340B74A9B00B2
:1017E0009B5804352FE6069BA4003F1BB44CBB421C
:1017F0000CD82378002B00D043E62B68019A1C12EA
:101800001340AE4A9B009B5804351CE6AD4801F0DE
:1018100091FF2378002B00D033E62B68019A1C122D
:101820001340A64A9B009B5804350CE6A300ED1814
:10183000002C00DA38E6A24B1B78002B00D020E603
:101840002B68019A1C1213409C4A9B009B5804353C
:10185000F9E5043F3B68042B04D1A300ED18002CEC
:1018600000DA21E6964B1B78002B00D009E62B68A6
:10187000019A1C121340914A9B009B580435E2E5E3
:10188000043F3B68042B04D0A300ED18002C00DAC1
:101890000AE68B4B1B78002B00D0F2E52B68019AEF
:1018A0001C121340854A9B009B580435CBE53E1F14
:1018B0003068C3070AD540100138002809DB01232E
:1018C0004000A40018432D193060EDE5FFF7B4FC8B
:1018D000F2E77B4B37001B78002B00D0D1E52B685B
:1018E000019A1C121340754A9B009B580435AAE5C7
:1018F0003A00069B0C32D31AD82B03DD1A22704B08
:101900001A70BEE5FF2361005B001940FE3BFF3B00
:1019100019433960039906988968241204916D1A55
:101920000399AD1089782D020D4302999D40091A43
:10193000891099401D430B43BB60039B7D609C70E5
:10194000E4B2614BE4000292E358039A93605C4A6C
:101950001278002A03D008331D00029F91E51D0074
:10196000019A9B680C351C121340544A9B009B58EB
:10197000029F68E53B1F1C68029A069B934232D186
:101980000A20E30711D4042C18D90F23226813402E
:10199000042B16D1200001F0DDFE0AF0FDFAC82369
:1019A0009B00984200D918000630643003F0F6FE20
:1019B00000280FD1043D069B029375E50720042CF7
:1019C000F3D02000431E9841FA234042FF331840D1
:1019D0000730EAE7039B2100587804F0F9FA002366
:1019E000039A1370E7E7029B029A0C3B1B6803996A
:1019F0005B109B00D31A0C3B1C601F1D1300083B9F
:101A00001B685A108A70D2B22F49D2005B00555819
:101A10009B0A039A9B009560ED18029B069A043B73
:101A20001B685B109B00D3180293254B1B78002B7F
:101A300000D026E52B68019A1C1213401F4A9B0018
:101A40009B580435FFE43B1F1868FFF7F5FBA40023
:101A500006003F1B1E2827DC00280DDC184B1B78D6
:101A6000002B00D00DE52B68019A1C121340134A7D
:101A70009B009B580435E6E401F0B8FB033E3618A2
:101A800001F0B4FB114B801B9842F9D80C4B1B782A
:101A9000002B00D0F5E42B68019A1C121340074A72
:101AA0009B009B580435CEE40123039A137001F088
:101AB0009DFB039B0A3886195E60F5E470D0000038
:101AC000A80200209CD200009C2500203F420F006D
:101AD0003B1F1868FFF7B0FBA40006003F1B00285F
:101AE0000DDCD14B1B78002B00D0CAE42B68019A87
:101AF0001C121340CD4A9B009B580435A3E4CC4BE9
:101B0000984203DD1D22C84B1A70BAE40123039AE0
:101B1000137001F06BFBFA239B005E430A3E301802
:101B2000039B5860C0E4A300FF1A002320001A00A2
:101B30003900FFF7CFFBBF4EBF4C3168200002F0E9
:101B400029F8BE4B31681860200004F0E3F83168D2
:101B5000200004F044FAB44B1B78002B00D090E432
:101B60002B68019A1C121340B04A9B009B58043505
:101B700069E4AD4BA4001B783F1B002B00D080E430
:101B80002B68019A1C121340A84A9B009B580435ED
:101B900059E4039803F066FEA34B1B78002B00D09A
:101BA0006FE42B68019A1C121340A04A9B009B58BB
:101BB000043548E43B1F1B68002B49D13B000C3B1C
:101BC0001868012303401E1E1FD046103A0001234F
:101BD0007100083A0B431360002E00DC94E00123EF
:101BE00072001A43391F0A603A00083A12681A4113
:101BF000921B04923A000C3A106818422BD0049AB7
:101C0000A400D2189A40134331E004281BD90F23B3
:101C100002681340092B02D143685E10D6E7042BFB
:101C200008D101F097FD0378002BCFD0FFF797FA8A
:101C30000136F8E7032B06D11609B6B2520FB600EB
:101C40001340F61AC2E71922774B1A70FFF719FCF6
:101C50005B105E1EC0E7042851D90F2102680A40BC
:101C6000092A16D1049BA40002339B001B58029A38
:101C7000A3506D4B1B78002B01D0FFF702FC2B68A3
:101C8000019A1C121340694A9B009B580435FFF7C8
:101C9000DAFB042A2BD1029BA4001B19079301F045
:101CA00059FD0600049C0134012C10DC3000FFF7C4
:101CB00056FA831B1800049301F060FF041E0ED037
:101CC00001F048FD049A310009F0C0FD07E03178C9
:101CD000013C002906D112220C00534B1A70079BBD
:101CE0001C60C6E73000FFF73AFA0600DCE7032A7B
:101CF00005D1049AA40082181279520083E71922B0
:101D0000494B1A70FFF7BDFB0435B2E7A300069AF2
:101D1000FB189B1AD82B12DC0123002C14DC424B3D
:101D20001B78002B01D0FFF7ACFB2B68019A1C122B
:101D300013403E4A9B009B580435FFF784FB1A2250
:101D4000394B1A70FFF79DFB3B60013C0437E4E719
:101D5000069A3B1D9B1A344ED82B03DD1A23337091
:101D6000FFF78FFB069B029AA40093422AD23B1FE7
:101D70001868FFF761FA011E21DD029B0C3B1A680F
:101D8000521082421BDB9007801A2D4B4018C0185E
:101D9000029B8000C2583B1B1A60234B3F1B1B78E1
:101DA0000437002B01D0FFF76CFB2B68019A1C1243
:101DB00013401E4A9B009B580435FFF744FB202329
:101DC0003370EAE71823FBE71C4BA4001A683B1B9F
:101DD0001F001A60144B04371B78002B01D0FFF74B
:101DE00050FB2B68019A1C121340104A9B009B5811
:101DF0000435FFF728FB3B1F1A68042A11D1A40001
:101E00002D19094B1B78002B01D0FFF73AFB2B68EB
:101E1000019A1C121340054A9B009B580435FFF79A
:101E200012FB1F00EDE7C046A802002070D00000A2
:101E300080EE3600CC050020A9020020080000201A
:101E4000FCFFFF3F3A1F1368042B04D000231360EC
:101E50003A00A4002D19D54B1B78002B02D0170097
:101E6000FFF70FFB2B6801991C120B40D0499B0018
:101E70005B5817000435FFF7E6FAA3009C46F81AF2
:101E8000002C17DC1C22C94B1A7000230360634628
:101E9000FF1AC64B04371B78002B01D0FFF7F1FA6D
:101EA0002B68019A1C121340C14A9B009B580435B1
:101EB000FFF7C9FA036804005A1063461E1801238D
:101EC00021680B4003D10D21B84A1170DEE749109B
:101ED0008A4200DD0A000434B442F0D101235200EA
:101EE0001343D3E7A3009C46F81A002C17DC1C22EE
:101EF000AE4B1A70002303606346FF1AAB4B0437E6
:101F00001B78002B01D0FFF7BCFA2B68019A1C123A
:101F10001340A74A9B009B580435FFF794FA0368C7
:101F200004005A1063461E18012321680B4003D198
:101F30000D219E4A1170DEE749108A4200DA0A003C
:101F40000434B442F0D1012352001343D3E73B00E1
:101F50000122083B1968A40011421DD03B1F1B68D9
:101F6000134219D0114113410022994200DA043280
:101F70003B1B1A608D4B3F1B1B780437002B01D095
:101F8000FFF77FFA2B68019A1C121340884A9B00C6
:101F90009B580435FFF757FA02203B1F1A6840424E
:101FA000FFF7F2F83E1B3060E4E73B00083B19689E
:101FB0000123A40019421ED03A1F12681A421AD0F7
:101FC00019415010CB0FD217884253413A1B9B0046
:101FD0001360764B3F1B1B780437002B01D0FFF7B3
:101FE00050FA2B68019A1C121340714A9B009B58AF
:101FF0000435FFF728FA01203B1F1A684042FFF71B
:10200000C3F83E1B3060E4E73B00083B18683B1F09
:102010001968A600BE1B0423814202D0042802D8FE
:102020000023336018E001239C461842F8D10F23A7
:1020300002681A40042AF3D163461942F0D10429F8
:10204000EED90B680B321340042BE9D1FFF714F9DA
:10205000431E984180003060544BA4001B783F1B06
:102060000437002B01D0FFF70CFA2B68019A1C12E1
:1020700013404F4A9B009B580435FFF7E4F93B009F
:10208000083B18683B1F1968A600BE1B002381424D
:1020900002D0042802D80423336018E001239C46B0
:1020A0001842F8D10F2302681A40042AF3D163467C
:1020B0001942F0D10429EED90B680B321340042BDE
:1020C000E9D1FFF7D9F84342584180003060374BDF
:1020D000A4001B783F1B0437002B01D0FFF7D1F978
:1020E0002B68019A1C121340314A9B009B580435FF
:1020F000FFF7A9F93B000122083B1968A40011422F
:102100001ED03B1F1B6813421AD05B104A10D80F19
:10211000C9179A4241413B1B89001960234B3F1B61
:102120001B780437002B01D0FFF7ABF92B68019A1D
:102130001C1213401E4A9B009B580435FFF783F97D
:102140003B1F1A680120FFF71FF83E1B3060E5E7D0
:102150003B000122083B1968A40011421DD03B1F1F
:102160001B68134219D0114113410022994200DD2E
:1021700004323B1B1A600D4B3F1B1B780437002BAE
:1021800001D0FFF77EF92B68019A1C121340084A10
:102190009B009B580435FFF756F93B1F1A68022035
:1021A000FEF7F2FF3E1B3060E5E7C046A8020020C4
:1021B00070D000003B1F1B68A400043B5A1E9341D3
:1021C0003A1B17009B001360F44B04371B78002B5D
:1021D00001D0FFF756F92B68019A1C121340F04A00
:1021E0009B009B580435FFF72EF93B00083B18680D
:1021F000FFF722F83B1F06001868FFF71DF832189A
:102200000120A4003B1B1F00520002431A60E34B55
:1022100004371B78002B01D0FFF733F92B68019AA4
:102220001C121340DE4A9B009B580435FFF70BF944
:102230003B00083B1868FEF7FFFF3B1F06001868CD
:10224000FEF7FAFF321A0120A4003B1B1F005200C8
:1022500002431A60D14B04371B78002B01D0FFF7E3
:1022600010F92B68019A1C121340CD4A9B009B5811
:102270000435FFF7E8F83B00083B1868FEF7DCFF81
:102280003B1F06001868FEF7D7FF02000120A400DC
:102290003B1B1F007243520002431A60BF4B0437BE
:1022A0001B78002B01D0FFF7ECF82B68019A1C1269
:1022B0001340BB4A9B009B580435FFF7C4F83B1FF3
:1022C0001868FEF7B9FF061E17D11F23B34A137013
:1022D000A4003B1B1F001E60B04B04371B78002B73
:1022E00001D0FFF7CEF82B68019A1C121340AC4ABC
:1022F0009B009B580435FFF7A6F83B00083B186885
:10230000FEF79AFF310007F079F9012640000643F5
:10231000DEE73B1F1868FEF78FFF061E17D11F234D
:102320009E4A1370A4003B1B1F001E609B4B04378A
:102330001B78002B01D0FFF7A4F82B68019A1C1220
:102340001340974A9B009B580435FFF77CF83B00ED
:10235000083B1868FEF770FF310007F035FA0126D8
:1023600049000E43DEE73B1F1868FEF765FFC21702
:10237000801850400122A4003B1B1F004000104366
:102380001860864B04371B78002B01D0FFF779F8D3
:102390002B68019A1C121340814A9B009B580435FC
:1023A000FFF751F8A300FE1A07943068012C23D1DF
:1023B000FEF742FF049009F045FD0499002900DC76
:1023C000012107F001FA0C190121079B64000C435D
:1023D00034609E00714BBF1B1B780437002B01D06B
:1023E000FFF74FF82B68019A1C1213406C4A9B00B0
:1023F0009B580435FFF727F8FEF71EFF04007068AE
:10240000FEF71AFF0130031B0493D4E7A300FE1A62
:1024100031002000049301F043FD049B3060FF1A5B
:102420005E4B04371B78002B01D0FFF72AF82B688E
:10243000019A1C1213405A4A9B009B580435FFF71F
:1024400002F83B00083B1868FEF7F6FE3B1F06004B
:102450001868FEF7F1FE02000120A4003B1B1F00DC
:102460003240520002431A604C4B04371B78002B59
:1024700001D0FFF706F82B68019A1C121340484A56
:102480009B009B580435FEF7DEFF3B00083B1868B5
:10249000FEF7D2FE06003B1F1868FEF7CDFE3200A5
:1024A00002430120A4003B1B1F00520002431A609C
:1024B0003A4B04371B78002B01D0FEF7E2FF2B6864
:1024C000019A1C121340364A9B009B580435FEF7B4
:1024D000BAFF3B00083B1868FEF7AEFE06003B1F44
:1024E0001868FEF7A9FE320042400120A4003B1B01
:1024F0001F00520002431A60284B04371B78002B40
:1025000001D0FEF7BEFF2B68019A1C121340244A2B
:102510009B009B580435FEF796FF3B1F1868FEF79B
:102520008BFEC0430122A4003B1B1F004000104350
:1025300018601A4B04371B78002B01D0FEF7A1FF5F
:102540002B68019A1C121340154A9B009B580435B6
:10255000FEF779FF3B00083B1868FEF76DFE0600AA
:102560003B1F1868FEF768FE3200824051000122CE
:10257000A4003B1B1F000A431A60084B04371B785A
:10258000002B01D0FEF77DFF2B68019A1C1213402F
:10259000034A9B009B580435FEF755FFA802002014
:1025A00070D000003B00083B1868FEF745FE0600AF
:1025B0003B1F1868FEF740FE320002415100012225
:1025C000A4003B1B1F000A431A60DE4B04371B7834
:1025D000002B01D0FEF755FF2B68019A1C12134007
:1025E000D94A9B009B580435FEF72DFF3B000C3B5E
:1025F0001868FEF721FE3B00083B06001868FEF74E
:102600001BFEF1170200C317300007F02FF93B1F24
:10261000049005911868FEF70FFE020004980599D2
:1026200007F0D8F843000120A4003E1B37001843F0
:10263000C44B30601B780437002B01D0FEF721FF1C
:102640002B68019A1C121340BF4A9B009B5804350B
:10265000FEF7F9FEA300FE1A310020000493FEF7F6
:10266000D7FB049B3060FF1AB64B04371B78002B56
:1026700001D0FEF706FF2B68019A1C121340B24AE4
:102680009B009B580435FEF7DEFEA300FF1A3900BD
:102690002000FEF7D5FBAB4B1B78002B01D0FEF7DB
:1026A000F0FE2B68019A1C121340A74A9B009B580E
:1026B0000435FEF7C8FEA300FE1A31002000049383
:1026C000FEF7FEFB049B3060FF1A9E4B04371B781D
:1026D000002B01D0FEF7D5FE2B68019A1C12134087
:1026E000994A9B009B580435FEF7ADFEA300FF1AE4
:1026F00039002000FEF768FC924B1B78002B01D0BC
:10270000FEF7BFFE2B68019A1C1213408E4A9B00F5
:102710009B580435FEF797FEA300FE1A31002000F7
:102720000493FEF7C3FC049B3060FF1A854B04370B
:102730001B78002B01D0FEF7A4FE2B68019A1C1217
:102740001340814A9B009B580435FEF77CFE3B1FDB
:10275000186800F0FFFF3A00083A12680300A4006E
:10276000D10729D4042A0CD910680F22104001384F
:1027700008280FD806F0AEFE052026220E0E0E0EFB
:1027800024007249180009F0FDFB434258413B1BED
:10279000800018606B4B3F1B1B780437002B01D067
:1027A000FEF76FFE2B68019A1C121340664A9B00CD
:1027B0009B580435FEF747FE6549E3E76549E1E7C5
:1027C0006549DFE76549DDE7069B3E1DF31A5D4C71
:1027D000D82B03DD1A232370FEF753FE00F010FD03
:1027E00043000120184323783860002B02D03700C3
:1027F000FEF747FE2B68019A1C121340524A9B00B9
:102800009B5837000435FEF71EFE069B3E1DF31A4B
:102810004C4CD82B03DD1A232370FEF732FE00F058
:10282000E5FC4F4B400018400123184323783860E3
:10283000002B02D03700FEF724FE2B68019A1C12F1
:102840001340414A9B009B5837000435FEF7FBFDBF
:10285000069B3E1DF31A3B4CD82B03DD1A23237035
:10286000FEF70FFE00F0CCFC3E4B1A68831A904234
:1028700001D23D4A9B1801205B0003433B60237853
:10288000002B02D03700FEF7FCFD2B68019A1C12CA
:1028900013402D4A9B009B5837000435FEF7D3FDAB
:1028A00000F0AEFC2F4BA4001860264B3F1B1B789A
:1028B000002B01D0FEF7E5FD2B68019A1C12134096
:1028C000214A9B009B580435FEF7BDFD00F0A0FC9B
:1028D000A300002810D1FF1A1A4B1B78002B01D03F
:1028E000FEF7CFFD2B68019A1C121340164A9B007D
:1028F0009B580435FEF7A7FD3E00FF1A0123200078
:102900001A003900FEF7E6FC184C2068643002F02B
:1029100045FF002803D1043D3700FEF7C5FD039BAA
:1029200021685A78124803F06CFB0123039A137054
:1029300000F05CFC0F4B22681B68063253431818EA
:10294000FFF7EEF8A802002070D00000ACD2000023
:10295000B4D20000BBD20000C2D20000C7D2000037
:10296000FEFFFF7FD405002037894100CC05002001
:10297000A90200200400002000F04AFCA300002867
:1029800010D1FF1AF24B1B78002B01D0FEF779FD16
:102990002B68019A1C121340EE4A9B009B58043589
:1029A000FEF751FD3E00FF1A2000012300223900EE
:1029B000FEF790FCE84C2068643002F0EFFE00283F
:1029C000A9D0E64803F096F8AFE7A4003E1BFEF757
:1029D00001FD3700DE4B30601B780437002B01D03F
:1029E000FEF74FFD2B68019A1C121340D94A9B0039
:1029F0009B580435FEF727FDD54BA4001B783F1BE1
:102A0000002B01D0FEF73DFD2B68019A1C121340EC
:102A1000D04A9B009B580435FEF715FDA4003E1BD1
:102A2000300000F022FC3700C94B30601B780437BF
:102A3000002B01D0FEF725FD2B68019A1C121340D4
:102A4000C44A9B009B580435FEF7FDFCA4003E1BC6
:102A5000300000F00CFC3700BD4B30601B780437B1
:102A6000002B01D0FEF70DFD2B68019A1C121340BC
:102A7000B84A9B009B580435FEF7E5FCA300FE1AFC
:102A800031002000049300F0F5FB049B3060FF1A36
:102A9000AF4B04371B78002B01D0FEF7F2FC2B68FC
:102AA000019A1C121340AB4A9B009B580435FEF759
:102AB000CAFCA4003F1B380000F00EFCA44B1B789E
:102AC000002B01D0FEF7DDFC2B68019A1C1213408D
:102AD000A04A9B009B580435FEF7B5FCA300FE1AE4
:102AE00031002000049300F01FFC049B3060FF1AAB
:102AF000974B04371B78002B01D0FEF7C2FC2B68E4
:102B0000019A1C121340934A9B009B580435FEF710
:102B10009AFCA4003F1B380000F048FC8C4B1B784B
:102B2000002B01D0FEF7ADFC2B68019A1C1213405C
:102B3000884A9B009B580435FEF785FC0121200044
:102B400000F01CFC824B1B78002B01D0FEF799FC97
:102B50002B68019A1C1213407E4A9B009B58043537
:102B6000FEF771FC0021200000F008FC784B1B7878
:102B7000002B01D0FEF785FC2B68019A1C12134034
:102B8000744A9B009B580435FEF75DFCA4003E1B75
:102B9000300000F02DFC37006D4B30601B7804379F
:102BA000002B01D0FEF76DFC2B68019A1C1213401C
:102BB000684A9B009B580435FEF745FCA4003E1B69
:102BC000300000F029FC3700614B30601B7804377F
:102BD000002B01D0FEF755FC2B68019A1C12134004
:102BE0005C4A9B009B580435FEF72DFCA4003F1B5C
:102BF000380000F0EBFB564B1B78002B01D0FEF7A2
:102C000040FC2B68019A1C121340524A9B009B58AF
:102C10000435FEF718FCA4003F1B380003F058FDF4
:102C20004B4B1B78002B01D0FEF72BFC2B68019A35
:102C30001C121340474A9B009B580435FEF703FCC7
:102C4000A4003E1B300003F0DDFD3700404B306038
:102C50001B780437002B01D0FEF713FC2B68019A78
:102C60001C1213403B4A9B009B580435FEF7EBFBBC
:102C7000A4003F1B380003F0CDFC354B1B78002B24
:102C800001D0FEF7FEFB2B68019A1C121340314A5B
:102C90009B009B580435FEF7D6FBA4003E1B30007A
:102CA00003F0CEFC37002A4B30601B780437002B32
:102CB00001D0FEF7E6FB2B68019A1C121340254A4F
:102CC0009B009B580435FEF7BEFBA300FF1A39009A
:102CD000200001F047FC1E4B1B78002B01D0FEF7B3
:102CE000D0FB2B68019A1C1213401A4A9B009B5878
:102CF0000435FEF7A8FBA300FF1A3900200001F0FD
:102D000045FA134B1B78002B01D0FEF7BAFB2B685A
:102D1000019A1C1213400F4A9B009B580435FEF782
:102D200092FBA300FF1A3900200001F053FB084B6F
:102D30001B78002B01D0FEF7A4FB2B68019A1C1214
:102D40001340044A9B009B580435FEF77CFBC046A9
:102D5000A802002070D00000CC050020A9020020AD
:102D6000A300FF1A3900200001F05CFB894B1B789F
:102D7000002B01D0FEF785FB2B68019A1C12134033
:102D8000854A9B009B580435FEF75DFBA300FE1AA5
:102D900031002000049303F0CDFD049B3060FF1A46
:102DA0007C4B04371B78002B01D0FEF76AFB2B68A5
:102DB000019A1C121340784A9B009B580435FEF779
:102DC00042FBA300FE1A31002000049303F0BAFD79
:102DD000049B3060FF1A6F4B04371B78002B01D027
:102DE000FEF74FFB2B68019A1C1213406A4A9B00A6
:102DF0009B580435FEF727FBA300FE1A3100200084
:102E0000049303F0A7FD049B3060FF1A614B043765
:102E10001B78002B01D0FEF734FB2B68019A1C12A3
:102E200013405D4A9B009B580435FEF70CFBA30042
:102E3000FE1A31002000049303F058FB049B30601D
:102E4000FF1A544B04371B78002B01D0FEF719FBF7
:102E50002B68019A1C1213404F4A9B009B58043563
:102E6000FEF7F1FAA300FF1A3900200001F0C6F9BD
:102E7000484B1B78002B01D0FEF703FB2B68019A0F
:102E80001C121340444A9B009B580435FEF7DBFAA2
:102E9000A300FF1A3900200001F0ECFA3D4B1B782B
:102EA000002B01D0FEF7EDFA2B68019A1C1213409B
:102EB000394A9B009B580435FEF7C5FAA300FE1A59
:102EC00031002000049301F051FA049B3060FF1A96
:102ED000304B04371B78002B01D0FEF7D2FA2B6859
:102EE000019A1C1213402C4A9B009B580435FEF794
:102EF000AAFAA300FF1A3900200001F0FFF9254BC0
:102F00001B78002B01D0FEF7BCFA2B68019A1C122B
:102F10001340214A9B009B580435FEF794FA069B08
:102F2000039AFB1A9B101361A300FF1A39002000BB
:102F300002F01EFE174B1B78002B01D0FEF7A1FA02
:102F40002B68019A1C121340134A9B009B580435AE
:102F5000FEF779FA069B039AFB1A9B101361A300F4
:102F6000FE1A31002000049302F002FE049B306040
:102F7000FF1A084B04371B78002B01D0FEF781FAAB
:102F80002B68019A1C121340034A9B009B5804357E
:102F9000FEF759FAA802002070D000000023F7B510
:102FA0005A1E0192002B07DA01F0F2FA02F010FF2C
:102FB00003F086F81923019300263000194B196895
:102FC000B14212DD184B1A6801328A420FDAF0243E
:102FD0001A601D68154F6C43E35D002B1FD0E41988
:102FE000022B06D12000FEF70DFA019BD8E7002244
:102FF000EDE7012B0DD1002801D100F0F7F8F02208
:103000006A43BB185B680A49C31A8B4201D8022382
:10301000BB54F0235D43054BEB5C022BE2D0013641
:10302000CCE7C046D0050020000000203C1C00205A
:103030003F420F00012200210A4B0B481A61195030
:1030400004301950A2210420C9005850C121C020C9
:103050008900800258501A60044BFC311960044BFF
:103060001A70704700A000400405000000E100E075
:10307000FB05002004207047F8B550C90123220049
:103080001A40101E2DD03340181E2AD06410002084
:103090001C2C26D81D4B761035009E4200DD1D00ED
:1030A0001B4F3B5D012B05D00121200004F002FEE7
:1030B00001233B55174B1B78002B01D1FFF7BAFFBB
:1030C0000023154A9E420DDCFF2514491448D65CA6
:1030D000B44202D15E007052D5540133042BF6D1B4
:1030E0000420F8BDD15C8C4203D10C4A5B009D5298
:1030F000F6E70133042BF5D10023D15CFF2901D180
:10310000D454F2E70133042BF7D1E9E78813000028
:10311000DC050020FB0500201C0000200E00002024
:10312000DC05000070B530C9012322001A40101ED2
:103130001BD02B40181E18D064101C2C00D9002462
:10314000174E335D012B05D00121200004F0B2FDA4
:103150000123335569100800124A1038124B90426F
:1031600004D9012252421A60042070BD1C600F482D
:1031700006F044FA0E4B18800E4B1B78002B02D140
:10318000FFF758FFF0E701220B4B9A64A922D20007
:103190009A588018A82280B2D2009850E4E7C0461E
:1031A000DC050020908601001800002020A1070007
:1031B0000C000020FB05002000A00040030010B51B
:1031C0000120002B02DC1B30FEF7FEF810BD0420AE
:1031D000704710B5002803DC1C20FEF7F5F810BD81
:1031E0000B680020DB07FAD40D30F6E70122034B11
:1031F0001A64A822D20098587047C0460080004048
:1032000010B5FFF7F3FFFA21890006F06DF910BD44
:10321000012070470048704724D300001D207047EC
:1032200070B5054E0400335C0D008B4202D004F0F3
:1032300041FD355570BDC046DC05002070B5002449
:10324000084D635D012B09D10021200004F050FDE1
:103250000021200004F02EFD0023635501341D2CB5
:10326000EED170BDDC05002070470D2070473B207B
:1032700070470000F8B501240B6806000D002342DA
:1032800004D10D20FEF7A0F82000F8BD5B1020004F
:10329000052BFAD80E4A9B009C580E4F3B5D002B25
:1032A00005D00021200004F005FD00233B55012E30
:1032B00006DD6B68042B03D10221200004F0FAFC28
:1032C000200004F0A5FB012440002043DDE7C046B8
:1032D0000CD30000DC050020F8B501260568354256
:1032E00002D04468344203D10D20FEF76DF8F8BDDA
:1032F0006D101C2DFBD80A4F7B5D012B04D03100D3
:10330000280004F0D7FC7E55064964108C4202DC8C
:10331000E143C9172140280004F000FCE7E7C0465C
:10332000DC050020FF03000070B501240D68254274
:1033300004D10D20FEF748F8200070BD6D101C2D43
:1033400017D80024012804DD4C68043C63425C412A
:103350006400094E735DA34204D02100280004F0EC
:10336000A9FC7455280004F0D9FC03000420012BAB
:10337000E3D00020E1E7C046DC05002070B5040082
:103380000D001C280ED8084E335C012B04D00121FF
:1033900004F090FC01233355290020004D1EA94163
:1033A00004F0A6FC70BDC046DC050020036810B523
:1033B000DA0703D40D20FEF707F810BD4168581056
:1033C00004394A425141FFF7D9FFF6E737B569465C
:1033D0000A00064B30CB30C203680220042B02D116
:1033E00000F0F8FF37BD01F01DF8FBE7D4D2000074
:1033F00010B5084C6379002B05D00021052004F09E
:1034000059FC00236371052004F088FC43425841B5
:10341000800010BDDC05002010B5084CE37A002BBD
:1034200005D000210B2004F045FC0023E3720B20A3
:1034300004F074FC43425841800010BDDC050020BC
:1034400070470000F7B5304D304E6B6C002B15D037
:10345000A8240023E40037596B642D4B186800281A
:103460000CDB2C4B19784A425141C9B2197004F057
:103470003FFC294B1B88DF19BFB23751AB6C002BC7
:1034800039D00021254B264FF458A9643A780C34E2
:103490000193244D8A4206D02B68032B03D8224A7D
:1034A000D05C04F025FC2B68204A0133134004D57E
:1034B0000422013B5242134301331B4900228C4634
:1034C0002B60042B18D06046C05C591CFF2802D129
:1034D0000B000122F5E7002A00D02B60012104F047
:1034E00007FC01233B702B68114A5B009B5AE418D0
:1034F000019BA4B2F450F7BD01235B422B60002373
:103500003B700C4BF3E7C046FCA0004000A000401D
:1035100018000020FA0500200C00002044050000DF
:10352000F9050020D80500201C00002003000080C1
:103530000E00002050460000084B094AFF201A8068
:103540005A809A80DA800023064A07491370074A96
:10355000087048708870C870136070470E000020B3
:10356000DC050000F90500201C000020D805002023
:103570000122024B52421A607047C04618000020D8
:1035800010B5034A0621034802F0CEF810BDC0462C
:10359000DCD20000CADA0000E12170B54902194806
:1035A00003F0ACFF002401220320174B17491A61D6
:1035B0005C50043158508018083158501A60063059
:1035C00004F020FAFF21124AA15401341D2CFBD132
:1035D000012200200F4B01001A6004230E4A0F4DF8
:1035E0001468002CFCD02C680002013B20431160C1
:1035F000002BF5D101220A4B1A6004F03BF901F0CF
:1036000013F970BDC41B00200080004004050000B9
:10361000DC05002000D0004000D1004008D500406B
:1036200004D00040F8B50B4E070030000D0003F049
:10363000ADFF0400A84200DD2C003D00EB1B9C42C6
:1036400005DD300003F0ACFF28700135F6E72000FF
:10365000F8BDC046C41B002010B50100014803F0AE
:1036600055FF10BDC41B002010B5054C200003F011
:103670005BFFE1212000490203F040FF10BDC0467E
:10368000C41B0020C3070CD4064B1B68834208D818
:10369000054B1B68984204D8031F1B68002B00D001
:1036A00018007047040600200006002000230122B5
:1036B00010B50A48990001334250642BFAD1084CE6
:1036C000084B00211A602000074A08F0DBF8074B7E
:1036D000074A6360074B1A6010BDC046942D002056
:1036E0000806002008000020D40900003027000050
:1036F0000C060020FC05002010B5044B044A1A609B
:10370000044B054A1A60FFF7D1FF10BD04060020E4
:103710000806002000060020DC0F0020044B1B6878
:103720001868000980B20238C343DB17184070479D
:10373000FC05002000B59BB00200054901A808F077
:10374000E5FB01A802F0F2F902F0BAFCFCE7C04682
:10375000A8D300000B4BC20704D4042804D80A4B9A
:1037600000D00A4B180070470F2203681A40031D4F
:10377000042AF7D0064B092AF4D0064B032AF1D0CD
:10378000054BEFE782D3000026CF000020CF0000DA
:103790008CD300009CD3000093D300000020064A85
:1037A0000649131F186013681B099BB202339B0064
:1037B000D2188A42F5D370470C060020DC0F002097
:1037C000F7B50F240126314B314A1968314B324D80
:1037D000186813681F002740072F26D813681B0995
:1037E0009BB202339B00D218AA42F2D300242B4E84
:1037F000A500AD192868FFF745FF01342860642C47
:10380000F6D1274C2068FFF73DFF2060254C20684B
:10381000002802D0FFF736FF20600025224B1B68EE
:103820000093009B9D4214DBF7BD1B099BB29B00DC
:10383000D3189A42D2D01F68374208D1B94206D273
:10384000B84204D3043F3F68002F00D01F60043B00
:10385000EFE7F0236B43154A9B181A78002A01D131
:103860000135DEE71F693C2300266B43DB199B0013
:1038700001930136BB1BF3D4019BB4001C1B0B4B03
:103880001C19A069FFF7FEFEA061F2E70406002004
:103890000C06002000060020DC0F0020942D0020E4
:1038A00008000020DC0F0020D00500203C1C002078
:1038B000F7B50124204246D1234B1B689C46984211
:1038C00041D3224B1B68019398423CD8031F1B68CD
:1038D000002B38D10200036800941B099BB2002B17
:1038E0000FD10099131F196090422CD015682B1F1F
:1038F0001B68990069180C68013B14600A602A0073
:10390000EDE79D0055192968009C214219D18C458D
:1039100017D8019C8C4214D30E1F3468002C10D190
:103920000F680F343C40072C08D92F60151F2B60FF
:103930000B680A601B099BB20A00D0E7009931604E
:10394000CDE7013BCBE7F7BD0406002000060020D1
:103950000D4970B50A000D4D1368141F1B09266828
:103960009BB2981C002E0BD000238A4200D00B0083
:1039700023608300C91880001218AA42ECD370BDDE
:103980001B011360F7E7C0460C060020DC0F002087
:10399000F8B5124C27000F223B681D09ADB2134247
:1039A0000DD06E1CB600A74204D0320039002000B2
:1039B00007F055FF0022A3190436A4191A60023536
:1039C000AD00074B7F199F42E5D31B1B9B10013BAA
:1039D0001B012360034B1C60F8BDC0460C06002091
:1039E000DC0F0020FC050020F0B59BB0FFF7FEFBCC
:1039F00000240700214AA300D0580134FFF758FFE4
:103A0000642CF7D11E4B1868FFF752FF1D4B186846
:103A1000002801D0FFF74CFF00261B4B1B689E427D
:103A200017DBFFF795FFFFF7CBFEFFF7B1FFFFF7BF
:103A3000DDFB164BC21B1B6815491B6801A81B093F
:103A40009BB2023B08F062FA01A802F06FF81BB0CB
:103A5000F0BDF02575430F4BED182B78002B01D1ED
:103A60000136DAE72B695C1E002CF9DBA300EB18AA
:103A70009869FFF71DFF013CF6E7C046942D002032
:103A800008000020DC0F0020D0050020FC050020ED
:103A900062D300003C1C0020F7B5174D4F1C2B686B
:103AA00006001B680C001B099BB201929F420BDBB6
:103AB000FFF79AFF2B681B681B099BB29F4203DB31
:103AC0000A20FDF781FCFEBD2868A71CBA00DB1B9D
:103AD00081181B010B6029600021031F19600F234F
:103AE0001E4003002401264340C3083A9A189A4214
:103AF000E9D9019902C3FAE7FC050020F7B50300F4
:103B00000122134004000D000193002B2BD1174B11
:103B10001B68834227D8164B1B68834223D90F2387
:103B2000144F386000681840FFF7B6FF019B3C68EF
:103B3000061E3B6017D0236804301B099BB29D42D0
:103B400000DD1D00AA00211D251F07F07FFEFFF7E5
:103B500025FE2E60FFF734FE00232B602268064B03
:103B60001340236034002000FEBDC0460406002040
:103B700000060020DC0F0020F0FF0F0003230430BC
:103B800010B5C11719400918891000220420FFF749
:103B900083FF10BD70B5050008000C00FFF7EEFFB5
:103BA0000023002804D170BDE95CC21811710133F3
:103BB000A342F9DBE343DB171C4000230419237104
:103BC000F1E7F0B50C009BB0022804DC1C20FDF7E7
:103BD000FBFB1BB0F0BD01230868184206D1042886
:103BE00004D90F2601683140042901D00E20EEE7E8
:103BF00061680D001D40F9D10429F7D90A683240E7
:103C0000042AF3D1A2681A4201D10D20DFE7FFF7A1
:103C1000A1FD06006068FFF79DFDA768010001ACEB
:103C20007F103000257003F076F8390064232200FD
:103C300003F0D6F8200008F0AFF901002000FFF7EC
:103C4000A9FFC6E710B51C4CA544041E02D1FFF71E
:103C500095FF0BE002F078FF0138062828D805F020
:103C600039FC090911182904240000208023DB00F5
:103C70009D4410BD200002F0E3FF011B2000FFF770
:103C800089FFF3E7200002F089FF43000120184379
:103C9000ECE780226946D200200002F096FF6846D9
:103CA00008F07AF901006846E9E704210348E6E7ED
:103CB0000020CCE70420D9E700FCFFFFF0D3000090
:103CC00070B50C00022803DC1C20FDF77DFB70BDE5
:103CD00001230868184206D1042804D90F25016879
:103CE0002940042901D00E20EFE761681942FAD17A
:103CF0000429F8D90A682A40042AF4D1A2681A4291
:103D000001D10D20E1E7FFF725FD05006068FFF711
:103D100021FDA46801006410280002F0FCFF2100CE
:103D200003F039F8FFF78EFFD1E770B50D000128D9
:103D300003DC1C20FDF748FB70BD0124086820420D
:103D400006D1042804D90F2102680A40042A01D0B0
:103D50000E20EFE76A682242FAD1042AF8D91368E4
:103D60000B40042BF4D1FFF7F5FC06006868FFF761
:103D7000F1FC0100300002F0CEFF03F050F84000EB
:103D80002043D9E7F8B507000C001C20012F0BDDFC
:103D900001250868284206D1042804D90F210268A9
:103DA0000A40042A03D00E20FDF70EFBF8BD62681E
:103DB0002A42F8D1042AF6D913680B40042BF2D119
:103DC000FFF7C8FC06006068FFF7C4FC0100022F83
:103DD00014D0A4682C4211D06410300002F09BFF74
:103DE000050002F0B1FE012811D1002C02DD0135E1
:103DF000012C06D12800FFF725FFD7E701246442F4
:103E0000EBE7280002F028FF013C0500F0E702285C
:103E1000F0D1002CEEDD0135012CEBD00022280082
:103E2000110002F04BFF02F017FF013C0500F3E721
:103E300010B501240868044016D04410200005F095
:103E400071FE154905F03CFD07F022FC04F074F802
:103E50000022124B06F0D6FD04F016F807F0A8FB7E
:103E600043000120184310BD042810D90F23026815
:103E70001340042B07D1FFF76DFC21000A2208F044
:103E800053F90400DAE7032B01D10430F5E70D20E4
:103E9000FDF79AFAD2E7C046D30237390000D04086
:103EA000086870B501240500254006D1042804D90E
:103EB0000F2302681340042B03D00E20FDF784FA71
:103EC00070BDFFF747FC03782900233B5A4253415A
:103ED0001022C01808F028F980239B05C218044B53
:103EE0009A4201D91420E9E740002043E8E7C046A0
:103EF000FFFFFF3F10B5034A0621034801F014FC01
:103F000010BDC046C0D30000B9D3000000207047E8
:103F100010B51E20FDF758FA10BD10B51E20FDF794
:103F200053FA10BD10B51E20FDF74EFA10BD10B5A6
:103F30001E20FDF749FA10BD10B51E20FDF744FA0A
:103F400010BD10B51E20FDF73FFA10BD10B51E20A4
:103F5000FDF73AFA10BD10B51E20FDF735FA10BD79
:103F600010B51E20FDF730FA10BD10B51E20FDF76C
:103F70002BFA10BD10B51E20FDF726FA10BD10B5A6
:103F80001E20FDF721FA10BD10B51E20FDF71CFA0A
:103F900010BD10B51E20FDF717FA10BD10B51E207C
:103FA000FDF712FA10BD10B51E20FDF70DFA10BD79
:103FB00010B5034A1121034801F0B6FB10BDC046FD
:103FC0002CD40000B4D400000120034B1860034B34
:103FD0001B6883401843704700100020E00F00204A
:103FE000F0B5EFF310810123194083F31088134CCF
:103FF000134AA4461268134E013A9340124F134AD3
:10400000002B17D0146803420FD03D682C60C046C7
:10401000C046C046C046C046C046C046C0460C4C1E
:104020001568246825605B08EAE765462C6014681B
:104030003460F8E781F31088F0BDC04608050050F1
:10404000200000200C050050EC0F0020F40F002091
:10405000E80F002030B585B001AD0C2206492800DC
:1040600007F0F4FB0024285D01210134FFF7D8F8A4
:104070000C2CF8D105B030BD9DD50000F7B56A46CF
:104080003B4B01AE13800A2393703A4B33801C23C1
:10409000B370FFF7ABF8384B384DC0182B68984217
:1040A00001D200232B602C68002C41D1375D012107
:1040B0003800FFF7B5F801340021380003F018FE8E
:1040C000032CF3D1002401276B461E5D390030001C
:1040D000FFF7A6F801343900300003F009FE032C85
:1040E000F2D1C8200138C046C046C046C046C046CE
:1040F000C046C046C046C046C046C046C046F1D1D4
:104100006B4600211878FFF78BF86B460021587832
:10411000FFF786F86B4600219878FFF781F8FFF7E4
:1041200065F8FA2300241B01C01828602000FEBD9A
:10413000FFF75CF82B6800249842F7D3032003F0C4
:1041400067FC0600042003F063FC36180A2003F025
:104150005FFC0B4B9B1B181A0A4BA04206DB186036
:104160000023094A2B6013600124DFE71C60F7E796
:10417000030400001A1B000010270000F80F0020A5
:10418000E3030000E00F0020001000200022054B98
:1041900010B51A60044B1B68934201D002F074FC06
:1041A000002010BDFC0F0020E81A002010B5041EEE
:1041B00010DA00240A4BA400E25801239340094A74
:1041C00009491360094A1160094A0A4911600A4AFB
:1041D000136010BDFFF722F8A042EADDEAE7C0460F
:1041E000D8E20000F40F002008050050EC0F00207A
:1041F000E80F00200C05005018050050F0B53B4BAF
:1042000085B01B680C00002B03D101204042FFF752
:10421000CDFF246801222700174028D0FF23601219
:10422000184033496714661040431F401E4005F094
:10423000E5F9050438002E49784305F0DFF900025E
:10424000054330002A49704305F0D8F9294B28432B
:104250001B68202B06D16400A40E274BA400E35852
:1042600000021843FFF7BCFE002005B0F0BD042C8F
:10427000FAD90F2321680B40092BF5D1636803920B
:104280005B100193019B9F42EEDABB00E3189E682E
:10429000039B1E4228D0FF237012184072101A4050
:1042A0001349751440431D40009205F0A7F903041B
:1042B00028000F496843029305F0A0F9029D00020F
:1042C000054300980A49404305F098F9094B2843F3
:1042D0001B68202B06D17600B60E074BB600F558AA
:1042E00000022843FFF77CFE0137CBE7F40F0020E4
:1042F000590600002000002084D700000200086852
:1043000010B5C3070FD540101823012A03DD4A68F2
:10431000042A00D10833054A1360FEF7A5FFFFF712
:1043200045FF002010BD01204042EDE720000020A5
:1043300010B50124044002D04410200010BD042810
:1043400010D90F2302681340042B07D1FFF702FA9C
:1043500021000A2207F0E8FE0400EEE7032B01D15A
:104360000430F5E70D20FDF72FF8E6E70868F8B50B
:10437000C3071AD5FFF7DCFF0300203B5E2B25D8CF
:104380000520434301221D180020114E9D4219D0E3
:1043900005211024F75C3C4200D0801801395200FE
:1043A00064100029F7D10133F0E704280ED90F2259
:1043B00003681A40042A09D11B099BB2002B05D0BF
:1043C0000379DAE7012340001843F8BD0120FCE738
:1043D000A9D5000070B508680D00FFF7A9FF04001B
:1043E0006868FFF7A5FF621E0100042A14D8451E65
:1043F000042D11D805236B439B18012215009D4005
:104400002B00064805682B430360054B1B68002BF7
:1044100002D0200002F039FB002070BDFC0F00200C
:10442000E81A002070B508680D00FFF781FF04004E
:104430006868FFF77DFF621E0100042A13D8451E3D
:10444000042D10D805236B439B1801229A4007487E
:10445000036893430360064B1B68002B03D00022C4
:10446000200002F012FB002070BDC046FC0F0020AF
:10447000E81A0020F0B5050089B008680C00FFF7C5
:1044800057FF0690022D36DD6068FFF751FF01905F
:10449000A068FFF74DFF04000127231D661E079348
:1044A000731C0293079B9E4235D0052373430593EB
:1044B000019B019D05330493049BAB421ED0042E47
:1044C00016D86B1E042B13D80122059B2349013BF0
:1044D0005B199A409446224A0B681068069A3A4043
:1044E00003920DD062461A430A60012200280DD1C2
:1044F0007F000135E0E701240194CDE7029ECFE77C
:10450000624693430B600028F2D0039A0299280078
:1045100002F0BBFAECE7019B1E1D042E1AD8012CF9
:1045200018D1002505273B0021006B439B199940BA
:104530000B000A4A013511689943094B11601B6849
:10454000002B05D0019B0022581D290002F09DFA86
:10455000052DE8D1002009B0F0BDC046FC0F0020B9
:10456000E81A0020086810B5C30703D5FFF7E0FE7E
:10457000054B1860054B1B68002B03D0024B1868D5
:1045800002F084FA002010BDFC0F0020E81A002081
:104590007FB5A04C2368002B0AD19F4A1268002ADD
:1045A00006D19E4B1B68002B01D0FFF767FD7FBD36
:1045B0009B4D2A68002A26D1984A1268002A1BD0EF
:1045C000FFF75CFD0028F2D0FFF744FD924B246812
:1045D0001A681C60002A16D0002C14D101AD0C22E0
:1045E0009049280007F032F9285D00210134FEF7D8
:1045F00017FE0C2CF8D1DAE7874A1268002AE5D1B9
:10460000002BE3D0E0E700211A2003F071FB00212A
:104610001B2003F06DFB00211C2003F069FB2E68BA
:10462000012E5CD0022E00D1A2E0002E50D1013626
:104630003100794C03202368994303F059FB04208F
:10464000216801404B42594103F052FB102123687D
:104650000A2019404B42594103F04AFB802123684C
:10466000090119404B425941062003F041FB8021CA
:104670002368090219404B425941072003F038FBD7
:1046800080212368490219404B425941092003F017
:104690002FFB80212368890219404B425941192080
:1046A00003F026FB80212368C90219404B4259417F
:1046B000182003F01DFB802321681B0319404B4287
:1046C0005941172003F014FB31001A2003F010FBAE
:1046D0002B680321581C05F077F8296067E7022151
:1046E0004D4C1720236819404B42594103F000FB01
:1046F00008212368182019404B42594103F0F8FA69
:1047000080212368C90019404B425941042003F01D
:10471000EFFA80212368490119404B4259410A2090
:1047200003F0E6FA80212368C90119404B42594140
:10473000032003F0DDFA80212368890319404B42EE
:104740005941092003F0D4FA802321681B04194041
:104750004B425941192003F0CBFA3100062003F0F7
:10476000C7FA3100072003F0C3FA31001B20ADE780
:104770002021294C1720236819404B42594103F04E
:10478000B7FA40212368182019404B42594103F0E1
:10479000AFFA80212368192019404B42594103F098
:1047A000A7FA80212368490019404B42594109204A
:1047B00003F09EFA80212368890019404B42594139
:1047C000072003F095FA80212368890119404B42A4
:1047D0005941062003F08CFA8021236849031940CF
:1047E0004B4259410A2003F083FA80212368C90310
:1047F00019404B425941032003F07AFA8023216883
:104800005B0419404B425941042003F071FA012125
:104810001C205BE7FC0F0020F00F002000100020A0
:10482000E40F00209DD50000012010B54042FFF7A5
:10483000BDFC10BD10B5034A0921034800F074FF08
:1048400010BDC04684D80000CCD800008023F0B54D
:1048500002255B051A690A4C0A4BA1261D51032744
:104860008025F600ED00BA43884202D300221A5197
:10487000F0BD5F59002FFCD098518018F4E7C04676
:104880000405000000E0014010B5002806D1C0205A
:10489000B02140028902FFF7D9FF10BDB02080216E
:1048A0008002C902F7E7000043425841064B4042EC
:1048B0001840B0239B02C018036800201A0E532A28
:1048C00001D11B02180A704700C0FEFF30B5012459
:1048D0008025054B054AED009C505C59002CFCD00E
:1048E00001600021995030BD00E001400405000046
:1048F00043425841074B40421840B0239B02C01826
:10490000A62310B50902DB05090A1943FFF7DEFFEC
:1049100010BDC04600C0FEFFF0B5012480260D4B3F
:104920000D4DF6005C51002902DC00225A51F0BD09
:10493000577814783F022743947824042743D47887
:10494000043224063C439F59002FFCD010C001398B
:10495000E9E7C04600E001400405000070B505002D
:104960004B680A009C1C2100A400FFF7D5FF281902
:1049700070BD0000134B1B68002B0CD08022B023AD
:10498000D2029B0200280BD11A1D5B681B0E522B12
:1049900000D110007047B022C02392025B02F1E701
:1049A00082420DD903681B0E522B09D14368023392
:1049B0009B00C018824203D903681B0E522BE9D01A
:1049C0000020E7E704110020F0B50020B7B0002474
:1049D000FFF7D0FF270005002600002D2ED1284D1F
:1049E0002868FFF761FF32003B00019000942549E1
:1049F00004A807F08BFA04A801F098F8224B642071
:104A00001C682B68A0215A425341204A5B42134044
:104A1000B02292029B18E41A6043490204F0EEFDB2
:104A2000A0225202030000921949220004A807F0B4
:104A30006DFA04A801F07AF837B0F0BDFF226B6878
:104A400029689C460233FF180B12013613409C4222
:104A500000DA1C00FF200A14024003926246014063
:104A600001920091039A0B4904A807F04FFA04A899
:104A700001F05CF82800FFF77DFF0500ADE7C046B8
:104A800004110020D6D900000811002000C0FEFF4C
:104A900080D90000C2D9000070B50020FFF704FFE4
:104AA00004000120FFF700FF844200DA04000A4BF3
:104AB0001D686A42554128001D60FFF7E5FEA022EF
:104AC0006B4252021340054A28009B18044A611C9D
:104AD0001360FFF70DFF70BD04110020048001007A
:104AE00008110020F8B50020FFF7DEFE07000120C6
:104AF000FFF7DAFE3E00204D0643204C0DD1802109
:104B0000C020C9024002FFF7A1FE01213000FFF7DB
:104B1000EFFE1B4B2E6023601DE0874209DD002362
:104B2000B0212B60164B89022360236800200125E9
:104B300017E0012380212B60124BC9022360F4E7A8
:104B4000120E522A08D0002800D023600E4800F030
:104B5000EDFFFFF7A1FFF8BD28005A68023292006E
:104B60009B188B4205D21A68561CE9D10028F2D056
:104B7000D1E72160EFE7C0460411002008110020B2
:104B80000480010004C002009BD9000070B5002021
:104B9000FFF7F0FEFF260500002801D1280070BDB8
:104BA00003681C143440FFF7E5FEDA2CF4D105004D
:104BB000F2E700008022F0B55200A1B00021674862
:104BC00006F060FE802200215200654806F05AFE81
:104BD000644BFF271B681A00049353425A4110008C
:104BE0000592FFF751FE049C0020631E9C415E4B22
:104BF00064421C405D4BE418FFF7C8FF0600002E1E
:104C00002DD10498FFF750FE411C0598FFF770FE68
:104C1000059A574D534B2C601A60FEF725FD514BFA
:104C200064201B68A0215A4253414F4A5B42134003
:104C3000B0222C6892029B18E41A6043490204F0E7
:104C4000DDFCA0225202030000924A49220007A87C
:104C500007F05CF907A800F069FF21B0F0BD3268E9
:104C6000131412123A403B4003921A000A3A092ADE
:104C700049D83A4B039A995C002931D110223E4819
:104C800006F000FE35002B6803991A123A40914253
:104C900009D11A143A400B2A27D0132A2DD00A2AF8
:104CA00001D1354B1D602800FFF764FE051EEAD1D7
:104CB000314B196800290FD02000FFF74FFE040088
:104CC0002D4B5B195968002903D02000FFF746FEE1
:104CD000040004350C2DF3D1204B0121039A995483
:104CE0003000FFF747FE060089E73B40022BDADC85
:104CF000214A9B00D3185D60D5E7102200211E4891
:104D000006F0C0FDCFE71A00153A082AE8D8144A81
:104D10000399525C002AE3D13500152B00D0150011
:104D2000300003681A143A40152A0FD01D2A00D10A
:104D30000025FFF71FFE0028F3D1002D04D020002E
:104D40002900FFF70BFE0400054BC6E7039A1B1270
:104D50003B409A42EDD10500EBE7C046041000202D
:104D60000C1100200411002000C0FEFF04C002004E
:104D70000811002065D90000242F002010B5FFF78E
:104D800019FF10BDF0B585B0039203220333DC1781
:104D9000294D1440E4182B68284F5A425341802271
:104DA0005B42D202A4103B409B18A21C0291244EED
:104DB000910000910190316800980A18934215D231
:104DC000FFF7F8FE2B685A42534180225B421F4096
:104DD000D202BF183368009A9B189F4206D2194826
:104DE00000F0A4FE0025280005B0F0BD029B356848
:104DF00019066B461A7BA423DB051343FF222F0001
:104E0000090C1943019B12041B0413401943280089
:104E1000FFF75CFD0837281D21003760FFF756FDBE
:104E2000002C04D00A9A21003800FFF775FD009B82
:104E3000083BFF183760D6E70411002000C0FEFFD2
:104E4000081100203FD9000070B59AB0FFF74AFE64
:104E5000FF221E4CD2000021200006F013FDFF258A
:104E6000FFF794FE0026002814D10200C300E35887
:104E70000130591E8B41D218FF28F7D1144901A8DF
:104E800007F044F801A800F051FE124800F04EFE71
:104E90001AB070BD03681A142A400A2A0AD11A12DD
:104EA0002A40FF2A03D0D200A1180B71A050FFF7AF
:104EB00061FDD8E7132AFAD11B122B40FF2BF6D045
:104EC000DB00E2181671E650F1E7C0469C25002091
:104ED0000BDA00001FDA00000021094B094A596073
:104EE0000131516059680029FCD00021196101236A
:104EF00093600222044B8131FF315A501A6070478F
:104F0000FC1000400010004000E100E00222064BCF
:104F10000121DA670022054B5A61054A11615A697D
:104F2000002AFCD07047C04604E100E0FC100040BD
:104F30000010004010B5044C2378002B01D0FFF77F
:104F4000E5FF0020207010BD0D12002080230120FD
:104F50005B055B6E5B001843704700000120024B4D
:104F60001B685B0018437047901200200120024B21
:104F70001B685B0018437047240000200120024B8F
:104F80001B685B00184370479412002070B5040042
:104F90000D001600FEF734F9802301215B055A6EDF
:104FA0002670002653006170E1706272010A5A0A8D
:104FB0006071A171A272010C5A0C000E5B0EA670FA
:104FC0002571E1712072E272237370BD10B5044C3B
:104FD000200006F0E1FF01002000FEF7DBFD10BD20
:104FE000991200200E4B10B51B680E4C5A1C0FD0A6
:104FF0000D4C002B0CD00D4C012B09D00C4C022B6E
:1050000006D0094C042B03D00A4C052B00D1074CC9
:10501000200006F0C1FF01002000FEF7BBFD10BD1F
:1050200028000020B0DA0000B4D20000BBDA000093
:10503000BBD20000B5DA000070B5214C2278002AFE
:105040003DD1204B01215A608022D20511605A685F
:10505000002AFCD0002207201B4B1C4901255A5076
:105060000439585008315A5019481A4958501A49A9
:105070001A485A501A495A50A622D2009D50082266
:1050800018495A50043158500220174958501749AE
:105090001748585017480439585018201649585086
:1050A000C12189005A500539FF39585892180243D6
:1050B0005A501249124A9950FFF70EFF257070BDE1
:1050C0000D120020FC000040001000400C05000004
:1050D000746962751C0500002405000020000402AC
:1050E0002C05000014050000340500003C050000FC
:1050F000FFFF000021100100540500000E120020E7
:105100000405000070B50E4B06001B78002B01D182
:10511000FFF792FF00200B4D2C7884420ED00A4BF3
:10512000202219780323091B1940084B4901C9188B
:10513000300006F08BFB0120013C2C7070BDC04696
:105140000D120020981200200C1200200E120020D8
:10515000002370B588B0984235DD0D6801262C001B
:1051600034409C422FD12300042D2CD90F222B68D0
:105170001A402300092A26D16A683F2A23DD68469F
:10518000FFF7C0FF230000281DD06B4619783300BD
:10519000A14203DB6B461B5D5B003343A200AA18F0
:1051A00001349360202CF2D1092169444A780B78AC
:1051B00012021A438B781B041A43CB781B06134345
:1051C000024A13600423180008B070BD9412002036
:1051D00070B5454B8AB01B78002B01D1FFF72CFF2F
:1051E00002AC2000FFF78EFF002802D100200AB099
:1051F00070BD23780B2BF9D96378012BF6D1E378B6
:10520000012BF3D100231120384E394D33602B7020
:1052100068442379374A41781360027809021143C0
:10522000827812041143C27812060A4332490A6096
:10523000002B0ED1152169444A780B7812021A43CB
:105240008B781B041A43CB781B061343336000236F
:1052500018E0012B1AD1152169444A780B78120203
:105260001A438B781B041A43CB781A211B0613436D
:1052700033600E23627C6944934200DD13000022F8
:105280009A422CD100220420EA54B0E7022B03D129
:10529000627B10331621EEE7042B0DD11521082275
:1052A0006944684606F0D2FA0098019902F05CFD64
:1052B00006F07EF93060CAE7052BC8D11521082217
:1052C0006944684606F0C2FA0098019902F04CFD64
:1052D00006F06EF93060627D0A231E21CBE7885C00
:1052E000A8540132CCE7C0460D12002090120020D5
:1052F00099120020280000209412002010B5134BB2
:1053000004001B78002B01D1FFF796FEFFF7FEFD8E
:1053100000200F4A0F49104B545058600130106064
:1053200058680028FCD0002018610130906018698E
:105330000028FCD0094B0A481B785B011B1853500E
:10534000FFF7E4FDFFF7C8FD10BDC0460D120020B9
:105350000010004004050000FC1000400C1200206A
:105360000E12002010B588B000281DDD0A6801214A
:1053700013000B4018D1042A16D90F2014682040BE
:10538000092811D150683F280EDD98001018806858
:105390000024084201D04010C4B26846C45401330E
:1053A000202BF2D1FFF7AAFF002008B010BD0000AB
:1053B00010B5002813DD0C68E30710D56410532CDA
:1053C0000DD8084B1B78002B01D1FFF735FEFFF7F6
:1053D0009DFDA123044ADB00D450FFF77DFD002092
:1053E00010BDC0460D1200200010004010B500286E
:1053F0000EDD0C68E3070BD56410FF2C08D8054BB5
:105400001B78002B01D1FFF717FE034A034BD45042
:10541000002010BD0D1200200010004024050000E7
:1054200013B5002814DD0C68E30711D5094B64108F
:105430000093094B0193072C0AD8084B1B78002BCB
:1054400001D1FFF7F9FD6B46054A1957054BD150BD
:10545000002016BDE2ECF0F4F8FC00040D12002070
:10546000001000400C05000070B588B0002820DD59
:105470000124086804401CD104281AD90F230268AB
:105480001340042B15D1FEF765F9060006F084FDE4
:105490000500122800D912252A0002210D32684683
:1054A000FFF774FD6B465D73A54205DC6846FFF7A8
:1054B00025FF002008B070BD2300325D6B449A7355
:1054C0000134F1E7F0B50D008BB0012832DD08683A
:1054D0000122040014402DD104282BD90F23016888
:1054E0000B40042B26D16B68134223D0FEF732F910
:1054F0006E6807007310019306F04EFD05000E283C
:1055000000D90E252A000121113202A8FFF73EFD25
:105510006A46127902AB5A7302AA73129373019B03
:1055200076141B0ED67313745574A54205DC02A8BD
:10553000FFF7E4FE00200BB0F0BD3A5D02A963184E
:105540009A740134F1E730B589B0002814DD0C6895
:10555000E30711D5102268460021FFF717FD6B46BF
:105560006A4665105D73684663122D0E641493736A
:10557000D4731574FFF7C2FE002009B030BD0000DF
:10558000174B184A5968002903D00021596001318E
:105590009160196900291FD0002018618023DB0069
:1055A000D3581149012B18D1A923DB00D3585B42F2
:1055B0000B600E490B78032B01D801330B700320CD
:1055C0000B490B78013303400B700A495B015B18F0
:1055D000094953500123936070470860FAE7C046B9
:1055E000FC10004000100040240000209812002011
:1055F0000C1200200E1200200405000010B5034A12
:105600001021034800F090F810BDC04630DA0000C9
:1056100027DA0000044A05491368C85401339B0582
:105620009B0D13607047C046C8160020C8120020AA
:1056300070B5114C114A2368834202DC00232360B9
:1056400016E0155C411C2E00FA3E012E05D8994249
:105650000FDA555C013D1F2D01D90800ECE7010070
:10566000151A565C6E5401318B42FADC181A206010
:1056700070BD1570FAE7C046D41A0020D416002079
:1056800010B5FDF7B3FD064B1A68824201D900221E
:105690001A601B68C31A034898428041404210BDFB
:1056A000C4120020204E000010B5094C094A23689E
:1056B0001268934200D110BD074AD05CFDF7CCFFC1
:1056C0000028F8D0236801339B059B0D2360ECE78D
:1056D000CC160020C8160020C812002010B5040007
:1056E000064B074A1B6812689B1ADB439B059B0D00
:1056F000A34200DB10BDFFF7D7FFF1E7C81600207B
:10570000CC16002070B5FFF741FAFF2504000028F1
:1057100001D1200070BD03681B142B401D2B00D14C
:105720000400FFF727F9F2E770B5074E33680B2B3B
:1057300008DC0C255D43054C013328516419616078
:10574000A260336070BDC046D0160020342F002008
:1057500010B5FBF7CFFCFFF76DF8FBF7F3FCFDF797
:105760000FFFFEF7C7FBFEF723FCFFF747FF00F034
:1057700083FF01F08DF901F0D7FB10BD962210B523
:1057800012010021034806F07DF80022024B1A6046
:1057900010BDC0463C1C0020D0050020064B074A27
:1057A0001B6812689B1ADB439B059B0D01228342F9
:1057B00000DC002210007047C8160020CC16002024
:1057C000F8B505000C0016001F1E0ED10320FFF7D0
:1057D000E5FF002808D0FA20FFF71CFFE8B2FFF72A
:1057E00019FFE0B2FFF716FFF8BD501DFFF7D6FF17
:1057F0000028F9D0FB20FFF70DFFE8B2FFF70AFF02
:10580000E0B2FFF707FFF0B2FFF704FF3012C0B2BB
:10581000FFF700FF3C00E31B9E42E5DD2078FFF729
:10582000F9FE0134F7E7000070B50024F0250B4BBA
:105830001B68A34202DCFFF7A1FF70BD2B0063438E
:10584000074A9B181A78002A05D05978002311209E
:105850001A00FFF7B5FF0134E9E7C046D005002084
:105860003C1C0020F8B507000024F0252B00634302
:105870000C4A01349E18B74211D0317800290BD060
:105880000133D15C002311201A00FFF799FF2A0091
:105890000021300005F0F6FF0A2CE7D1F8BD024BDD
:1058A0001C60F9E73C1C0020D0050020F0B5150075
:1058B00001222F007A4C1740A54401900291002F3D
:1058C00011D005AB1A706A105A70120E1A710522A7
:1058D000691299706D140299DD70FFF771FFCF2383
:1058E0009B009D44F0BD042D2AD90F242868044054
:1058F000042C32D1022304AA28001371FDF72AFFD9
:10590000050006F049FBC82302009B00984200DD19
:105910001A007C1C97420DD1984206D9614804AB0D
:1059200003226149C01805F091FF220005AB0299DE
:105930000198D2E72700611E695C05ACE155E8E7F4
:10594000042D00D0A7E0032304AA043D13716B4289
:105950005D4105AB55710222E9E7092C7ED1042295
:1059600005AB1A706A6851100091694652120978A5
:105970009A70009A59701F2A01DD202200926A460F
:10598000127806ACDA70009BBB4202DC05ABE21A6F
:10599000CDE70126BB00EB189868064006D1042825
:1059A00037D90F210368194002290CD10123237034
:1059B0004310637042121B0E4014A270E0702371FA
:1059C00005340137DFE7042921D102232370FDF7D5
:1059D000C1FE039006F0E0FAA31C0C2809D8607001
:1059E000864201D19C19ECE7039A925D9A550136E3
:1059F000F6E70C226270039A925D9A550136092EE1
:105A0000F9D12E23E372237363730E34D9E701298E
:105A100007D1032304382370434258416070023495
:105A2000CFE7092909D10423237043685A10627013
:105A30005B12A370E6700434C3E703290BD105237E
:105A400023700068020992B2430F92000B40D31AF0
:105A500063701B12EDE726700134B2E7032C00D00F
:105A60003DE7052205AB01091A7089B2420F890092
:105A700022408A1A11125A709970642A00DD642239
:105A80000421DA70081F824201DC04324FE7685CAF
:105A900058540131F6E7002D00D020E753E7C04607
:105AA000C4FCFFFF2203000030CF000070B50200ED
:105AB0000024F0210D4E080060438019457895427E
:105AC00003D001340A2CF6D170BDF022002105F07C
:105AD000D9FE074A1368013BA34200D1146000239A
:105AE00029001A001120FFF76BFEEDE73C1C002097
:105AF000D005002010B5B2B002236A46040013702E
:105B000006F04AFAC72800D9C7200023984207DCCC
:105B1000421C6B46FE211420FFF752FE32B010BD2E
:105B2000694601335A1EA25CCA54EFE730B5B3B0E0
:105B300002236A460500137006F02EFA0400C728F7
:105B400000D9C72400239C420BDC20003230FFF731
:105B5000C5FD621C6B46FF211420FFF731FE33B0F8
:105B600030BD694601335A1EAA5CCA54EBE70000F7
:105B7000F0B5BBB004900C00012803DC1B20FBF740
:105B800023FC51E02A4B08680293C30709D4042878
:105B900007D90F2302681340042B02D1FDF7DAFD69
:105BA0000290234B60680393C30709D4042807D9E4
:105BB0000F2302681340042B02D1FDF7CBFD0390A5
:105BC00000271C4B1B680693069BBB420BDC039B08
:105BD000194A0093C821029B08A806F065F908A895
:105BE000FFF7A4FFCAE70C267E43144B0299F61870
:105BF000306806F0C7F9051E05D17368B6680793CB
:105C0000079B9D4201DB0137DEE73068039905966B
:105C100006F0B8F90836002808D121000498059B41
:105C2000083102385B6898473BB0F0BD0135E7E7C3
:105C3000B8D30000D01600208CDB0000342F0020E9
:105C4000F7B5234B06001B68F02100930023009A50
:105C50009A4211DC0024F0231A0062430192019958
:105C60001C4A55182F78002F12D001340A2CF3D17A
:105C70001948FFF75BFF29E00A005A4315488218CC
:105C80005078B04202D11278002A1FD10133DEE7EA
:105C9000F0223900280005F0F5FD02230D4A019994
:105CA000EB6053540D4AF1008A58009B6E70AE7041
:105CB000AA602F616F61A34202DC054B01341C60B6
:105CC000002331001A001020FFF77AFDF7BDC0460F
:105CD000D00500203C1C0020D5DF00009C250020C2
:105CE00010B5FFF7A1FDFF24084AE3005B429B18B3
:105CF000074AD35C043B012B03D8E043C0B2FFF753
:105D00009FFF013C002CEFD110BDC046FC070000F6
:105D10009C250020F7B50F00FF247F2501901E4A27
:105D2000E300D31A1D4A9A181278062A01D0032AD2
:105D300020D1FF22D2009B18186883682B401C2BAF
:105D400018D1C3681A002A40042A13D102692A40D4
:105D5000192A0FD11B0A01339B000C30C018FDF724
:105D6000F9FC03780600002B10D006F015F900238B
:105D7000B84209D0013C002CD1D1F7BD019AF15CA9
:105D8000D25C9142F6D101339F42F7DCE043C0B2CE
:105D9000FFF756FFEEE7C0469C250020FC070000F9
:105DA00070B50500FF24084AE3005B429B18074AD0
:105DB000D35CAB4203D1E043C0B2FFF741FF013CEB
:105DC000002CF0D170BDC046FC0700009C250020CF
:105DD000F7B5FDF70BFA574B1A68824201D900223A
:105DE0001A601A685449821A8A420DD9FF2253490F
:105DF0001860D3005248CB1A1B181B78073B022BA4
:105E00000CD9013A002AF4D1F7BD0720FFF7C8FFEB
:105E10004C4B27E00820FFF7C3FF38E0FDF7F0F90F
:105E2000071E00D101270020FDF7E2FA01900020B3
:105E3000FDF7F2FA019B0090434C444D002B12D029
:105E40002368002B6ED12B682760002B6ED0404B4F
:105E500001261B78002BD8D10920FFF7A1FF394B71
:105E60001E703B4B1E70009B002B12D02B68002B2A
:105E70000FD123682F60002B1ED0324B01261B78D8
:105E8000002BC7D10920FFF78BFF2E4B1E70304B24
:105E90001E702368002B0FD02A4E3278002A0BD1B7
:105EA0009F4200D227602368FB1A312B04D90720B8
:105EB000FFF776FF012333702B68002B0FD0244EA1
:105EC0003278002A0BD1BB4200D92F602B68FF1A11
:105ED000312F04D90820FFF763FF012333702368B3
:105EE000002B0CD0019B002B09D1164E3378002BD0
:105EF00002D10720FFF754FF0023236033702B6883
:105F0000002B00D180E7009B002B00D07CE7104CD9
:105F10002378002B02D10820FFF742FF00232B60DB
:105F2000237071E7009A002AA0D1B5E7009B002BEF
:105F30009FD1AEE7C01200200F2700009C25002053
:105F4000FC070000B4120020B0120020B81200209C
:105F5000BC12002037B500240500FFF765FC01A83E
:105F60000194FDF733FA21002000FEF70FF9FEF748
:105F70000FFBFDF765FAFDF7DFFAFDF7F9FAFEF71B
:105F800053FCFDF75BF9A54204D0FDF78FFB0248F7
:105F9000FFF7CCFD37BDC046C6DF0000002310B5BB
:105FA00001001A001120FFF70BFC10BD07B56B466E
:105FB000197069465A7013128B701314120ECB703D
:105FC0000A716B46010005221320FFF7F9FB07BD9C
:105FD00010B50A0001001220FFF768FC10BD70B573
:105FE00005000C00FDF714F9002809D0200032301C
:105FF000FFF774FB2B00220000211B20FFF7E0FBC2
:1060000070BD10B50C000300110014202200FFF732
:10601000D7FB10BD012370B5FF24084A41185B422D
:10602000884201D3D84370BD06781D0A23407340CF
:106030009B009B5801306B40F2E7C046A8DB000094
:1060400013B50400FE2813D80A4BC200D05800280C
:106050000ED0436808309900FFF7DCFF019009205B
:10606000FFF73CFB01AB042221001720FFF7A8FB40
:1060700013BDC0469C250020F7B50190FFF742FBF9
:1060800001250400FF276D42002C01D12800FEBD30
:10609000266833143B40152B0DD12100019808319F
:1060A00005F070FF002801D135123D402000FEF7B9
:1060B00061FC0400E8E71D2BF8D101256D42F5E7EE
:1060C000F0B580279FB0FFF7EFFAB54CB54D2068CB
:1060D000FF00391A4019FDF7A5FA23680600C31816
:1060E0002360002B0ED11FB0F0BD2068391A28188C
:1060F000FDF798FA236806001B182360FDF776F871
:10610000A94B1860002EF0DC2B78FA2B00D00EE1A2
:106110002368022B07DCFFF7B3FA0028E3D0012045
:10612000FFF786FADFE76B78AC78981E182800D95D
:10613000F2E003F0CFF90D2024282B34F13E707AE1
:106140007E94CDDEF1F1F1F1F1F1F1F1F1F1EC003C
:10615000FF2C0ED02000FFF7A9FC0022934BE1009A
:10616000CA505B181A712100009213001320FEF729
:1061700009FE0320D4E72000FFF762FDF9E72000C5
:10618000FFF794FCF5E7FFF7ABFDF2E7FFF74CFBF9
:106190000020FFF7DFFE8648FFF7C8FCE9E7632C25
:1061A000E7D8844BA200D25821001520FFF77EFBD0
:1061B000DFE7FFF7A7FAFF270400002CD9D02568F6
:1061C0002B143B40152B04D02000FEF7D3FB04001A
:1061D000F3E72000083005F0DFFE06000530FFF78A
:1061E0007DFAFB20FFF716FA2D121D20FFF712FA99
:1061F000E8B2FFF70FFAF0B2FFF70CFA3012C0B2B4
:10620000FFF708FA25002B1B9E42DDDD287AFFF7F9
:1062100001FA0135F7E700211D2000910B000A006B
:10622000FEF7B0FDFDF742FAA3E72000FFF708FFF5
:106230009FE7FCF7EFFF05AC5F4A642100905F4BDE
:10624000200005F031FE02232000237005F0A4FE9B
:106250002300020000211620FFF7B2FA89E700268A
:10626000524AF3009B181C68002C28D01B7903931A
:10627000636808349F00B81D0293FFF72FFAFB20D4
:10628000FFF7C8F901207D1CFFF7C4F9F0B2FFF752
:10629000C1F9E8B22D12FFF7BDF9E8B2FFF7BAF97C
:1062A0000398FFF7B7F9E719A7420CD8FFF7FCF9F5
:1062B00005230298584301F0FBFAFFF7F5F9013680
:1062C000FF2ECDD155E72078FFF7A4F90134EBE795
:1062D0000024FFF7A9FA2200210000942300DA200D
:1062E000FEF750FDFF222100D200304805F0CAFA27
:1062F00098E7012C02D1FEF767FB3AE7022C02D1A6
:10630000FEF73CFD35E70120FFF724FE31E70023CF
:1063100021001A001A209FE71A00C83A052A00D95E
:1063200027E7002218001100FAF718FF21E7FB2BDE
:1063300000D0F4E62268042A00DCECE62E79E87846
:106340001F4B360206439E4200DDE8E6331D9A42AB
:1063500000DCE0E6EB5CFE2B00D0E0E66878AC7891
:10636000771E1B2800D17DE02ED8072863D008288F
:1063700038D001282DD1FF2C10D02000FFF796FB3C
:106380006D79104AB31E009221002A000A20FEF700
:10639000F9FC064BE400E0501B191D71701DBFE6AF
:1063A000D41A0020D4160020C41200209C250020FE
:1063B000A8DF0000942D0020BFDF0000BADF00003E
:1063C000F6030000DA1600201D285DD04FD31E28EA
:1063D00071D00300C83B052BE0D8404A3900FAF7DA
:1063E000BDFEDBE7632CD9D86A79022A13D0032AD1
:1063F0001BD0012AD2D1E979AB79090219432B7A52
:10640000A4001B0419436B7A1B060B435B00134368
:10641000334AA350C2E7002FC0DDB11E3148FDF75B
:10642000B9FB2F4BA400E050B8E7AB79A4005A1E8B
:1064300093419B00ECE7632FB0DC05AD3A002749A0
:10644000280005F003FA00232800EB55FFF714FE9F
:106450000028A3DB224B8000C25821001520FFF743
:1064600025FA9BE739001D48FFF754FC96E7FF2CFF
:1064700094D06A79022A91D81A490B200091210000
:10648000B31EFEF77FFC89E7632F00DD632700233F
:1064900005A9BB420ADBFB430022DB173B40CB18BC
:1064A0001A70152000917B1C2100EAE7EA18527946
:1064B000CA540133EDE7012C00D06FE7002F00DC58
:1064C0006CE76B79002B03D01C00322B00DD3224EB
:1064D00064235C43044B1C6060E7C046D91600206F
:1064E000942D0020DA160020040000200122094B20
:1064F0001A60094A1368002BFCD00322074B1B6863
:10650000D8171040C01801238010063840001843E7
:106510007047C04600C0004000C1004008C50040B0
:106520000120704710B5064C200000F02DFE0549F3
:10653000200000F05DFE0122034B1A6010BDC04632
:106540000C1B0020801A0600D81A002010B501216B
:106550000D20FCF765FE01210E20FCF761FE0021F5
:106560000F20FCF75DFE044C200000F04FFD1021D1
:10657000200000F067FD10BDEC1A0020F8B50125E1
:106580000C682C4203D10D20FAF71EFFF8BD6410F1
:106590002DD4FCF743FEA04229DB00212000FCF7AC
:1065A0003FFEFA222900D200200001F0B3F90028B2
:1065B0001DD0002500270726FA2201219200200085
:1065C00001F0A8F9002812D0282802DD0123B340E9
:1065D0001F43013EF0D20E4EAF550135052DE9D1D6
:1065E000012206210920FDF757FA002801D10020D9
:1065F000CCE70B23012443600023F25C9900520096
:106600004118224301338A60052BF6D1BEE7C0460C
:10661000DC1A002010B504680D20E30703D56410D0
:10662000FF2C03D91720FAF7CFFE10BDFFF78EFF1E
:10663000E1B2024800F028FD0020F6E7EC1A002045
:1066400010B5FFF783FF0021034800F01DFD430054
:106650000120184310BDC046EC1A002010B50020E0
:1066600001F0D6F9800810BD10B5FFF7F7FF430021
:106670000120184310BD000010B5034A0A21034849
:10668000FFF752F810BDC046ECDF00003CE0000010
:106690000D4B70B51B6804000E001500002B01D1D6
:1066A000FFF740FFE1B2094C200000F038FEF1B2E4
:1066B000200000F035FDE9B2200000F031FD20009F
:1066C00000F098FE70BDC046D81A00200C1B0020B8
:1066D00010B501240368234205D04168214202D04D
:1066E0008268224203D10D20FAF76EFE10BD5810C9
:1066F000802801D91520F7E74910FF2901D9162074
:10670000F2E75210FF2A01D91720EDE7FFF7C0FF8B
:106710000020EBE7F7B501221400904222DD0D685E
:106720002A421FD01D4B15411B684C68002B01D11C
:10673000FFF7F8FEE9B201272500194E3D40300071
:1067400000F0EDFD002D0FD03C413000E1B200F033
:10675000E7FC300000F04EFE0024A04202D02320CF
:10676000FAF732FE2000FEBD042CF2D90F23226876
:106770001340092BEDD163685B100193019BAB4281
:10678000E7DDAB00E3189968394204D04910C9B27B
:10679000300000F0C5FC0135F0E7C046D81A0020F3
:1067A0000C1B0020154B70B51B6805000E00002B5C
:1067B00001D1FFF7B7FE124CEDB22900200000F026
:1067C000AEFDF1B2200000F0ABFC0021200000F093
:1067D000B1FD002801D0404270BD72B601222900EF
:1067E000200000F097FD62B6200000F08AFC00282F
:1067F000F2D0200000F08AFCEEE7C046D81A002054
:106800000C1B002010B501240368234202D041680C
:10681000214203D10D20FAF7D7FD10BD5810802872
:1068200001D91520F7E74910FF2901D91620F2E711
:10683000FFF7B8FF40002043EFE7000010B50D213F
:106840001D20FFF7AFFF164C5A2809D101222A213B
:1068500022703D38FFF71CFF0122124B1A6010BD59
:106860000F211920FFF79EFF332805D102235F2255
:10687000237020211A38EDE70D211E20FFF792FF2B
:10688000C7280AD1032300222A21A9382370FFF741
:10689000FFFE1B222A211E20DCE700232370DBE7FA
:1068A0002C000020E41A0020204B10B51B680400C7
:1068B000002B01D1FFF7C2FF1D4B1B785BB2022BEF
:1068C0000AD0032B29D0012B2CD121001D2001241B
:1068D000FFF768FF644205E0012C13D1292119203C
:1068E000FFF760FF7F2801DD0138FF3803007F33A9
:1068F00001DA7F204042C8237F21584302F07EFE08
:10690000604310BD032C0BD12B211920FFF74AFF48
:10691000043CE7E72D211920D9E721001E20D6E706
:10692000052CF7D0012400206442E4E7E41A00209B
:106930002C00002010B50120FFF7B6FF4300012016
:10694000184310BD10B50320FFF7AEFF4300012030
:10695000184310BD10B50520FFF7A6FF4300012026
:10696000184310BD144B70B51B68002B02D10120D9
:10697000FFF79AFF114B1B785BB2013301D1FFF790
:106980005DFF0120FFF790FF04000320FFF78CFF5D
:1069900005000520FFF788FF6D43644340436419F9
:1069A000201804F03BFE01F00FFB04F001FE430051
:1069B0000120184370BDC046E41A00202C000020BE
:1069C000F8B501231C0098422BDD0F683B4228D00C
:1069D0004E6835001D4024D1042E22D90F22316883
:1069E0000A40092A1DD173685C10202C00DD202488
:1069F000144B1B68002B01D1FFF794FD72B67F107A
:106A0000F9B2114F2200380000F084FC62B6A542B2
:106A100014DA380000F075FB002804D101246D0061
:106A20002C432000F8BD380000F070FB0122AB00C1
:106A30004000F31810439860AD18E8E764000125A2
:106A4000EEE7C046D81A00200C1B0020002070473B
:106A500001207047002070470020704700207047D9
:106A600001207047002070470020704700207047C9
:106A700000207047002070470020704700207047BA
:106A80000020704700207047704770477047000033
:106A900010B5034A0F210348FEF746FE10BDC0465D
:106AA000A0E0000018E100000378013B1F2B00D993
:106AB00070470130F8E710B5FFF7F6FF0378002BB9
:106AC0000BD00130222B11D10378002B03D0421CB4
:106AD000222B03D11000FFF7E7FF10BD5C2B03D181
:106AE0004378002B00D0821C1000EDE73A2BF2D047
:106AF0002C2BF0D07B2B0BD1FFF7D6FF0378002B8C
:106B0000E9D07D2B01D10130E5E7FFF7D4FFF5E7B0
:106B100020225B2B14D1FFF7C7FF0378002BDAD0BC
:106B20005D2BF0D0FFF7C7FFF7E7202BD3DD2C2B31
:106B3000D3D0190091435D29CFD0222BCDD0013085
:106B40000378002BF1D1C6E7002210B5904216D091
:106B5000FFF7AAFF03780422222B10D0023A7B2BE6
:106B60000DD0013A5B2B0AD01900303902320929C5
:106B700005D92D2B05D14178303909290AD81000C3
:106B800010BD0522742BFAD00132662BF7D00132EA
:106B90006E2BF4D0581E83415A42F0E770B5FFF7D0
:106BA00083FF037801222D2B01D18018023A0023A4
:106BB0000A2502E06B430130CB1801783039CCB2A2
:106BC000092CF7D95A43100070BDF8B50C00150018
:106BD000FFF76AFF0378222B02D000232370F8BD51
:106BE0000D236A1E210008250C260A279C46013029
:106BF0000378222B02D100230B70F0E7002BFAD090
:106C0000441C5C2B0BD14378841C622B0ED0662B6A
:106C10000ED06E2B0ED0722B0ED0742B0ED0002AFD
:106C2000E9DD0B70013A01312000E1E72B00F6E7C6
:106C30003300F4E73B00F2E76346F0E70923EEE7B1
:106C400010B50400FFF737FFA04202D90378202BCC
:106C500000D910BD0138F7E710B5002815D003782A
:106C6000002B13D0FFF720FF2021037802008B4375
:106C700000205D2B09D01000FFF71DFF03782C3B8F
:106C80005A425341C018FFF70FFF10BD1800FCE730
:106C90000300002070B50C0081420EDD1A785B2ADB
:106CA0000BD1581CFFF700FF0125AC4205D0FFF7C0
:106CB000D3FF002801D00135F7E770BD70B50C0097
:106CC0001500002901D000230B70002820D0037884
:106CD000002B1ED0FFF7E8FE037806002C2B03D113
:106CE0000130FFF7E1FE0600337800207D2B0FD046
:106CF000844204D02A0021003000FFF766FF3000F4
:106D0000FFF7D9FE03783A2B02D10130FFF7CCFE12
:106D100070BD1800FCE7F0B50D0004009DB02E78A2
:106D2000002E35D02E21280005F01EF9071E14D0A4
:106D3000431B0193303E092E14D82800FFF72EFF85
:106D400001002000FFF7A4FF0400002C20D0002F3A
:106D50001ED0019B0133ED18E1E7280005F01CF976
:106D60000190E7E723787B2B11D1601C642203A9F3
:106D7000FFF7A4FF041E0BD0019A290003A805F019
:106D800012F90028E1D02000FFF795FEEEE700247D
:106D900020001DB0F0BD70B5050000200C00814240
:106DA0001DDD2800FFF7D0FE0300681C012B14D066
:106DB0000020022B13D10022681C1100FFF77EFF78
:106DC000012C0CD0FFF748FF00221100FFF776FFDF
:106DD000013CF5E7FFF740FF013C012CFAD170BD03
:106DE000F8B5050000200C0016001F0081420DDDE3
:106DF0002800FFF7A9FE03000020022B06D1681C23
:106E00003A003100FFF75AFF012C00D1F8BDFFF71F
:106E100023FF3A003100FFF751FF013CF4E710B5C2
:106E20000024A04218D0FFF73FFE03787B2B0AD145
:106E3000013000221100FFF741FF00280CD0FFF7BE
:106E40003AFE0134F5E75B2B06D10130FFF704FF72
:106E5000002801D00134F9E7200010BDF8B5002862
:106E600016DD0D68EB0713D56D10013D0124FDF70C
:106E70008DFE0026FF27644200280CD1002E21D071
:106E8000300005F089F801003000FCF783FEF8BD02
:106E900001256D42EAE703681A143A40152A0BD11E
:106EA0001B123B409C4200DA1C009D4201D10600AF
:106EB0000836FDF75FFDDFE71D2AFAD10124002621
:106EC0006442F6E70120013464002043DFE700005C
:106ED00010B508680C00FCF73DFCFFF7CDF8002862
:106EE00003DB6268024B8000C250002010BDC04628
:106EF000942D002010B50868FCF72CFCFFF7BCF8B7
:106F00000123002802DB024B8000C358180010BD8B
:106F1000942D002010B50868FCF71CFCFFF7ACF8B6
:106F2000C043C00F800010BD10B5034A04210348C0
:106F3000FEF7FAFB10BDC046B4E10000AEE1000070
:106F400010B5FCF729FBFCF7D7FBFEF701FC044862
:106F5000FEF7ECFDFDF778FFFEF7C2FE10BDC04660
:106F600003E2000010B5FCF719F810BD70B500255C
:106F700004AC24780573A94205D10A4B0A4A25219D
:106F80000A4804F0F5FB01600949920052589B0041
:106F900002715B58A40083716358856043710223BA
:106FA000C37170BD1BE200007AE2000029E200001C
:106FB000D8E20000037B002B04D143738373036189
:106FC00001330373704700001FB50191A021002415
:106FD0000068C900D2B24450012A10D0A24209D0A0
:106FE000032A0AD0074A8350074B019AC250012353
:106FF00043501FBD02221343F4E70422FBE706229D
:10700000F9E7C046540500002405000010B504004F
:10701000FFF7D0FFA1222368A179D20099506179AE
:10702000064A20009950217904329950044B19687E
:107030005A689B68FFF7C8FF10BDC0460C050000EA
:10704000001B00204BB2002B0FDB80233F290FD801
:107050001F290FD80F290FD807290FD803290FD8B8
:107060001B060168074A8B50704780239B04F8E792
:10707000DB04F6E71B05F4E75B05F2E79B05F0E7A9
:10708000DB05EEE7240500000368074A99501A0063
:10709000FC32D1680029FCD0A321C9005858002334
:1070A000C0B2D3607047C0461C05000007B58022FF
:1070B000074BD2051A6000229A6002321A710F2320
:1070C0000C3200930349023B0348FFF74FFF07BD13
:1070D000001B002000300040EC1A0020F8B505002D
:1070E0000E0017000024BC4208D02B68315D1B68DD
:1070F00028009847002801D00134F4E72000F8BDAB
:10710000704710B51C3000F0AFF910BD10B51C3041
:1071100000F09CF910BD10B51C3000F0ABF910BDAB
:1071200070B5437E0D00002B01D1002070BD64308E
:10713000040000F0A8F90028F7D12000290000F091
:1071400076F90120F2E70000F7B50193FA23002554
:1071500004009B0083600B4B4560083303601C30C8
:107160000F00160000F058F92000643000F054F9C8
:107170006B461B79276166756576A5762000A37539
:10718000FEBDC046B8E20000012330B5A024C3759F
:10719000837D13499B005A58437DC132114DFF3204
:1071A000E40592009B005B581551CC22C133FF339C
:1071B0009B001D5104690C4B5204E25005220469E6
:1071C000243BE250837D04699B005A58A123DB00D5
:1071D000E250437D02699B005958044BD15030BDA9
:1071E000D8E200000C060000240500000C05000099
:1071F000A022002310B50469D200A3500A4CA1427A
:107200000FD90A4C8C425B4109495B420B40CD21AE
:10721000C9045B1804690749635005210369995043
:1072200010BDCC235B04F5E7A086010090D00300DD
:10723000000098FD24050000F7B5040000200D00B3
:107240000193824265D01600402A00D940262700CB
:107250001C37380000F0F6F8B1232269DB00D55066
:1072600080220123216992008B50A27E002A03D143
:1072700022691362226913600025731EAB4207D195
:10728000019B002B04D08022022123699200995097
:10729000012223691A622369FC33DA68002A02D1C9
:1072A0009A6A002AF9D09A6A002A0BD1DA60A323DD
:1072B0002269DB00D1583800C9B2013500F0B7F8B7
:1072C000B542DAD3019B2269002B0FD11300FC33A6
:1072D0009B6A002B0AD10133A376D3612369FC3367
:1072E000DA6C002AFCD00022DA640AE000230121D3
:1072F000A37651611A002369FC3399680029FCD0F8
:107300009A602369FC339A6A002A01D000229A62AB
:10731000E8B2FEBD10B50123FFF78EFF10BD0300DC
:10732000AC3310B504001970643000F08BF8012301
:10733000637610BD0023020070B5AC3243760D00B9
:107340001178B12204000069D200815080222169A5
:1073500092008B50226901331362226993602600E8
:107360006436300000F080F8002812D0300000F0C1
:107370006DF81E4B2269D0502369FC331A6A002A2B
:1073800002D19A6A002AF9D09A6A002A01D11A62B7
:10739000E5E723690122002D0DD11900FC31896A2E
:1073A000002908D1DA612369FC33DA6C002AFCD0A9
:1073B0000022DA6407E05A612369FC339A68002AE4
:1073C000FCD000229A6000202369FC339A6A824232
:1073D0000BD098622169064A8B588B501800022BFB
:1073E00003D0181F431E9841033070BD1C050000D8
:1073F000C404000010B50121FFF79CFF10BD000080
:1074000010B51323142202490248FFF79DFE10BD58
:10741000004000400C1B002010B540220021040059
:1074200004F030FA002320002364636410BD10B51B
:107430003F24026C531C2340446C9C4201D0815475
:10744000036410BD0023036443647047436C026C03
:10745000934206D03F21C25C01330B4043641000CD
:10746000704701204042FBE7036C406C181A00D5BE
:1074700040307047436C026C934201D0C05C70474F
:1074800001204042FBE73F22036C406C0133134074
:10749000181A43425841C0B27047000003210A48FD
:1074A00002680A430260094802680A430260084908
:1074B000084A094B9B1A03DD043BC858D050FBDC3B
:1074C00000F012F8F8F720FE2405004054050040B3
:1074D00028E800000000002068020020FEE7FEE728
:1074E000FEE7FEE7FEE7FEE7014B024A1A6070473F
:1074F000300000200024F4000120704710B503681C
:107500001322DB69984710BD70470000054B0269E4
:10751000D1500369FC331A6A002AFCD000220120F2
:107520001A6270471C050000030010B55C331A781E
:107530001F231A401E3B19009140114AD167C222F5
:10754000042104699200A150026953600269D3606A
:10755000A02300220169DB00CA5001230169094A06
:107560005B428B500169084A8B5001690C3A8B5081
:10757000016908328B501430FFF764FF10BDC0461C
:1075800004E100E00C0500001405000010B5143003
:10759000FFF76AFF10BD10B51430FFF76BFF10BD89
:1075A00010B51430FFF752FF10BD0000030070B596
:1075B0005E331A780469724BE25003005D331A7827
:1075C0000469704BE250030061331C7802696E4B12
:1075D000012C00D09EE005005F352E78A225ED003D
:1075E0005651020060321578A1220669D200B550CA
:1075F0000269D4509623DB00994200D88CE0962390
:107600001B01994200D88AE096235B01994200D879
:1076100088E096239B01994200D885E0E1239B01F5
:10762000994200D882E09623DB01994200D880E09D
:10763000E123DB01994200D87DE096231B029942A9
:1076400000D87AE0E1231B02994200D877E0962324
:107650005B02994200D874E0E1235B02994200D8B2
:1076600071E0E1239B02994200D86EE0474B9942BA
:1076700000D86CE0E123DB02994200D86AE0E12205
:10768000002312038A425B41414A5B42134080223D
:1076900052059B1801693F4A8B50A02304220169BF
:1076A000DB00CA5000210369FC33D9600369FC3355
:1076B0001962012301690B6001698B60C1210469B2
:1076C000890062501F215C3002780A409340623189
:1076D000314AFF3153500021415600293CDA0F2333
:1076E0000B40083B2D4C9B089B001B190324214099
:1076F000A140FC348C40DD69A5432C00C0258D40A1
:1077000029002143D9611F23017819401E3B8B407A
:10771000136070BD00246CE79E23DB02BAE79D2353
:107720001B03B7E71E4BB5E71E4BB3E7EC239B03E8
:10773000B0E71D4BAEE71D4BACE71D4BAAE71D4B59
:10774000A8E71D4BA6E71D4BA4E71D4BA2E780232E
:10775000DB049FE71B4B9DE78C080F4BA400E4184C
:1077600003230B40FF21C025DB009940AD00665983
:107770008E433100C0269E4033000B436351C2E765
:107780000C050000140500006C05000090D00300FB
:1077900000D0BEFE2405000000E100E000ED00E0A6
:1077A00000B013000050270000A04E0000F075004C
:1077B00000509D0000F0EB0000903A0100E0D7017E
:1077C00000B0AF0300705F07F7B5009308AB1B78FC
:1077D00000250193FA2304009B0083600E4B456053
:1077E0000833036014300F001600FFF715FE230066
:1077F0005C3327611E70009B084A9B009958230048
:107800005D331970019B20009B009A5823005E3362
:10781000DD701A70FEBDC0465CE30000D8E20000D7
:10782000036910B51A00FC32D2680400002A0AD09D
:10783000A322D20099581430C9B2FFF7F8FD0022F4
:107840002369FC33DA6010BD10B50248FFF7E8FF8A
:1078500010BDC046C41B0020162307B502220093AA
:107860000249013B0248FFF7AFFF07BD002000407F
:10787000C41B002010B5002801D004F0BFFA10BDD1
:107880000849094A094B10B51B688858FA22190A99
:107890001B0618439200002301F0E8FF4904C00BC7
:1078A000084310BD0010014004050000281C002002
:1078B00070B5041E09D0FFF7E3FF050000F014F8CF
:1078C000FFF7DEFF401BA042F8D370BD0022044B3F
:1078D0009A60044A13680133DBB213607047C046F4
:1078E000FC100140281C00207047704710B500F0C4
:1078F0005FF8FFF7FAFF0120FFF7DAFFFFF720FB41
:10790000FFF730FB024B002BFAD000E000BFF7E797
:1079100000000000F8B54C1EA1410125104B114F8D
:107920008000C3584C4238680F499D40160001F052
:10793000DBFD0A21704301F0D7FD2C40030022003B
:1079400029000A4800F016F8FA21094C890044433E
:10795000386801F0C9FD0100200001F0C5FDF8BD47
:10796000D8E200003000002040420F001005005017
:107970001027000030B504680C40944206D1013B4A
:10798000002BF8D112E0013B002B0FD004680C4013
:107990009442F8D1002405680D40954204D1013489
:1079A0009C42F8D1002002E0201C00E0181C30BDF1
:1079B000C420114B80001A5810491140C0221202F5
:1079C0000A431A50C0218022490092025A501A607C
:1079D0008023A3220021DB05D20099500122F93037
:1079E0009A60074BFF301950C120023180001950B6
:1079F000403019501A60704700E100E0FF00FFFFBF
:107A000000100140014B18607047C0467C00002008
:107A1000F7B5002320285AD8384B8000C258042AD2
:107A20005BD007D8022A54D055D80423012A09D0A4
:107A300000234CE0062A54D051D31A2A53D00223F3
:107A40001B2AF5D12E4A116808294ED909294FD091
:107A50000A240226A02001252A4AC00015502A48DF
:107A60002A4D07681C20BF0007402948019700687D
:107A70005759009027481B0207401F43C023009816
:107A80009B020340FF2057515759000207401F43F4
:107A9000019B1F43009B58016023184007433E434E
:107AA000565101251C4B156058680028FCD0002059
:107AB0005860A1230125DB00D3585560A025ED00B7
:107AC00050511BB2A14202D015D2611ACB4018000E
:107AD000FEBD0823B6E71023B4E72023B2E7402316
:107AE000B0E78023AEE70123ACE708240026B1E726
:107AF0000C000126AEE7091B8B40E8E7D8E2000046
:107B000078000020007000403400002004050000D0
:107B100038000020FF00FFFFFC700040F0B5202877
:107B20005BD8364B8000C258354B1E68002E30D1D2
:107B3000C227344BBF00D859334C03250440C02022
:107B400000022043D851C0248020640080001851D6
:107B50002E4F18602E4B803CD859FF3CA043D85183
:107B60000437D859A8432043D8510837D8590C3581
:107B7000A8438446072065462843D851A820C00062
:107B80001E50C1208026800076021E501C601C4BB7
:107B90001C60142500202B001E4C2E004643365935
:107BA000771C1BD14343E250A0230325C132FF328F
:107BB0009200DB05D550184B1A68082A14D11423FB
:107BC0004343E3189A6812485132FF3292005960D9
:107BD0001150DA68C1239B00C250F0BD9642E1D03B
:107BE00001300328D9D1F8E7082A02D9083AD14050
:107BF000E5E708239A1A9140E1E7C046D8E2000081
:107C00002C1C002000E100E0FF00FFFF0405000045
:107C1000009000403C0000207C0000202149F0B58D
:107C20004A6C2148002A14D0A025A1260023012453
:107C3000ED05F600C258571C06D0C7187F68002F04
:107C400002D027009740AF5114333C2BF2D10023D0
:107C50004B64A0230121DB0500260F009C46142362
:107C60004B43C3181A1F1268104C0E4D9200141982
:107C70005219526C002A10D01A00143A1268551C7E
:107C800009D0103B1B68FF2B05D03B009340654695
:107C90001A00074BEA50FC34666401310429DED136
:107CA000F0BDC046FC9000403C0000200090004029
:107CB0000C05000000B5202810D80C4A800083581D
:107CC00003290BD8A0220800C133FF33D2059B0043
:107CD00001F000FC020905070021D15000BD0C2174
:107CE000FBE70421F9E70321F7E7C046D8E20000EB
:107CF00020280AD8074B8000C25801239340A022B5
:107D0000D205002902D1044953507047A121C9006E
:107D1000FAE7C046D8E200000C050000030000208E
:107D2000202B0AD8A021A222C905D2008858034AD4
:107D30009B009B58D840012318407047D8E20000B0
:107D4000F7B506000D000C008B180193019B671B13
:107D50009C4207D0336821781B6830009847013473
:107D60000028F3D13800FEBDF0B5C64600B5CB0FF4
:107D70009846404A4B005B0D9A1882B00D000400F3
:107D8000132A2FDC002A49DB3B4F17413E000E40EF
:107D9000064323D07F08390029400C430AD03749D5
:107DA000BD438C4663445C425C418023DB0213414B
:107DB000E4071D434146CE0031492B008E192200B5
:107DC000346875682000290001F0F6FE00900191EA
:107DD0000098019922002B0003F086F802B004BC41
:107DE0009046F0BD332A08DD8023DB009A42F5D1AE
:107DF00002000B0001F0E0FEF0E7224A9446012267
:107E000063445242DA400242E8D052080242D1D0E2
:107E100094438022D2051A411443CBE74B005B0800
:107E20000343DBD00B031B0B1C436342234380241F
:107E30004D0C24031B0B23406D042B4319004346B8
:107E4000DA000F4B9B181C685D6802000B002000D5
:107E5000290001F0B1FE00900191009801992200E3
:107E60002B0003F041F842464B005B08D607334332
:107E70001900B3E701FCFFFFFFFF0F00EEFBFFFF60
:107E800090E30000EDFBFFFFF8B5274A4B005B0DC8
:107E90009A180C000700132A10DC002A36DB234B4B
:107EA00013410B423AD0802424031441002064186B
:107EB0009C430600250030002900F8BD332A0EDD62
:107EC00080230600DB000D009A42F4D102000B0073
:107ED0003800210001F070FE06000D00EBE7144DA4
:107EE0000600AC46012563446D42DD40AC46634666
:107EF0000D000342DFD033239A1A323B9340181807
:107F0000874200D94C1C63469843D2E7C90FCC077F
:107F10000020531CCDD1074B1C43CAE706000D00BF
:107F20000028C0D1C7E7C04601FCFFFFFFFF0F00DC
:107F3000EDFBFFFF0000F03F30B5214A4B0087B05A
:107F40005B0893421EDD1F4A934205DD02000B00D1
:107F500002F0CAFF07B030BD02AA00F095F8032373
:107F60001840049A059B012813D002281DD0002830
:107F700014D00298039900F06FFB80231B069C46E7
:107F80006144E7E7002300220093002301F0DEF8BC
:107F9000E0E70298039900F05FFBDBE70124029819
:107FA0000399009401F0D2F8D4E7012402980399D0
:107FB000009401F0CBF880231B069C466144C9E77E
:107FC000FB21E93FFFFFEF7FF0B54746CE4680B586
:107FD0008DB004000D0000F067FA294B06001B78F5
:107FE0000F005BB29846013310D022002B00200016
:107FF000290003F0C1FA8146002807D1002200239E
:108000002000290001F00AFC002806D130003900C8
:108010000DB00CBC90469946F0BD01230293194B5C
:108020000694079503934B460A934346049405959B
:10803000002B15D0002300221900100002F0D8F800
:10804000434608900991022B0ED103F0AFFB212388
:1080500003600A9B0193002B0CD1089E099FD5E772
:10806000002300240893099402A801F0C1F9002814
:10807000EFD1EAE703F09AFB0A9B01930360ECE778
:1080800080000020A0E30000F0B54E464546DE46E5
:108090005746E0B5E14B4C008FB0904689466408E6
:1080A0009C4200DC87E0DE4B9C4222DCDD4A00295A
:1080B00000DC92E0DC4B02F017FFDB4B06000F0008
:1080C0009C4200D17EE1D94AD94B02F00DFF02005B
:1080D0000B00414630000A604B60390002F004FF9B
:1080E000D34BD24A02F000FF434601259860D96085
:1080F0006BE0D04B9C4200DC8FE0CF4B9C4200DD1C
:1081000055E1CE4A231592469A4451460905631A11
:1081100019001D00040003F04BFA03F07FFA02007F
:108120000B00200029000892099302F0DDFE0022D6
:10813000C34B02F067FC0F00060003F039FA03F0AE
:108140006DFA04000D0002000B00300039000A94A3
:108150000B9502F0C9FE0022B94B02F053FC00223D
:1081600000230C900D9101F053FB002800D192E107
:10817000002300222000290001F04AFB4342434132
:108180000133B04A41460192022208A800925246A9
:1081900000F07CFB4B460500002B16DA802243469C
:1081A0001206944642465B68454263445360D36876
:1081B0006344D36009E00B00020041460A604B6053
:1081C0000022002300258A60CB6028000FB03CBC51
:1081D00090469946A246AB46F0BD934B01F0ECFCAD
:1081E000914B06000F009C4200D13DE18F4A904B1D
:1081F00001F0E2FC02000B00414630000A604B60D7
:10820000390002F071FE894A894B01F0D5FC012545
:1082100043466D429860D960D7E701F049F88A4A31
:108220008A4B06000F0002F0EDFB0022884B01F0A4
:10823000C3FC03F0BDF9050003F0F0F9794A7A4B6D
:108240000490059102F0DEFB02000B0030003900C3
:1082500002F04AFE754A06000F0004980599744B17
:1082600002F0D0FB029003911F2D00DCC7E0029AC0
:10827000039B3000390002F037FE83468A4653469E
:108280005B0024155B0DE31A102B6CDD0498059937
:10829000D322674B520502F0B5FB02000B00300001
:1082A00039000292039302F01FFE0A00010013003E
:1082B0000691079202003900300002F015FE029A82
:1082C000039B02F011FE06000F0004980599614A15
:1082D000614B02F097FB32003B0002F005FE069E68
:1082E000079F0B000200390030000292039302F056
:1082F000FBFD4B005B0D83468A46E41A312C32DDD0
:1083000004980599B822544B920502F07BFB0300B8
:108310000C000200029303940B000698079902F0E8
:10832000E3FD02000B0006000F000698079902F01B
:10833000DBFD029A039B02F0D7FD484A02900391AD
:1083400004980599464B02F05DFB029A039B02F0EC
:10835000CBFD02000B00300039000292039302F0C3
:10836000C3FD83468A465A465346414630000A605A
:108370004B60390002F0B8FD029A039B02F0B4FD95
:1083800044460B000200A260E3604B46002B00DB7A
:108390001BE75B46236080231B06534463608023F6
:1083A0001B069C466144A060E1606D420DE70B0036
:1083B000020002F099FD434600259860D9601860DC
:1083C000596002E7D3221A4B520502F08DFD214A73
:1083D000214B0D00040002F087FD02000B00414616
:1083E00020000A604B60290002F07EFD1A4B194AFA
:1083F00002F07AFD434601259860D960E5E6020067
:108400000B003000390002F06FFD6B1E154A9B0017
:108410009B5883468A46A342A5D130E7FB21E93F1A
:108420007BD9024000004054FB21F93F3163621ABE
:1084300061B4D03DFB213941FFFFEF7FEAFBFFFF35
:108440000000704128E4000083C8C96D305FE43F3C
:108450000000E03F7370032E8A19A33BC149202519
:108460009A837B39A8E30000D3220C4B520501F01C
:10847000A3FB0B4A0B4B04000D0001F09DFB020017
:108480000B00414620000A604B60290002F02CFDE1
:10849000034A044BB9E6032373E6C04661B4D03DFA
:1084A0007370032E8A19A33BF8B54746CE46674B37
:1084B00080B50A000F00190005003940994200D12B
:1084C0009BE004000100002F69DD3F1500D1B4E0FE
:1084D0005F4B12039C468023120B5B0313435B002C
:1084E000CA0F67449B184A00F80703D5D20F5B00F8
:1084F0009B188A0079108C4600218020162489461A
:1085000080030D189D4202DC29185B1B8144D50FA6
:108510005B00013C5B1952004008002CF1D10020A7
:108520008046802020250027000609E08B425CD091
:10853000D40F5B00013DE31852004008002D16D017
:10854000C4198B42F2DD27180E00002C49DB5B1AA0
:10855000A242894149425B1A121BD40F5B00013DC4
:1085600080443100E31852004008002DE8D1134345
:108570004ED143465B0837494A4688464946521021
:108580004244C90702D5802109060B4361460F0505
:10859000BD18180029000CBC90469946F8BD7B0018
:1085A0005B0803433900002BF5D0002F3CD1E30AD0
:1085B000153A6405002BFAD08020400303423FD1D6
:1085C000002700E00F005B00791C0342FAD0250071
:1085D00020208D40401A2900D71B2200C2401A4398
:1085E00076E7FE43F60F8E19B1E79442A0D827181C
:1085F000002CF6DB1E000023AEE702003B00280043
:10860000390002F0FFF92A003B0001F0D5FAC2E779
:108610004346013303D0434601335B08ABE70123F4
:1086200098460023C144A6E73B00020002F05CFC30
:1086300002000B0001F0DCFDADE713000022BBE7F8
:108640000127210020207F42C6E7C0460000F07FBE
:1086500001FCFFFF0000E03FF0B54746CE4680B585
:1086600087B000920193754B4F00814688467F0882
:108670009F4263DC02F09CFF002800D1D4E04A4610
:1086800043464846414602F0BDF904000D006C4ADD
:108690006C4B02F0B7F96C4A6C4B01F08DFA22007A
:1086A0002B0002F0AFF96A4A6A4B02F01DFC22006F
:1086B0002B0002F0A7F9684A684B01F07DFA22000E
:1086C0002B0002F09FF9664A664B02F00DFC220077
:1086D0002B0002F097F9644A644B01F06DFA220016
:1086E0002B0002F08FF9029003910022604B2000D2
:1086F000290002F087F9029A039B06000F00200070
:10870000290002F07FF9009A019B04000D00484601
:10871000414602F077F902000B002000290002F028
:10872000E3FB02000B003000390002F0DDFB020029
:108730000B0000204F4902F0D7FB70E002000B0055
:1087400002F060F904000D003D4A3E4B02F05AF978
:108750003D4A3E4B01F030FA22002B0002F052F964
:108760003B4A3C4B02F0C0FB22002B0002F04AF9CE
:10877000394A3A4B01F020FA22002B0002F042F96C
:10878000374A384B02F0B0FB22002B0002F03AF9D6
:10879000354A364B01F010FA2B00220002F032F974
:1087A000354B029003919F429FDD344B00229F4244
:1087B0003DDC334900207B182E4916001F0002F0D3
:1087C00093FB049005910022294B2000290002F020
:1087D00019F932003B0002F087FB029A039B060066
:1087E0000F002000290002F00DF9009A019B0400FF
:1087F0000D004846414602F005F902000B0020003A
:10880000290002F071FB02000B003000390002F079
:108810006BFB02000B000498059902F065FB07B0A2
:108820000CBC90469946F0BD00201249F7E7154B65
:10883000002604920593144FC5E7C046FFFF3F3E54
:10884000D43888BEE9FAA8BDC4B1B4BD9EEE213EBD
:10885000AD529C804F7E923E9015CB19A001FA3EFE
:108860007751C1166CC1563F4C5555555555A53FCE
:108870000000E03F0000F03F3233D33F0000E93F0B
:108880000000E0FF0000E73F0000D23FF0B5DE4609
:108890004E4645465746E0B5DC4CA5440D911400C4
:1088A0001900A49A0993DA4B9200D6584D1E0390F2
:1088B0001821E01E0696029500F0A0FEC3430100B9
:1088C000DB1719404B1C9A009B1ADB001B190B91FC
:1088D00005934C1B771918D4A59BA5009C463F19FE
:1088E00022AE6544013707E0286802F097FE0134A4
:1088F00003C60435BC4208D0002CF5DA0020002164
:10890000013403C60435BC42F6D1069B002B01DAC4
:1089100000F0FDFB069B03990133DB009A46099B9F
:10892000DA00944600920022914672AA0492B94A53
:108930006144934688469AAB63449B44029B002B58
:1089400000DABCE15D4600260027039C4D442A68FE
:108950006B6803CC02F056F802000B0030003900BF
:1089600001F02AF9083D06000F004445EFD1049BB1
:108970004B441E605F6008239C46E144D145DDD135
:108980000EA804218446494261448C46069A93000D
:108990009C44614684460A910399083B63448C4693
:1089A0000C93009B009263449B46009A0498D1006C
:1089B00003008C46634408911E685F68002A33DD1B
:1089C000954980468C466244D300984470AB9A46E1
:1089D0000EAB99460022914B3000390002F012F89C
:1089E00002F0E6FD02F01AFE00228D4B04000D009D
:1089F00002F008F802000B003000390002F074FAAF
:108A000002F0D6FD4B4601C39946434620001A6842
:108A10005B68290001F0D0F808235B429C46E044E3
:108A200006000F00D045D5D1059B30001A00390053
:108A3000984600F0DFFCFF2300229B0504000D0098
:108A400001F0E0FF00F038FC0022764B01F0DAFF85
:108A500002000B002000290002F046FA0D0004007D
:108A600002F0A6FD814602F0D9FD02000B002000B5
:108A7000290002F039FA060040460F00002800DC09
:108A8000EEE0009B18215A1E92000EAB9B58091A6B
:108A90001D000D41A9448D405D1B0EAB9D50172359
:108AA0001B1A1D41002D2DDD01239C46009BE14436
:108AB000002B00DC1CE20E9C0123002C00D0B5E052
:108AC000009A012A09D099000EAA54580133002CAB
:108AD00000D0ACE0009A9A42F5D1059B002B0EDD48
:108AE000012B00D1A8E1022B09D1009B0EA95A1E2F
:108AF00092000EAB9B5807939B029B0A8B50022D52
:108B000000D1C1E0002300223000390000F080FED7
:108B1000009B002800D194E2069A591E8A4210DC7C
:108B2000414A0A9894460EAA6344944600229B0048
:108B300063441C68043B22438342FAD1002A00D0DC
:108B4000C0E0069B0EAA013B9B00D358002B00D02F
:108B5000B3E001220C9B043B596801320029FAD092
:108B6000009B9C466244110007921A0001338B421D
:108B700046DC0B9863468046A59C4344A046099C6E
:108B80009B00A1464A449844D30022AA9146049AE5
:108B900099449446089BA59A63448446614494464C
:108BA0009A468B00634400934346586802F036FDB2
:108BB0004B4618605960029B002B24DB4D46039CFA
:108BC0000026002701E0286869680CCC01F01AFF34
:108BD00002000B003000390000F0EEFF083D0600F7
:108BE0000F005C45EFD153469E60DF6004239C4636
:108BF0000433E0449C46009BE144E2449845D3D1D1
:108C0000079B0093D1E600260027ECE794FDFFFFC9
:108C100070E5000018FEFFFFFFFFFF1F0000703E21
:108C20000000704100002040FFFFFF3F0021802234
:108C30005204141B0EAA5450009999420EDD0EA83E
:108C400084469B000EAA8900D25861446344CF48F1
:108C500000E01A68821A04C38B42FAD101243CE76F
:108C6000059B002B06D1009B0EAA013B9B00D5580B
:108C7000ED1517E70022C64B300000F0EDFD00288F
:108C800000D024E100253DE732003B000020C1492F
:108C900002F02AF906000F00002C00D132E7059AF5
:108CA0000020BC4900F0A6FB02000B003000390098
:108CB00002F01AF906000F0024E7012250E700260F
:108CC000002754E64B46059A079388468B000EA969
:108CD000CB58183A08950592002B0DD18C46414689
:108CE000AD4B43449B006344043B58680139183A38
:108CF0000028F9D088460592059A0020A54900F081
:108D000079FB434604000D00002B00DA05E29E00CB
:108D10000EAB9C464346DB0066449C46059370AB15
:108D20009946049F67440097306802F077FC220060
:108D30002B0001F067FE002238607960974B20001D
:108D4000290001F05FFE083F04000D00043EB94514
:108D5000EAD14AAB03939B4600239A46069B4246C0
:108D6000994643460132029204934B46002B00DAA7
:108D7000AAE080208A4B009D9846C00589490026BC
:108D80000027002408E008239C460835E0445445A9
:108D900011DC4346186859682A686B6801F032FE96
:108DA00002000B003000390000F006FF013406001D
:108DB0000F00A145E7DA5B46C0C39B4601239C46F2
:108DC000009BE244083B0093029B9A45CDD1049B53
:108DD0009846A49B022B00DD8EE0002B37DC1FD1D0
:108DE000059B00271D00039B00249C461E00654434
:108DF000083E2A686B683800210000F0DDFE083D5F
:108E000007000C00AE42F4D1089B002B03D0802356
:108E10001B069C4664443A0023000D990A604B608F
:108E20000720079B18409B239B009D443CBC904619
:108E30009946A246AB46F0BD009B0EA95A1E920071
:108E40000EAB9B5807935B025B0A8B5057E6434679
:108E5000002B00DA70E100200021DB004AAAD618BE
:108E600048AF32687368083E00F0A6FEB742F8D1FA
:108E7000089B002B00D025E10B0002004A984B997B
:108E80000D9C2260636002F02FF8434607000C003F
:108E9000002B13DD01254CAEB14638002E00210019
:108EA0004C4601360CCC00F087FEA146B045F7DAFF
:108EB000089B07000C00002B00D015E13A002300AE
:108EC0000D998A60CB60ABE70026002773E701238A
:108ED0009C46009BE1440225002B00DDEBE53200BF
:108EE0003B0000202B4901F0FFFF06000F0009E6C0
:108EF0000024F2E54AAB0393A49B032B00D08FE739
:108F00004346002B00DC14E1039ADB009B46130070
:108F100091465B441E685F68234B43440293DB0029
:108F2000994448AB9A464B465C681B681800210080
:108F300032003B000090019100F03EFE04000D0065
:108F400002000B000098019901F0CEFF3B003200B7
:108F500000F032FE4B469860D9601C605D600823CB
:108F60005B429C46E14426002F00CA45DBD14346C4
:108F7000012B00DCE3E0039A13005B441E685F688A
:108F8000029BDB0099464A44904610E0FFFFFF0039
:108F90000000E03F0000F03FFFFFFF3F0000703E99
:108FA00030E50000FB21F93FFFFFFF1F98464346D5
:108FB0005C681B681800210032003B0000900191A2
:108FC00000F0FAFD04000D0002000B00009801996A
:108FD00001F08AFF32003B0000F0EEFD4346039AA9
:108FE0009860D9601C605D60083B26002F009A42A3
:108FF000DCD14D469446002600244746083565449A
:109000002A686B683000210000F0D6FD083D06009C
:109010000C00AF42F4D1039B4A9F5D689968D86801
:10902000089B002B65D08022120694460D9B654458
:10903000604464441F605D609960D8601E615C613B
:10904000EEE69A464B460793059B30005A4239009C
:10905000089500F0CFF900223A4B06000F0000F00F
:10906000FBFB002824D0384B00223000390001F0EF
:10907000C9FC02F09DFA52460400950002F0CEFAB7
:109080000022304B01F0BEFC02000B003000390022
:1090900001F02AFF02F08CFA0EAA50510122059B22
:1090A000524418339046059393000EAAD45023E6F9
:1090B0005346300039009C0002F07AFA0EAB18518A
:1090C000D04619E680230D9A1B06CB18106053601A
:1090D0000B0002004A984B9901F006FF4346070037
:1090E0000C00002B00DDD5E680231B069C46644463
:1090F000E4E62B003A000D9D2A606B600A00030035
:10910000AA60EB60320023002A616B6188E6099B4C
:10911000DB00009372AB049332E4A49B022B00DDCE
:10912000E8E6002B00DD92E600D079E60027002477
:109130006AE6002600246EE70020002198E600265B
:10914000340068E7000070410000703EF0B5CE4684
:10915000474680B587B000920193474A4B0081464D
:1091600088465B08934207DC4146484602F020FAF5
:109170004146031E484666D04A4643464846414655
:1091800001F040FC04000D0002000B00484641467F
:1091900001F038FC394A3A4B06000F002000290044
:1091A00001F030FC374A384B01F09EFE22002B00C4
:1091B00001F028FC354A364B00F0FEFC22002B0063
:1091C00001F020FC334A344B01F08EFE22002B00CC
:1091D00001F018FC314B324A00F0EEFC0E9B02907D
:1091E0000391002B34D00098019900222D4B01F0FF
:1091F00009FC029A039B049005913000390001F0AC
:1092000001FC02000B000498059901F06DFE22009C
:109210002B0001F0F7FB009A019B01F065FE224A4A
:1092200004000D00214B3000390001F0EBFB02007F
:109230000B002000290000F0BFFC02000B00484694
:10924000414601F051FE07B00CBC90469946F0BD76
:1092500002000B002000290001F0D4FB124A134B3E
:1092600001F042FE32003B0001F0CCFB4A4643468F
:1092700000F0A2FCE7E7C046FFFF3F3E7CD5CF5A97
:109280003AD9E53DEB9C2B8AE6E55A3E7DFEB15787
:10929000E31DC73ED561C119A0012A3F1111813FCD
:1092A000A6F810110000E03F495555555555C53FEA
:1092B00049004B0819007047474AF0B54F469146A0
:1092C0004B005B0D99444646D6464A46C0B505005C
:1092D0000C000E0088460700132A27DC002A4BDB0F
:1092E0003E4B13419A460B0052461340034318D09D
:1092F0003B4A3C4B2800210000F05EFC002200238A
:1093000000F0A0FA002847D0002C04DA80234A4657
:109310005B03134198444646534600279E4338005A
:1093200031001CBC90469946A246F0BD332A08DDA8
:109330008023DB009945F4D102000B0000F03CFCD7
:10934000EFE7294A9446012263445242DA409246AA
:109350000242E6D0224A234B2800210000F02CFCD8
:109360000022002300F06EFA002815D0002C1EDB2E
:10937000534646469F430FE0194A1A4B28002100E6
:1093800000F01AFC0022002300F05CFA002803D051
:10939000002C04DB0027002638003100C1E7640000
:1093A000640825430027002DF6D0104EF4E74B4605
:1093B000142B0BD03422D21A012393405D19BD42E5
:1093C00008D201239C462F00E044D1E7133B9C4682
:1093D000E044CDE72F00CBE701FCFFFFFFFF0F00CC
:1093E0009C7500883CE4377EEDFBFFFF0000F0BF7A
:1093F000002070474B0070B55B0D14000A00002B75
:109400001AD14B005B08034315D0234B002201F017
:10941000F9FA224B9C422DDB0A004B005B0D363BD8
:109420001F4DE318AB422ADC002B0DDD1D4C1B0544
:1094300022401A43110070BD1B4DAB42F0D1020017
:109440000B0000F0B9FBF6E71D00353519DA174BB4
:1094500002009C4209DD0B001548164900F032F865
:10946000134A144B01F0CEFAE5E70B0012481349FA
:1094700000F028F8104A114B01F0C4FADBE70200B3
:10948000E9E7084C363322401B051343190000223C
:109490000B4B01F0B7FACEE700005043B03CFFFFA2
:1094A000FE070000FFFF0F80FF07000050C3000011
:1094B0009C7500883CE4377E59F3F8C21F6EA50105
:1094C0000000903C30B54A00DB0FDB0752081A431E
:1094D000110030BD02B4714649084900095C4900D9
:1094E0008E4402BC7047C046002243088B4274D3AE
:1094F00003098B425FD3030A8B4244D3030B8B4295
:1095000028D3030C8B420DD3FF22090212BA030C9D
:109510008B4202D31212090265D0030B8B4219D37E
:1095200000E0090AC30B8B4201D3CB03C01A52419E
:10953000830B8B4201D38B03C01A5241430B8B42E6
:1095400001D34B03C01A5241030B8B4201D30B03CF
:10955000C01A5241C30A8B4201D3CB02C01A5241F6
:10956000830A8B4201D38B02C01A5241430A8B42B9
:1095700001D34B02C01A5241030A8B4201D30B02A2
:10958000C01A5241CDD2C3098B4201D3CB01C01ABC
:10959000524183098B4201D38B01C01A52414309C6
:1095A0008B4201D34B01C01A524103098B4201D3B4
:1095B0000B01C01A5241C3088B4201D3CB00C01A21
:1095C000524183088B4201D38B00C01A5241430899
:1095D0008B4201D34B00C01A5241411A00D20146BE
:1095E000524110467047FFE701B5002000F0F0F847
:1095F00002BDC0460029F7D076E7704703460B430B
:109600007FD4002243088B4274D303098B425FD37B
:10961000030A8B4244D3030B8B4228D3030C8B42A7
:109620000DD3FF22090212BA030C8B4202D312128D
:10963000090265D0030B8B4219D300E0090AC30B62
:109640008B4201D3CB03C01A5241830B8B4201D30F
:109650008B03C01A5241430B8B4201D34B03C01AF8
:109660005241030B8B4201D30B03C01A5241C30A70
:109670008B4201D3CB02C01A5241830A8B4201D3E1
:109680008B02C01A5241430A8B4201D34B02C01ACB
:109690005241030A8B4201D30B02C01A5241CDD270
:1096A000C3098B4201D3CB01C01A524183098B42BB
:1096B00001D38B01C01A524143098B4201D34B01A4
:1096C000C01A524103098B4201D30B01C01A524107
:1096D000C3088B4201D3CB00C01A524183088B428E
:1096E00001D38B00C01A524143088B4201D34B0077
:1096F000C01A5241411A00D20146524110467047E9
:109700005DE0CA0F00D04942031000D340425340ED
:1097100000229C4603098B422DD3030A8B4212D3AD
:10972000FC22890112BA030A8B420CD389019211DF
:109730008B4208D3890192118B4204D389013AD01C
:10974000921100E08909C3098B4201D3CB01C01AF1
:10975000524183098B4201D38B01C01A5241430904
:109760008B4201D34B01C01A524103098B4201D3F2
:109770000B01C01A5241C3088B4201D3CB00C01A5F
:10978000524183088B4201D38B00C01A5241D9D277
:1097900043088B4201D34B00C01A5241411A00D2F8
:1097A0000146634652415B10104601D34042002BF4
:1097B00000D54942704763465B1000D3404201B573
:1097C000002000F005F802BD0029F8D016E7704728
:1097D0007047C046D0400B1C1141203A03D49C4630
:1097E0001341184363465242934018437047C046A2
:1097F0008446101C62468C46191C634600E0C04635
:109800001FB501F097F8002801D40021C8421FBD00
:1098100010B500F0EFFF4042013010BD10B501F06F
:1098200089F8002801DB002010BD012010BDC046D2
:1098300010B501F07FF8002801DD002010BD0120E7
:1098400010BDC04610B501F011F8002801DC002061
:1098500010BD012010BDC04610B501F007F800286A
:1098600001DA002010BD012010BDC046F0B5CE4683
:10987000474615042D0C2E0080B50704140C3F0C30
:109880009946030C7E435D43674363437F19340C61
:10989000E4199C46A54203D980235B029846C44440
:1098A0004B4643435143250C36046544360C24048F
:1098B000A4195B19591820000CBC90469946F0BDBC
:1098C000F0B54E4657464546DE46E0B543025B0AD4
:1098D000450083B00F1C99462D0EC60F002D57D0A2
:1098E000FF2D24D08020DB00C004184300238146D4
:1098F0009A469B467F3D7C027A00FB0F640A120E5B
:10990000984623D0FF2A4BD0E30080240020E404B3
:109910007F3A1C43AD186B1C474601935346774072
:109920003A000F2B48D87D499B00CB589F46002B0F
:1099300000D085E008339A46063B9B467C027A00BD
:10994000FB0FFF25640A120E9846DBD1002C00D0D5
:1099500090E0524601231A4392460120DBE74C4631
:1099600058461700022824D0032800D1CFE0002257
:10997000002301284DD15802D205400AFF071043A9
:10998000384303B03CBC90469946A246AB46F0BD76
:10999000002B5BD104239A46033B00259B46AAE794
:1099A000FF35002C60D1524602231A439246022012
:1099B000B1E7FF220023DEE74B461B0C9C464B46DB
:1099C0002604360C180461463300220C6446000C51
:1099D00043434E435043544380191A0C1218964285
:1099E00003D9802149028C4664441B041B0C1004DB
:1099F000C01883015E1EB341800E1843130C1B195F
:109A00009B0103431C00230179D5012362081C40FC
:109A10001443019A7F32002A4DDD630704D00F23DF
:109A20002340042B00D00434230103D53C4B019A7E
:109A30001C408032FE2ABCDCA3015B0AD2B29AE74A
:109A40000C239A46093BFF259B4654E7180001F07A
:109A500071FE4A46431F76259A4000236D42914687
:109A60002D1A9A469B4646E7524603231A439246CE
:109A7000032050E7200001F05DFE431F2D1A9C409B
:109A8000763D002047E780230027DB03FF2272E7B3
:109A9000424666E74C463200584662E780234A4613
:109AA000DB031A4222D01C4220D123435B025B0A13
:109AB0004746FF225FE701239A1A1B2A21DC230075
:109AC0000199D3409E318C401A0023005C1EA341B3
:109AD00013435A0704D00F221A40042A00D004333B
:109AE0005A0111D49B015B0A002244E780234A46B5
:109AF000DB0313435B025B0A3700FF223BE7019560
:109B000087E70022002336E70122002333E7802382
:109B1000DB0323435B025B0AFF222CE780E50000A6
:109B2000FFFFFFF770B500283DD0C317C5185D4093
:109B3000C40F280001F0FEFD9E22121A962A07DCAF
:109B4000D2B2082833DD083885406802400A23E095
:109B5000992A0BDD052329001B1AD94003001B336A
:109B60009D402B005D1EAB4119430D00052801DD12
:109B7000431F9D402B000F490B406E0709D00F2655
:109B80003540042D05D004335D0102D59F220B40E2
:109B9000121A9B01580AD2B24002D205400AE407C9
:109BA0001043204370BD002400220020F4E7680227
:109BB000400AF1E7FFFFFFFBF0B54F464646D646A9
:109BC0000C000903C0B5490A470F5E0039431F0363
:109BD000DB0F9C4665007B0A570F1F436D0DE40F9A
:109BE000760DA146C000B846D200AB1B64457BD0C1
:109BF000002B5FDD002E00D0A4E03E00164300D114
:109C000012E15E1E002E00D09EE1871A4346B84244
:109C100080410125C91A4042091A0B0200D431E1E2
:109C200049024E0A002E00D16EE1300001F082FDA3
:109C30000300083B1F2B00DD61E120223900D21A0E
:109C40009E40D1409F400E439D4200DD51E15D1B8F
:109C50006B1C1F2B00DD7CE12021C91A3D00300068
:109C60008F408840DD40791E8F4131000722284314
:109C7000D940002507433A40002A09D00F233B4032
:109C8000042B05D03B1DBB42BF417F42C9191F00B9
:109C90000B0200D426E26A1CC64B55056D0D9A4294
:109CA00000D106E1C44AFF080A40530752023B4371
:109CB000120B8EE0002B00D0B8E06B1C5B055B0D37
:109CC000012B00DC30E1871A4346B842B641CB1A7B
:109CD00076429E1B330200D54CE13B003343A1D1B9
:109CE00000220024002570E0002B00DCE5E0002EBF
:109CF00000D183E0AF4EB54260D0802636043743B2
:109D0000B846382B00DC3EE1434613431F007A1E61
:109D100097413F1887428041404209180B0200D406
:109D2000B0E0A44B01359D4200D1C3E0A24A7B08BC
:109D30000A4001210F401F435108D30707221F4348
:109D40003A4099E79B4EB54238D0802636043743D7
:109D5000B846382B00DDDCE01F2B00DC30E11E00B4
:109D60004746203EF740BC46202B04D04026F31A3D
:109D700046469E403243170063467A1E97411F4372
:109D8000CCE0002B00D104E24346134300D159E15B
:109D90004B07C00818438023C9081B03194208D089
:109DA0004546ED081D4204D14346D00859070843F3
:109DB0002900420FC9007F4D1143C0004B07CA085C
:109DC0007C49C00803438D4268D012036D05120B15
:109DD0006D0D002112031800130B0A0D12051A4312
:109DE000764B2D0513402B435B00E4075B082343B0
:109DF00019001CBC90469946A246F0BD3E00164391
:109E000012D05E1E002E00D000E1871887428041EC
:109E100041444042091801250B0233D5022585E74C
:109E200064463300414610001D00C7E7002D00D0F6
:109E3000DAE00C000443F3D05C1C00D19FE15D4CE0
:109E4000A64200D12FE1DB43382B00DD66E11F2B5A
:109E500000DD83E120240500E41A0F00DD40D94035
:109E6000A0404346A7405B1A441EA04198462F439A
:109E70003843171ABA42924143465242991A6446ED
:109E80003500CAE607223A40002A00D0F6E64B0722
:109E9000CA084849FF083B438D4296D11900114337
:109EA00000D19EE1802109030A431203120B414DA8
:109EB0008FE71500002200238BE7002B00D0C7E0BE
:109EC0006B1C5F057F0D012F00DCF1E0394DAB42CB
:109ED00000D1B9E085180A008542894142444942CF
:109EE00051180722CF076D082F4349083A401D003B
:109EF000C2E607223049ED1A31403A40BCE63E0046
:109F00002838864000279FE6380001F013FC2030F7
:109F10008EE6434613431F007A1E9741C71BB84283
:109F200080414042091A78E60E003B000643134385
:109F3000002D61D1002E00D0F4E0002B00D11BE1F8
:109F400064463900100039E71A4FBB427AD033001B
:109F5000FFE630001F3DE840202B03D04021CB1A04
:109F60009E4037437B1E9F41072207433A40002112
:109F7000002589E7171A4346BA42B641591A764274
:109F80008E1B64464EE61F2B00DDADE020264746C3
:109F9000F61AB740B9461700B246DF404E463E4378
:109FA00037005646B240561EB24117434246DA4089
:109FB0008918AEE6FF070000FFFF7FFFFFFF0F805D
:109FC00020264746F61AB740B9461700B246DF408A
:109FD0004E463E4337005646B240561EB2411743E6
:109FE0004246DA40891A99E77F4CA6425BD080242A
:109FF00024045B42214327E7002E0CD1002B00D123
:10A00000CBE0644639001000774DD7E6764FBB426F
:10A0100018D0330075E6002B14D04B07C008184346
:10A020008023C9081B03194207D0FC081C4204D135
:10A030007907D0080843E14621004C46420FC90089
:10A040001143C000684DB9E61D0000220023C0E6A0
:10A05000002D5BD10D00054300D1E2E65D1C00D16F
:10A06000B0E0614DAE421FD0DB43382B71DC1F2BBB
:10A0700000DD96E020250F00ED1AAF40B94607003D
:10A08000AA46DF404D463D432F005546A840D940E3
:10A09000451EA84188440743BF1897429241514248
:10A0A000414435003AE6644635004146100085E6F5
:10A0B0000B000343002D00D063E6002BF5D0434690
:10A0C000134300D17AE68718874280410722414432
:10A0D000404209183A400B0200D4D5E6434B013503
:10A0E0001940C9E5380069E61E004746203EF740A2
:10A0F000BC46202B04D04026F31A46469E403243ED
:10A10000170063467A1E97411F4302E6364DAE4262
:10A11000CAD080252D045B422943A6E70843411E8F
:10A120008841A6E6002B00D148E6871A4346B8428C
:10A13000B641CB1A76429E1B33024BD5171A4346C3
:10A14000BA429241591A5242891A072264463A4049
:10A1500092E501430F00791E8F419DE71C000F001F
:10A16000203CE740202B03D04024E31A99400843C9
:10A17000411E884138437CE60022002425E6171A58
:10A180004346BA429241591A5242891A64463500EE
:10A1900043E541461000144D10E6802200241203CE
:10A1A00080E61D000F00203DEF40BC46202B03D071
:10A1B0004025EB1A9940084307006346781E874103
:10A1C0001F4369E7871897429B4141445B42C91886
:10A1D0003500A3E53B003343CED0072231003A409F
:10A1E00052E600231A00F4E5FF070000FFFF7FFF9F
:10A1F000F0B55746DE464E464546E0B58346070075
:10A200000E03480085B092461C00360B400DCD0F62
:10A21000002800D19DE0954B984239D08023F6006C
:10A220001B041E43924A7B0F334399469446030016
:10A230006344009300230026FF00029323031B0BBB
:10A2400098466300E40F52465B0D019400D1B3E0E1
:10A2500086498B4200D19EE04246D1008022120402
:10A260000A435146490F11438B46814952468C4659
:10A2700000996344CB1A0021D20000932B00634065
:10A280009A460F2E00D905E17A4BB6009B599F469E
:10A290005B463343994600D0B8E0022308260027E6
:10A2A00000900293CAE7CB463A0002990195019BC0
:10A2B0009A46022927D0032900D180E2012944D0FF
:10A2C0006D49009B8C4663441C00002C38DD53070D
:10A2D00000D013E2D2085B46DB0109D55946674B33
:10A2E00019408B468021C9008C46009B63441C00AA
:10A2F000634B9C4207DC5B4664055F075B021743C8
:10A300001B0B620D02E000230027584A00211B03AB
:10A310001C0B0B0D1B05234314055A4A3800134030
:10A320001C4353466400DB0764081C43210005B04E
:10A330003CBC90469946A246AB46F0BD0122524233
:10A3400001231B1B382B00DCADE10022002300277A
:10A35000DCE75B46334399465ED0002E00D18AE1AC
:10A36000300001F0E7F903000B3B1C2B00DD7BE123
:10A370001D22D31A5A460100DA4008398E401300D4
:10A380005F46334399468F403F4B00261B1A00938C
:10A390000023029352E7414653460B433B499B46F9
:10A3A0008C46009B634400935B46002B3BD1022309
:10A3B00000221E43022161E7434613439B4637D0E8
:10A3C0004346002B00D162E1404601F0B3F903009F
:10A3D0000B3B1C2B00DD53E102004146083A914043
:10A3E00088461D21CB1A5146D9400B0041460B43EC
:10A3F0009B46534693401A00009B25499C46604467
:10A4000003008C4663440093002137E70323B146E1
:10A4100000900C26029311E70023009301330426D9
:10A42000002702930AE70323C3461E43032125E7BF
:10A4300001331E430022012120E700239A46802396
:10A4400000271B03094A61E7802349461B03194281
:10A4500000D1E2E05946194200D0DEE00B431B0375
:10A4600017001B0BA246014A50E7C046FF07000039
:10A4700001FCFFFFC0E50000FF030000FFFFFFFE3F
:10A48000FE070000FFFF0F800DFCFFFF01F8FFFF3C
:10A49000F3030000D94500D9CBE000D1C6E03C0071
:10A4A00048460027009B013B00935B46160E1B02AB
:10A4B0001E431302984633041B0C9946310C01913C
:10A4C000FFF798F84A4642430B04210C0500194354
:10A4D0008A4207D98919013D8E4203D88A4201D99F
:10A4E000851E8919881A0199FFF784F809048C469A
:10A4F0004A46210464464243090C030021438A4230
:10A5000004D98919013B8E4200D8F1E02D041D4386
:10A51000AB464346891A4246280C12041D0C5B4682
:10A52000140C22001B041B0C5A4303946B4344433A
:10A53000029568431B19150CEB189C4203D9802423
:10A540006402A44660441C0C15041B042D0C201846
:10A550005D19814277D373D00C1AA24A7D1BAF429A
:10A56000BF419446009B7F426344E01B1C0086422F
:10A5700000D1DBE00199FFF73DF84A4642430B0466
:10A58000290C070019438A4207D98919013F8E42D5
:10A5900003D88A4201D9871E8919881A0199FFF7C1
:10A5A00029F809044A46894629044D464243090CC4
:10A5B000030029438A4207D98919013B8E4203D8F7
:10A5C0008A4201D9831E89193F04891A3A00039FE0
:10A5D0001A43380013041B0C584381460298150C8B
:10A5E0006F43434345434846000C8446DB196344AC
:10A5F0009F4203D9802040028446654448461F0C90
:10A6000000041B04000C7D191818A94200D284E034
:10A6100000D17FE001231A4357E680234A461B03FB
:10A6200013431B031B0BAA466F4A6FE6BA4200D9BD
:10A6300035E74B46DC0758087B081C43FF0734E727
:10A640000024AF4289D247444745A4415B46644257
:10A65000A4196418013BA6421ED2A0426DD800D1B5
:10A66000B6E0241A9B4678E703005A46283B9A40F6
:10A670000027914688E6584601F05CF8203072E6E3
:10A6800003005246283B9A4093460022B4E65046C7
:10A6900001F050F820309AE6A642E2D1B845DCD964
:10A6A000341A9B4659E71F2B65DC504C0099A44691
:10A6B0005C46614408008C4011008240D940501E25
:10A6C00082410C4314435A46DA401300620709D012
:10A6D0000F222240042A05D02200141D94428941F1
:10A6E00049425B181A0262D50122002300270DE6B9
:10A6F0008A4200D80AE7831E891907E70F2313400F
:10A70000042B00D1E6E5171D9742924153429B442A
:10A71000FA08E0E5002800D1D7E57118531EB142D0
:10A7200027D3A94215D358D01A0073E7002B00DCB9
:10A7300004E6012300229B44CDE50223474447451C
:10A7400089415B429C46494289190C19E344241A09
:10A7500003E743465F0047459B41B8465B429E196D
:10A76000023A8919A94200D054E7404500D051E788
:10A77000ABE51A00F6E71F215F4649420C1BE74094
:10A78000202B07D01A49009B8C46634418005B4677
:10A7900083401A43501E82413A4307270023174043
:10A7A00009D00F21002311401400042995D1220063
:10A7B0005F075B021B0BD20817430022A6E580232C
:10A7C00059461B030B431B0317001B0B064A9DE551
:10A7D000BD42B2D89B460024BFE68045B9D31A00DB
:10A7E000C3E7C046FF030000FF0700001E0400008F
:10A7F0003E040000F0B54F464646D6468446C0B5F6
:10A800008046194E18030F034D00000B5C00824672
:10A810003F0B6D0DC90F9146640DDB0F0120B54252
:10A820000AD0B44203D0A54201D157450CD01CBC7C
:10A8300090469946A246F0BD66463E43F7D1AC42EB
:10A84000F5D154461443F2D10120C845EFD19942C5
:10A8500007D0002DEBD163461F433800471EB84197
:10A86000E5E70020E3E7C046FF070000F0B54F46EC
:10A870004646D6464D00C0B50E03C90F8A462C4940
:10A880001F035C008046360B6D0D91463F0B640D37
:10A89000DB0F8D421ED08C4216D0002D1ED13043CE
:10A8A0008446002C01D13A4323D06246002A1AD0B4
:10A8B0009A4529D0514602200139084001381CBC74
:10A8C00090469946A246F0BD39001143E5D00220DA
:10A8D0004042F4E73043FAD1AC420FD0002C0FD104
:10A8E0003A43E7D00CE00122013B934318000130CA
:10A8F000E5E763460020002BE1D0DBE73A43E6D1F1
:10A900009A45D7D1A542D5DCA54205DBBE42D1D8B8
:10A9100008D00020BE42D2D25046012301389843CD
:10A920000130CCE7C845C5D80020C845F4D3C6E7F8
:10A93000FF070000F0B54F464646D6464D00C0B56D
:10A940000E03C90F8A462E491F035C008046360B52
:10A950006D0D91463F0B640DDB0F8D4218D08C427C
:10A9600011D0002D18D130438446002C1ED13A431B
:10A970001CD163460020002B30D051460220013903
:10A98000084001382AE039001143EAD0022025E0CE
:10A990003043FBD1AC4226D0002C26D13A4324D1FF
:10A9A0005146022001390840013817E06246002A6A
:10A9B0000FD09A45E1D1A54205DBBE42DDD819D0C2
:10A9C0000020BE420AD2504601230138984301308C
:10A9D00004E00122013B9343180001301CBC904667
:10A9E0009946A246F0BD3A43D0D19A45C5D1A54279
:10A9F000C3DCE0E7C845C0D80020C845E3D3EDE795
:10AA0000FF070000F0B55746DE464E464546E0B526
:10AA1000834606000F03480087B092461D003F0B97
:10AA2000400DCC0F002800D16FE0DE4B984238D0AB
:10AA30008023FF001B041F43730F3B430193DA4B3A
:10AA40000027994600239B46F60081442B036900AA
:10AA50001B0B52469846490DED0F002900D185E0A9
:10AA6000D04B994200D173E04346DA0080231B04A7
:10AA700013435246CC48520F84461343524600209B
:10AA80006144D20089442100694000918C46012133
:10AA900049448A460F2F00D990E0C449BF00CF59DE
:10AAA000BF465B463B43019300D06AE1022308277F
:10AAB000002681469B46C9E732005846019B614605
:10AAC0000091022800D175E0032800D1FEE10128A1
:10AAD00000D02CE100230027002600253F032A0D8B
:10AAE0003F0BB34812053A4302401B051343009A3B
:10AAF0005B00D1075B080B433000190007B03CBC7A
:10AB000090469946A246AB46F0BD5B463B43019357
:10AB100000D12FE1002F00D1A5E1380000F00AFE9E
:10AB200003000B3B1C2B00DD96E11D22D31A5A4675
:10AB30000100DA405E4608398F4013008E403B43E7
:10AB400001939C4B00271B1A994600239B467DE7E7
:10AB5000414653460B4393498C46E144002B00D0B9
:10AB60001AE102220220174300228CE7134300D18E
:10AB70000DE14346002B00D181E1404600F0DAFDB3
:10AB800002000B3A1C2A00DD72E10100434608393D
:10AB90008B4098461D239A1A5346D3401A004346C9
:10ABA000134352468A404946081A824989468144DD
:10ABB000002068E77B4B002700268EE7140C120468
:10ABC000120C1100370C3604350C794328008C46E2
:10ABD0002E0060436044834656432100300C80467B
:10ABE0005846794340440291844506D988468021DD
:10ABF00049028C46E044414602913604010C360C71
:10AC000000048B4681191E0C1B041B0C03911900B8
:10AC100079438C46280075436544A8465843050C83
:10AC200045447743A94203D9802149028C466744B1
:10AC3000290C8C4639000004000C2D042D186144A9
:10AC4000AB4405915946049101990F043F0C080C3F
:10AC5000390051434243904602008C46090C8B4612
:10AC600062437C4344445C44A04503D980214902AB
:10AC700088464244210C884661460904090C8C46EA
:10AC800039005943434370437E430F0CF6182404A4
:10AC9000BE19644442448C46B34203D980235B020C
:10ACA00098464044029B61469846049B37044344BF
:10ACB0009B46AB45AD416B420D0405992D0C8C466E
:10ACC0007F196744FD18A8465D462D19A542A44189
:10ACD00093466442A446C344DC448F42BF41984536
:10ACE0009B4193459241A445A4415B427F421F434F
:10ACF000360C52426442BF192243BF1862463818CC
:10AD00004302D20D039913436A020A43501E824143
:10AD10006146ED0D2A434E023243D90100D4B3E01F
:10AD20000126500832400243DE0732435B08224CC2
:10AD30005444002C62DD510709D00F201040042834
:10AD400005D0101D9042924152429B180200D90139
:10AD500004D580241948E400034054441848844230
:10AD600000DD27E75E075B02D2081F0B6305164371
:10AD70005B0DB2E6002399460133042700269B466B
:10AD800064E60323019781460C279B465EE6012279
:10AD900001201743002276E6032303201F43434686
:10ADA00071E6C046FF07000001FCFFFF00E600005F
:10ADB000FFFF0F800DFCFFFFFF030000FFFFFFFE02
:10ADC000FE0700000023802700933F030026434B2B
:10ADD00083E6019B3200A446584670E6AC466EE618
:10ADE000802701993F0339422DD03B422BD11F438D
:10ADF0003F033F0B00951600384B6EE601252D1BD7
:10AE0000382D00DD66E61F2D40DC35481C0050441F
:10AE1000160082408440EE40501E82413443144369
:10AE2000EB40620709D00F222240042A05D02200FD
:10AE3000141D9442804140421B181A023ED5012342
:10AE40000027002649E68027019B3F031F433F035D
:10AE50003F0B0094214B40E603005A46283B9A40A2
:10AE6000002601926DE6584600F064FC203057E65B
:10AE700003005246283B9A401300002293E65046B6
:10AE800000F058FC20307BE6CA4650E71F201E0029
:10AE90004042041BE640202D03D0124C5444A340F2
:10AEA0001A43501E8241324307260027164009D01C
:10AEB0000F200023104014000428B9D122005E079F
:10AEC0005B021F0BD2081643002306E680273F03D0
:10AED0001F433F033F0B1600004BFEE5FF0700003A
:10AEE0001E0400003E040000F8B557464E46454695
:10AEF000DE460C000903E0B5490A460F5F00314306
:10AF00001E03DB0F760A9B46530F3343C84E650082
:10AF1000C000E40FD2006D0DA24681467F0D9C4615
:10AF20009046B74200D1B9E05B46012673409B468C
:10AF3000EE1BA34500D183E0002E63DD002F00D07F
:10AF4000B1E06346134300D123E1731E002B00D010
:10AF5000BAE1861A6346B04280410125C91A4042CF
:10AF6000091A0B0200D447E149024B0A98464346AE
:10AF7000002B00D189E1404600F0DCFB0300083BD8
:10AF80001F2B00DD7CE120223000D21A4146D04048
:10AF9000994002009E400A439D4200DD6AE15D1B2C
:10AFA0006B1C1F2B00DD94E1202110003500C91A15
:10AFB0008E40DA408840DD40711E8E41110007222C
:10AFC0002843002506433240002A09D00F2333408E
:10AFD000042B05D0331DB342B641764289191E00B9
:10AFE0000B0200D43DE26A1C914B55056D0D9A424F
:10AFF00000D119E18F4AF6080A4057075202374339
:10B00000120B9BE0002E00D0C5E06E1C7605760D7D
:10B01000012E00DC48E16746861ACB1BB042BF41D7
:10B020007F42B8461F004346FF1A3B00B8461B024A
:10B0300000D55FE137439AD100220024002579E052
:10B04000002E00DCFAE0002F00D18DE0784B9D420D
:10B0500067D0802367461B041F43BC46382E00DCA4
:10B0600052E1634613435A1E93411E1886428041A3
:10B07000404209180B0200D4BEE06D4B01359D42E1
:10B0800000D1D2E06B4A73080A4001210E401E43F2
:10B090005108D30707221E43324095E71E0016438E
:10B0A00000D045E740E7624B9D423AD08023674697
:10B0B0001B041F43BC46382E00DDEBE01F2E00DCD6
:10B0C0003AE133006746203BDF403B00202E05D0AD
:10B0D0004027BF1B6646BE40324390464646721E1E
:10B0E00096413343DAE0002B00D114E26346134368
:10B0F00000D168E180234E07C008C9081B0306433E
:10B10000194208D06046C008184204D163460100C5
:10B11000D2085E071643F3009946C900720F444DEA
:10B1200011434B46DE08424B4F073743CA089D4246
:10B1300000D16EE012036D05120B6D0D002112039C
:10B14000130B0A0D12051A433B4B2D0513402B43DD
:10B150005B00E4075B082343380019003CBC9046C1
:10B160009946A246AB46F8BD6346134311D0731E01
:10B17000002B00D007E1861886428041614440429E
:10B18000091801250B0237D502257BE73E006146F1
:10B1900091463500C5E75C46002D00D0E1E00B008C
:10B1A0000343F3D0731C00D1ACE1214B9F4200D18B
:10B1B0003AE1F343382B00DD6FE11F2B00DD8CE11A
:10B1C00020250E00ED1AAE40B0460600AA46DE402D
:10B1D000454635432E005546D940A8406346451E96
:10B1E000A8415B1A9C463043161AB242924163460C
:10B1F0005242991A3D00B4E607223240002A00D09C
:10B20000E4E60B4BF6084F073743CA089D4200D0CF
:10B2100090E73B00134300D1A6E180231B031A43B0
:10B220001203120B024D89E715000022002785E763
:10B23000FF070000FFFF7FFFFFFF0F80002E00D001
:10B24000C7E06B1C5E05760D012E00DCF0E0C84DFA
:10B25000AB4200D1B9E085180A00854289416244B9
:10B26000494251180722CE076D082E434908324043
:10B270001D00A9E6BF49ED1A114007223240A3E69E
:10B28000320028388240002686E6300000F052FA6C
:10B29000203073E6634613435A1E9341C61AB042E8
:10B2A00080414042091A5CE60E0067460643174398
:10B2B000002D5ED1002E00D0F3E0002F00D11EE162
:10B2C0005C46614691462CE7A94FBE427BD01E00EA
:10B2D000F1E610001F3DE840202B03D04021CB1A9F
:10B2E0009A401643731E9E410722064332400021B6
:10B2F000002583E7161A6346B2428041591A40423C
:10B300000B1A98465C4632E61F2E00DDABE0202784
:10B31000BB1B9A4663465746BB40994613004F46AF
:10B32000F3401F433B005746BA40571EBA411343F0
:10B330006246F240891898E62027BB1B9A4663466E
:10B340005746BB40994613004F46F3401F433B000E
:10B350005746BA40571EBA4113436246F240891A13
:10B360009CE7834B9F425FD080252D047342294385
:10B3700020E7002E0CD1002F00D1D0E05C466146C2
:10B3800091467B4DCDE67A4FBE421CD01E0065E64D
:10B39000002F18D0C0084E0706438020C9080003BC
:10B3A000014208D06346DC08044204D12100DA4699
:10B3B000D2085E071643F300994601245346C9009C
:10B3C000720F11431C406A4DABE61D00002200279E
:10B3D000B4E6002D59D10B00034300D1D6E6731C0F
:10B3E00000D1B2E0624B9F421ED0F343382B6FDC9A
:10B3F0001F2B00DD97E020250E00ED1AAE40B04671
:10B400000600AA46DE40454635432E005546A84074
:10B41000D940451EA8418C440643B6189642924135
:10B42000514261443D0025E63D006146914678E683
:10B430000B000343002D00D055E6002BF5D06346EA
:10B44000134300D16DE68618864280416144404234
:10B45000091800220B0200D4D0E6464B01351940F2
:10B46000B2E5B1465DE633006746203BDF403B0076
:10B47000202E05D04027BF1B6646BE403243904673
:10B480004646721E96413343EFE5394B9F42CBD07F
:10B4900080252D0473422943A8E70843411E8841B3
:10B4A000A2E6002F00D13CE66346861ACF1AB042CE
:10B4B0009B415B42FB1A98461B024ED5161A634607
:10B4C000B2429241591A5242891A5C4600227BE5E7
:10B4D00001430E00711E8E419FE71D000E00203DAE
:10B4E000EE40B046202B04D04025EB1A994008438B
:10B4F000814648464346411E8841184374E600226F
:10B50000002417E6161A6346B2429241591A524273
:10B51000891A3D0025E561469146154D01E68022D8
:10B520000024120379E61D000E00203DEE40B046D7
:10B53000202B04D04025EB1A9940084381464E4603
:10B540004346711E8E411E4367E7861896429B4113
:10B5500061445B42C9183D008CE547463743CED075
:10B5600007224146324049E600273A00E6E5C04658
:10B57000FF070000FFFF7FFF70B50C4E0D031C039B
:10B5800049005B002D0B490D240B5B0DB14208D027
:10B59000064900208B4203D114432000441EA041E1
:10B5A00070BD05430120002DFAD1F1E7FF0700002F
:10B5B00030B5144D0A034B00120B5B0DC90F00246C
:10B5C000AB4211DD104CA34210DC80246403224303
:10B5D0000E4CE41A1F2C0CDD0D48C31ADA40130080
:10B5E0005C42002900D11C00200030BD094BCC1862
:10B5F000FAE7094DE040AC4663449A401300034328
:10B60000EEE7C046FE0300001D0400003304000006
:10B6100013040000FFFFFF7FEDFBFFFF70B5002864
:10B620002DD0C317C5185D40C40F280000F082F864
:10B63000154B1B1A5B055B0D0A2815DD0B38854081
:10B6400000222D032D0B002110002D030A0D2D0BC0
:10B6500012052A430D4D1B052A4013435B00E407E6
:10B660005B082343190070BD020029001532914088
:10B670000A000B21081AC5402D032D0BE3E7002417
:10B68000002300250022DEE71E040000FFFF0F80DC
:10B690004100090E4B1C70B5DBB24602750AC40F9F
:10B6A000012B14DDE0239B006D07360BCB18002126
:10B6B0000A0D280012051C4D32435B052A405B0829
:10B6C00013435B00E4075B082343190070BD0029A6
:10B6D00014D1002D1ED0280000F02CF80A281CDC04
:10B6E0000B232A001B1ADA40030015339D400F4B31
:10B6F00012031B1A5B05160B5B0DD8E7002D06D055
:10B70000320B802636036D071643094BCFE7084BF3
:10B710000026CCE700230026C9E703002A000B3BE4
:10B720009A400025E3E7C046FFFF0F808903000031
:10B73000FF0700001C2101231B04984201D3000CC9
:10B7400010391B0A984201D3000A08391B09984294
:10B7500001D30009043902A2105C40187047C046AA
:10B7600004030202010101010000000000000000CA
:10B7700030B51C00094B05001B6885B0D868084B24
:10B78000002A01D1074B1A000292019300912B006D
:10B790002200054900F026F800F0A6FD84000020F4
:10B7A00040E60000B8D300004DE60000014B1868E9
:10B7B0007047C04684000020084B10B50400002BE1
:10B7C00002D0002100E000BF054B1868836A002BFF
:10B7D00000D09847200001F05DFBC046000000004B
:10B7E0007CE600000EB403B5010003AB044804CBB3
:10B7F0000068019300F076F802B008BC03B0184767
:10B800008400002070B500260C4D0D4C641BA41064
:10B81000A64209D1002601F03FFB0A4D0A4C641BE9
:10B82000A410A64205D170BDB300EB58984701366D
:10B83000EEE7B300EB5898470136F2E754020020D8
:10B84000540200205402002064020020002310B59E
:10B850009A4200D110BDCC5CC4540133F8E710B556
:10B86000884202D98B18984203D3002307E08B5CEF
:10B870008354013AFBD210BDCC5CC45401339A42CC
:10B88000FAD1F8E703001218934200D170471970FB
:10B890000133F9E7936810B5013B9360002B04DA9C
:10B8A0009469A34207DB0A2905D01368581C10606D
:10B8B0001970080010BD00F04BFC0100F9E7F8B565
:10B8C00006000F001400D518AC4201D1002007E09B
:10B8D00021783A003000FFF7DDFF0134431CF3D13B
:10B8E000F8BD0000F0B59FB002900F001600059360
:10B8F000002805D083690493002B01D100F0F4FDEA
:10B900007B4B9F425BD1029B5F68BB891B0762D563
:10B910003B69002B5FD0002306AC63612033637664
:10B920001033A37635002B78002B01D0252B5CD16A
:10B93000AB1B04930CD0320039000298FFF7BFFF15
:10B94000431C00D1C4E06269049B94466344636174
:10B950002B78002B00D1BBE0012200235242626011
:10B9600002A9543252186E1C2360E360A360137066
:10B97000A365317805225F4800F0D4FE751C0028CD
:10B9800035D12268D30604D5532302A95B182021A0
:10B990001970130704D5532302A95B182B211970C2
:10B9A00033782A2B2CD0350000210A20E3682A782E
:10B9B0006E1C303A092A64D900292ED026E04E4B5D
:10B9C0009F4202D1029B9F689FE74C4B9F429CD1B4
:10B9D000029BDF6899E73900029800F00FFC00280D
:10B9E00099D0012040421FB0F0BD01359BE7414B8B
:10B9F0002268C01A01238340134323602E00B8E756
:10BA0000059B191D1B680591002B01DB099304E0C0
:10BA10005B42E3600223134323602B782E2B0AD171
:10BA20006B782A2B35D1059B02351A1D1B680592B0
:10BA3000002B2BDB0793324E29780322300000F0D5
:10BA400071FE002806D04023801B83402268013508
:10BA500013432360297806222A486E1C217600F0C1
:10BA600061FE00283AD0284B002B25D10722059BE8
:10BA700007339343083305936369039A9B18636103
:10BA800050E7434301219B18350090E701235B42B7
:10BA9000D0E700230A201A000135636029786E1C64
:10BAA0003039092903D9002BC5D00792C3E7424397
:10BAB000012352183500F1E705AB00933A00134B10
:10BAC0002100029800E000BF0390039B0133D3D113
:10BAD000BB895B0600D584E70B9884E705AB009330
:10BAE0003A000A4B2100029800F080F8ECE7C046CB
:10BAF000D4E6000080E60000F4E60000B4E60000B2
:10BB000086E600008AE6000000000000BFB80000E2
:10BB1000F7B5150001938A680B6900900C009342F9
:10BB200000DA130022002B6043321278002A01D081
:10BB300001332B6023689B0602D52B6802332B60F0
:10BB4000062723681F4027D0230043331B785A1E43
:10BB500093412268920630D4220001994332009822
:10BB6000089EB047431C25D0062320682A68E16858
:10BB700003400025042B03D18D1AEB43DB171D4036
:10BB8000A3682269934201DD9B1AED180027BD428C
:10BB900020D1002010E00137E3682A689B1ABB42DD
:10BBA000D2DD22000123193201990098089EB04786
:10BBB000431CF0D101204042FEBD3020E11843314A
:10BBC000087021005A1C45310978A218433202330B
:10BBD0001170C1E7220001231A3201990098089ED2
:10BBE000B047431CE6D00137D1E70000F0B589B07B
:10BBF00004920A0043320593039002920A7E0C00DD
:10BC00000E9B6E2A00D186E01FD8632A33D008D855
:10BC1000002A00D18CE0582A4DD0250042352A70E8
:10BC200030E0642A01D0692AF7D1196825680A1D15
:10BC3000280629D508681A60002803DA2D23029AFD
:10BC4000404213706B4E0A274FE0732A74D008D815
:10BC50006F2A1FD0702AE0D1202209680A4322608F
:10BC600003E0752A16D0782AD7D1220078214532F0
:10BC70001170614E22E025001A684235111D1960CD
:10BC800013682B70012365E008681A606906D3D534
:10BC900000B2D1E719682568081D186008682E06EB
:10BCA00005D5544E08276F2A1BD00A2719E06D06C8
:10BCB000F7D580B2F5E745314E4E0A701868226814
:10BCC000011D00681960150621D5D30702D5202370
:10BCD0001A4322601027002803D1202322689A43A8
:10BCE00022602300002243331A706368A360002B94
:10BCF00058DB0422216891432160002854D1029D21
:10BD0000002B5AD02500337842352B7055E055066C
:10BD1000DBD580B2D9E71A680D68101D4969186033
:10BD200013682E0601D5196002E06D06FBD5198057
:10BD30000023029D23614FE01A68111D19601568E8
:10BD400000216268280000F0EDFC002801D0401BB3
:10BD50006060636823610023029A13703CE02369EA
:10BD60002A0004990398059DA847431C3ED02368E8
:10BD70009B0715D4079BE068984239DA180037E032
:10BD800022000123193204990398059EB047431CF1
:10BD90002CD00135E368079A9B1AAB42F0DCE9E747
:10BDA0000025F7E70028ADD0029D3900FDF722FC01
:10BDB000735C013D2B700028F7D1082F09D123684F
:10BDC000DB0706D563682269934202DC3023013D1C
:10BDD0002B70029B5B1B2361059B07AA009321002C
:10BDE000049B0398FFF794FE431CB8D10120404206
:10BDF00009B0F0BD91E60000A2E600000D4B70B561
:10BE00001C680500A36B002B0FD1182000F06EFCFE
:10BE1000094BA0630360094B01224360084B836018
:10BE20000B2383810023026143610022A36B1D6108
:10BE30005A6170BD840000200E33CDAB34126DE624
:10BE4000ECDE0500124B10B51C68A36B002B0FD164
:10BE5000182000F04BFC0F4BA06303600E4B012237
:10BE600043600E4B83600B23838100230261436197
:10BE7000A46B0B4A206961690A4BFDF7F7FC0122AC
:10BE8000002380185941206161614800400810BDBD
:10BE9000840000200E33CDAB34126DE6ECDE0500DD
:10BEA0002D7F954C2DF451580CB430B5164B9DB0E8
:10BEB0000C1E1D6808DA8B2301202B6040421DB048
:10BEC00030BC08BC02B01847822302A99B008B81BA
:10BED0000023029008619C4200D0631E8B604B617E
:10BEE00001235B42CB81209A21AB2800019300F013
:10BEF00055FD431C01DA8B232B60002CDFD000237F
:10BF0000029A1370DBE7C046840000200EB400B52F
:10BF10000B499CB01DAB0290069007910491094813
:10BF2000094904CB0591006802A9019300F036FD90
:10BF30000023029A13701CB008BC03B01847C04617
:10BF4000FFFFFF7F840000200802FFFF020010B502
:10BF50001378541C002B05D1CC5CD4540133002C35
:10BF6000FAD110BD2200F3E7C9B20378002B04D048
:10BF70008B4200D170470130F7E74B4259414942AB
:10BF80000840F7E702780B78002A03D0013001312E
:10BF90009A42F7D0D01A70470023C25C0133002ABE
:10BFA000FBD1581E7047002330B59A420AD0013A9F
:10BFB000C45CCD5CAC4204D1934202D00133002C6E
:10BFC000F6D1631B180030BD30B50500002A00D142
:10BFD00030BD0C78013A6B1C2C700131002C05D15E
:10BFE0009A189A42F4D01C700133FAE71D00EDE76D
:10BFF00010B50378002B0FD10B785A4253415B42A6
:10C00000184010BD0023CA5C002AFAD0C45C9442D8
:10C0100001D10133F7E701300378002BF2D118008A
:10C02000EFE70000F0B51F000E0087B0059001910A
:10C0300002920C98347800F0EAFA0822001943784A
:10C04000751C134036D12D2C36D1B51C74780126C1
:10C05000002F62D0102F09D1302C07D120222B784D
:10C060009343582B54D110276C7802352D4B39004F
:10C07000F31818000393FDF7BDFA04910121002382
:10C08000494202008C4618002100303909291AD88B
:10C090000C00A74223DD591C09D06346824206D317
:10C0A00002D10499A14202DB0123784320182C78A5
:10C0B0000135E9E72E00BCE72B2C01D01E00C7E7B5
:10C0C000B51C7478FAE721004139192901D8373CA9
:10C0D000DFE721006139192901D8573CD9E75A1CFB
:10C0E00008D1059A23331360029B0398002B09D1D2
:10C0F00007B0F0BD002E00D04042029A002AF7D0CF
:10C10000002B01D06B1E0193029B019A1A60EFE78E
:10C110003024002FAAD10827A8E7302C9ED00A2768
:10C12000A4E7C046FFFFFF7F37B51300064A0500AE
:10C130001068046A002C00D1044C0A000094290005
:10C14000FFF770FF3EBDC04684000020E8000020DD
:10C15000F8B505000E001400002804D08369002BF8
:10C1600001D100F0C1F9224B9C422DD16C68A3692A
:10C17000A360A3891B0731D52369002B2ED0236828
:10C180002269F7B2981A6369F6B2834205DC21008E
:10C19000280000F03BF9002826D1A3680130013BBC
:10C1A000A36023685A1C22601F706369834204D015
:10C1B000A389DB071AD50A2E18D12100280000F028
:10C1C00025F9002812D00FE00A4B9C4201D1AC683F
:10C1D000CDE7094B9C42CAD1EC68C8E72100280092
:10C1E00000F00CF80028CAD0012676423000F8BDD5
:10C1F000D4E60000F4E60000B4E60000364B70B56B
:10C200001D6806000C00002D05D0AB69002B02D183
:10C21000280000F069F9314B9C420FD16C680C2367
:10C22000E25E93B219072DD4D90611D40923012057
:10C23000336037331343A381404270BD284B9C4287
:10C2400001D1AC68EBE7274B9C42E8D1EC68E6E70C
:10C250005B0713D5616B002908D023004433994252
:10C2600002D0300000F06AFA002363632422A3891D
:10C270009343A38100236360236923600823A28979
:10C280001343A3812369002B0BD1A0218022A38912
:10C29000890092000B40934203D02100300000F04F
:10C2A000E1F90123A289134011D00023A36063693F
:10C2B0005B42A361002023698342BED10C23E25E6E
:10C2C0001306BAD540231343A3810138B5E792077B
:10C2D00000D46369A360EDE784000020D4E6000089
:10C2E000F4E60000B4E6000010B5062000F090FC73
:10C2F000012000F0CFFD0000F7B58A8905000C0091
:10C30000130760D44B68002B04DC0B6C002B01DCA2
:10C310000020FEBDE76A002FFAD000232E682B60B4
:10C3200080235B01216A1A4034D0606DA3895B07CA
:10C3300006D56368C01A636B002B01D0236CC01A4A
:10C340000200216A00232800E76AB847A189431C3C
:10C3500006D12B681D2B30D82B4ADA40D3072CD5B9
:10C360000023636023692360CB0405D5431C02D1FD
:10C370002B68002B00D16065616B2E600029C7D04F
:10C3800023004433994202D0280000F0D7F900205E
:10C390006063BEE701232800B847431CC6D12B6861
:10C3A000002BC3D01D2B01D0162B01D12E60AFE77F
:10C3B0004023A2891343A381ABE740230B43012011
:10C3C000A3814042A5E70F69002FA1D00B680F6041
:10C3D000DB1B01930023920700D14B69A360019BF3
:10C3E000002B00DC94E7019B3A00216A2800A66A32
:10C3F000B047002803DC4023A2891343DFE7019BF9
:10C400003F181B1A0193EAE7010040200B6970B541
:10C4100005000C00002B01D1002070BD002804D0C5
:10C420008369002B01D100F05FF80B4B9C4209D1CE
:10C430006C680C22A35E002BEED021002800FFF7D1
:10C440005BFFEAE7054B9C4201D1AC68F1E7044B86
:10C450009C42EED1EC68ECE7D4E60000F4E6000084
:10C46000B4E60000002310B504000360436083605D
:10C4700081814366C281036143618361190008229F
:10C480005C30FFF7FFF9054B24626362044BA36243
:10C49000044BE362044B236310BDC04651CC000043
:10C4A00079CC0000B1CC0000DDCC000010B5024911
:10C4B00000F08CF810BDC0460DC4000070B56825B2
:10C4C0004A1E55430E002900743100F081F9041E04
:10C4D00008D000212A00016046600C30A06068325C
:10C4E000FFF7D0F9200070BD836913B50400002B5D
:10C4F00028D18364C3640365134B144A1B688262AA
:10C500000193984201D101238361200000F020F8BB
:10C510006060200000F01CF8A060200000F018F817
:10C520000022E06004216068FFF79CFF01220921DE
:10C53000A068FFF797FF02221221E068FFF792FF41
:10C540000123A36113BDC0467CE60000ADC400001A
:10C55000F8B51C4B07001E68B369002B02D13000F0
:10C56000FFF7C2FF4836B4687368013B04D53368EF
:10C57000002B07D03668F6E70C22A55E002D0DD003
:10C580006834F2E704213800FFF798FF3060002894
:10C59000F0D10C2304003B602000F8BD20000A4BC2
:10C5A000656625606560A560E36025616561A561DC
:10C5B000082229005C30FFF765F96563A563A5646F
:10C5C000E564E9E77CE600000100FFFFF7B5040041
:10C5D0000700002601914834002C01D13000FEBD37
:10C5E0006368A5680093009B013B009301D5246814
:10C5F000F2E7AB89012B08D90E22AB5E013304D0E0
:10C6000029003800019B984706436835EBE7EC307A
:10C610000068704770B50E001D000E23C95E96B00D
:10C620001400002907DA00232B60B3891B0611D4FC
:10C630008023DB000FE06A4600F088FB0028F2DB75
:10C64000F022019B12021340054A9B185A425341A3
:10C650002B60EDE740230020236016B070BDC0467C
:10C6600000E0FFFFF7B502268B8905000C0033427E
:10C6700006D0230047332360236101236361F7BDA4
:10C6800001AB6A46FFF7C6FF00990700280000F0DB
:10C690009FF8002808D10C22A35E9A05EFD403224C
:10C6A00093431E43A681E4E70F4BAB628023A2892C
:10C6B00020601343A381009B20616361019B002BD9
:10C6C0000DD00E23E15E280000F052FB002806D0BA
:10C6D0000322A38993431A0001231343A381A08952
:10C6E0003843A081CBE7C046ADC4000010B5034B72
:10C6F0000100186800F06CF810BDC04684000020EE
:10C7000082B0002900D101A9101E06D0002B06D04E
:10C7100013780B601078431E984102B070470220D6
:10C720004042FAE7C9B28218904201D10020704716
:10C7300003788B42FBD00130F6E7000070B50500AE
:10C74000002910D00C1F2368002B00DAE418280001
:10C7500000F034FB1D4A1368002B05D163601460A0
:10C76000280000F02CFB70BDA34209D92168601895
:10C770008342F3D118685B6841182160EEE713002B
:10C780005A68002A01D0A242F9D919685818A04263
:10C790000BD120680918581819608242E0D110683E
:10C7A0005268411819605A60DAE7A04202D90C2396
:10C7B0002B60D5E721686018824203D11068526867
:10C7C0004118216062605C60CAE7C046301C0020EE
:10C7D000032370B5CD1C9D43083506000C2D1ED2D9
:10C7E0000C25A9421DD8300000F0E8FA254A14684B
:10C7F0002100002919D1244C2368002B03D13000DB
:10C8000000F0CAF920602900300000F0C5F9431C8F
:10C810002BD10C233000336000F0D1FA03E0002D5F
:10C82000DFDA0C233360002070BD0B685B1B19D46A
:10C830000B2B03D90B60CC18256003E04B688C42AE
:10C840000DD11360300000F0BAFA200007220B303F
:10C85000231D9043C31AE7D05A42E250E4E76360D5
:10C860000C00EFE70C004968C3E70323C41C9C439A
:10C87000A042E1D0211A300000F08EF9431CDBD138
:10C88000C7E7C046301C0020341C0020F8B5070064
:10C890000D001600002905D11100FFF799FF0400D3
:10C8A0002000F8BD002A03D1FFF748FF3400F7E766
:10C8B00000F086FA2C00B042F2D231003800FFF7C7
:10C8C00087FF041EECD029003200FEF7BFFF2900CD
:10C8D0003800FFF733FFE3E7F0B58E6885B0070057
:10C8E0000C00039201939E423CD890238A89DB007E
:10C8F0001A4234D00325096923685B1A02936369DD
:10C9000002985D43EB0F5D19019B6D1001331B18FD
:10C91000AB4200D91D00530532D529003800FFF77E
:10C9200057FF061E09D10C233B6040230120A2893A
:10C9300040421343A38105B0F0BD029A2169FEF77E
:10C9400085FFA389144A1A4080231343A381029BC5
:10C950002661F61826606561019EED1AA560019BAF
:10C960009E4200D9019E320003992068FEF777FFAE
:10C97000A36800209B1BA36023689E192660DAE74A
:10C980002A003800FFF782FF061EE0D12169380037
:10C99000FFF7D4FEC7E7C0467FFBFFFFF0B59FB0AF
:10C9A000029005938B890F0016001B0611D50B69A9
:10C9B000002B0ED14021FFF70BFF386038610028B3
:10C9C00005D10C23029A013813601FB0F0BD40233B
:10C9D0007B61002306AC6361203363761033A3765A
:10C9E00035002B78002B01D0252B46D1AB1B0493AF
:10C9F0000CD0320039000298FFF76EFF431C00D1C3
:10CA0000AEE06269049B9446634463612B78002B1B
:10CA100000D1A5E0012200235242626002A95432F3
:10CA200052186E1C2360E360A3601370A365317815
:10CA300005225448FFF776FE751C00281FD1226896
:10CA4000D30604D5532302A95B18202119701307BC
:10CA500004D5532302A95B182B21197033782A2B94
:10CA600016D0350000210A20E3682A786E1C303A7F
:10CA7000092A4ED9002918D010E00135B1E7414B01
:10CA80002268C01A01238340134323602E00CEE79F
:10CA9000059B191D1B680591002B01DB099304E020
:10CAA0005B42E3600223134323602B782E2B0AD1D1
:10CAB0006B782A2B35D1059B02351A1D1B68059210
:10CAC000002B2BDB0793304E297803223000FFF731
:10CAD00029FE002806D04023801B834022680135B0
:10CAE000134323602978062228486E1C2176FFF71D
:10CAF00019FE00283CD0264B002B25D10722059B90
:10CB000007339343083305936369039A9B18636162
:10CB100066E7434301219B183500A6E701235B42EA
:10CB2000D0E700230A201A000135636029786E1CC3
:10CB30003039092903D9002BC5D00792C3E74243F6
:10CB4000012352183500F1E705AB00933A00114B71
:10CB50002100029800E000BF0390039B0133D3D172
:10CB6000BB890B985B0600D42FE7012040422CE7DD
:10CB700005AB00933A00074B21000298FFF736F807
:10CB8000EAE7C04680E6000086E600008AE600008C
:10CB900000000000D9C80000002370B5064C050055
:10CBA0000800236000F060F9431C03D12368002BC8
:10CBB00000D02B6070BDC046C42F002070B50400AB
:10CBC0000D001F2904D9162303600120404270BDC7
:10CBD000436C002B04D08A009B181A68002A08D1E5
:10CBE000200000F031F82A000100200000F01AF8BF
:10CBF000EDE70020012AEAD0511C03D116230130B1
:10CC00002360E4E7002428001C6090472000DEE752
:10CC100010B5034B01001868FFF7D0FF10BDC046E8
:10CC200084000020002370B5064C050008001100A8
:10CC3000236000F001F9431C03D12368002B00D0CE
:10CC40002B6070BDC42F002010B500F0E5F810BDBA
:10CC500070B50C000E25495F00F0BAF8002803DB20
:10CC6000636D1B18636570BDA389024A1340A381DD
:10CC7000F9E7C046FFEFFFFFF8B51F008B890500FD
:10CC80000C001600DB0505D50E23C95E0022022329
:10CC900000F080F8A389054A28001340A3813200E0
:10CCA0000E23E15E3B0000F02BF8F8BDFFEFFFFF25
:10CCB00070B50C000E25495F00F06CF8A389421C8A
:10CCC00003D1054A1340A38170BD80225201134352
:10CCD000A3816065F8E7C046FFEFFFFF10B50E23A4
:10CCE000C95E00F021F810BD0B1E04D0FF2A04D944
:10CCF0008A2303608B3B180070470A700123FAE710
:10CD000070B50500080011000022064C22601A00D0
:10CD100000F0B8F8431C03D12368002B00D02B602F
:10CD200070BDC046C42F0020002370B5064C05001E
:10CD30000800236000F060F8431C03D12368002B37
:10CD400000D02B6070BDC046C42F0020002370B5FA
:10CD5000064C050008001100236000F055F8431C44
:10CD600003D12368002B00D02B6070BDC42F00209E
:10CD7000002370B5064C05000800236000F054F84D
:10CD8000431C03D12368002B00D02B6070BDC0462C
:10CD9000C42F002070B50500080011000022064CC9
:10CDA00022601A0000F050F8431C03D12368002BC6
:10CDB00000D02B6070BDC046C42F00207047704764
:10CDC0000B1F1B68181F002B01DA0B58C018704787
:10CDD00070B50500080011000022064C22601A0000
:10CDE00000F03AF8431C03D12368002B00D02B60DD
:10CDF00070BDC046C42F002058220120014B404284
:10CE00001A607047C42F002058220120014B404275
:10CE10001A607047C42F002058220120014B404265
:10CE20001A607047C42F00205822024B00201A605D
:10CE30007047C046C42F002058220120014B4042B9
:10CE40001A607047C42F002058220120014B404235
:10CE50001A607047C42F002058220120014B404225
:10CE60001A607047C42F0020044A1368002B00D1B9
:10CE7000034B1818106018007047C046381C00207B
:10CE8000C82F002058220120014B40421A607047F1
:10CE9000C42F0020FEE7C046F8B5C046F8BC08BC69
:10CEA0009E467047F8B5C046F8BC08BC9E46704721
:10CEB000646174610000000034CF0000EF010000E5
:10CEC0003DCF0000E302000045CF0000190900003B
:10CED0004CCF0000290A000051CF0000410500009E
:10CEE0005CCF00005303000061CF0000810C000004
:10CEF0006DCF00001F02000077CF00002108000066
:10CF000085CF0000CD06000092CF00000305000091
:10CF100072616E646F6D00616C6C006C61737400A3
:10CF200066616C7365007472756500252E3135730A
:10CF30002E2E2E006D616B654C6973740061646404
:10CF40004C6173740064656C657465006A6F696E2A
:10CF500000636F707946726F6D546F0066696E641E
:10CF6000006A6F696E537472696E677300756E69DB
:10CF7000636F6465417400756E69636F64655374B3
:10CF800072696E67006E657742797465417272618D
:10CF90007900667265654D656D6F727900000000FD
:10CFA00005D000000D1100000AD000002B11000078
:10CFB00045CF00002F11000010D00000111100001B
:10CFC0001AD000003311000023D0000037110000F8
:10CFD0002DD000003B11000038D000003F110000B0
:10CFE00044D00000151100004DD0000023110000B6
:10CFF00057D000001911000062D000002711000076
:10D0000066696C65006F70656E00636C6F736500B8
:10D01000656E644F6646696C6500726561644C6953
:10D020006E65007265616442797465730061707049
:10D03000656E644C696E6500617070656E644279FE
:10D040007465730066696C6553697A650073746111
:10D0500072744C697374006E657874496E4C6973B0
:10D06000740073797374656D496E666F000000001B
:10D07000481400005814000072140000F01400005E
:10D08000281500005E15000096150000BC15000074
:10D09000F81500003A16000090160000D4160000A3
:10D0A0004017000088170000AE170000E6170000C8
:10D0B0002C1800005218000080180000AE18000064
:10D0C000F018000074190000461A0000D01A000081
:10D0D000261B0000721B0000921B0000B41B000006
:10D0E0000C1D0000501D0000C81D0000F61D0000B2
:10D0F000441E00007A1E0000E41E00004E1F0000C7
:10D10000AA1F0000082000007E200000F42000007C
:10D1100050210000B4210000EA210000302200006C
:10D1200076220000BE2200001223000066230000C9
:10D13000A42300000C240000422400008A240000E4
:10D14000D22400001A25000054250000A425000068
:10D15000EC2500004E27000080180000E6170000B4
:10D1600054260000481400008A260000B62600005D
:10D17000EC260000182700004814000048140000A6
:10D180004814000048140000C82700000A280000C6
:10D1900050280000A0280000CC28000078290000BA
:10D1A000CA290000F82900004814000048140000B3
:10D1B0001C2A00004C2A00007C2A0000B22A000031
:10D1C000DC2A0000122B00003C2B0000642B000026
:10D1D0008C2B0000BC2B0000EC2B0000162C000058
:10D1E000402C0000702C00009A2C00004814000015
:10D1F00048140000481400004814000048140000BF
:10D20000CA2C0000F62C0000222D0000602D00002A
:10D210008C2D0000C22D0000F82D00002E2E0000E5
:10D22000642E0000902E0000BC2E0000F22E0000A4
:10D23000481400004814000048140000481400007E
:10D24000481400004814000048140000481400006E
:10D25000481400004814000048140000481400005E
:10D2600048140000481400001E2F0000542F000036
:10D270005B2564206974656D206C6973745D00289A
:10D2800025642062797465732900286F626A65637A
:10D290007420747970653A202564290053746163A1
:10D2A0006B20756E646572666C6F7700626F6F6C71
:10D2B00065616E006E756D62657200737472696E81
:10D2C00067006C69737400627974652061727261C1
:10D2D0007900000007000000030000002ED30000CA
:10D2E0007530000036D30000253100003FD3000028
:10D2F000CF31000048D300007930000051D3000046
:10D30000D331000059D30000BD31000000000000FF
:10D310000100000002000000030000000400000003
:10D320000A0000006D6963726F3A62697400686197
:10D3300073546F6E6500706C6179546F6E65006830
:10D340006173536572766F00736574536572766F9F
:10D3500000646163496E6974006461635772697443
:10D360006500474320746F6F6B20256420757365DB
:10D3700063733B206672656520256420776F726455
:10D3800073003C496E74656765723E003C4C69737E
:10D39000743E003C4F626A6563743E003C4279749F
:10D3A0006541727261793E000D0A564D2050616EE2
:10D3B00069633A2025730D0A006D697363000000EC
:10D3C000F5D30000A13E0000FED30000313E000076
:10D3D00002D40000853D00000AD400002B3D00006F
:10D3E00014D40000C13C000020D40000C33B000066
:10D3F0006E756C6C00686578546F496E7400736963
:10D400006E006A736F6E476574006A736F6E436F68
:10D41000756E74006A736F6E56616C756541740049
:10D420006A736F6E4B65794174000000B8D40000D8
:10D430000D3F0000C0D40000113F0000CAD400001E
:10D440002F3F0000D3D40000393F0000DED400009D
:10D45000433F0000EAD400004D3F0000F8D4000034
:10D46000573F000000D50000613F000006D50000D6
:10D470006B3F00001BD50000753F000030D5000059
:10D480007F3F00003CD50000893F00004CD50000E4
:10D49000933F000058D500009D3F000065D5000077
:10D4A000A73F000074D500001B3F000087D5000097
:10D4B000253F00006E657400686173576946690016
:10D4C0007374617274576946690073746F70576939
:10D4D00046690077696669537461747573006D7984
:10D4E000495041646472657373007374617274535C
:10D4F0005349447363616E00676574535349440034
:10D500006D794D414300687474705365727665722D
:10D510004765745265717565737400726573706FD9
:10D520006E64546F487474705265717565737400DD
:10D5300068747470436F6E6E6563740068747470A1
:10D540004973436F6E6E65637465640068747470CC
:10D550005265717565737400687474705265737088
:10D560006F6E736500776562536F636B6574537498
:10D5700061727400776562536F636B65744C61739D
:10D58000744576656E7400776562536F636B65747E
:10D5900053656E64546F436C69656E74001A1B1C8E
:10D5A00003040607090A17181900000000000808FC
:10D5B0000800080A4A4000000A5FEA5FEA0ED92E16
:10D5C000D36E19324489330C924C924D08080000F6
:10D5D0000004880808040804848488000A448A40F7
:10D5E00000048EC480000000048800000EC000000B
:10D5F0000000080001224488100C9252524C048C06
:10D6000084848E1C824C901E1EC244924C06CA52C8
:10D610005FE21FF01EC13E02448ED12E1FE24488FD
:10D62000100ED12ED12E0ED12EC488000800080075
:10D6300000048004880244880482000EC00EC008E2
:10D64000048244880ED126C0040ED135B36C0C92EE
:10D650005ED2521C925C925C0ED010100E1C925244
:10D66000525C1ED01C901E1ED01C90100ED0137148
:10D670002E12525ED2521C8808081C1FE242524CE5
:10D680001254981492101010101E113B75B13111E4
:10D690003935B3710C9252524C1C925C90100C9222
:10D6A000524C861C925C92510ED00C825C1FE4841A
:10D6B0008484125252524C1131312A44113135BBFB
:10D6C0007112524C9252112A4484841EC488101E36
:10D6D0000EC808080E10080482410EC242424E04D1
:10D6E0008A400000000000001F0804800000000EB7
:10D6F000D2524F10101C925C000ED0100E02424EFF
:10D70000D24E0C925C900E06C81C88080ED24EC2F7
:10D710004C10101C92520800080808024002424CAB
:10D7200010149814920808080806001B75B13100FF
:10D730001C925252000C92524C001C925C90000EB3
:10D74000D24EC2000ED010100006C8049808080E71
:10D75000C807001252524F0011312A4400113135CE
:10D76000BB00124C8C9200112A4498001EC4881EE3
:10D7700006C48C8486080808080818080C88180055
:10D78000000C8360000000000100000002000000A7
:10D790000300000004000000050000000600000077
:10D7A0000700000008000000090000000A00000057
:10D7B0000B0000000C0000000D0000000E00000037
:10D7C0000F00000010000000120000001400000014
:10D7D00016000000180000001A0000001C000000E5
:10D7E0001E000000200000002300000026000000B2
:10D7F000290000002C0000002F0000003200000073
:10D80000360000003A0000003E0000004200000028
:10D81000460000004B0000005000000055000000D2
:10D820005A00000061000000680000006F00000066
:10D83000760000007D000000840000008B000000E6
:10D840009200000099000000A0000000A700000066
:10D85000AE000000B5000000BC000000C3000000E6
:10D86000CA000000D1000000D8000000DF00000066
:10D87000E6000000ED000000F4000000FB000000E6
:10D88000FF000000D4D80000C93F0000DFD800002E
:10D8900065450000E9D800008D410000F6D8000081
:10D8A000D5430000FDD800002544000006D9000043
:10D8B0007544000012D900006D43000023D9000018
:10D8C000FD41000030D90000FD4200006469737022
:10D8D0006C6179006C696768744C6576656C006D85
:10D8E00062446973706C6179006D62446973706C35
:10D8F00061794F6666006D62506C6F74006D6255A1
:10D900006E706C6F74006D62447261775368617001
:10D9100065006D625368617065466F724C65747422
:10D920006572006E656F506978656C53656E640052
:10D930006E656F506978656C53657450696E004E02
:10D940006F7420656E6F75676820726F6F6D2065EC
:10D9500076656E20616674657220636F6D706163B9
:10D9600074696F6E00436F6D706163746564204607
:10D970006C61736820636F64652073746F72650AED
:10D980002564206279746573207573656420282589
:10D9900064252529206F6620256400426164207279
:10D9A00065636F726420666F756E6420647572695A
:10D9B0006E6720696E697469616C697A6174696FF8
:10D9C0006E002564202564202564202825642077A6
:10D9D0006F72647329002564207265636F726473CB
:10D9E0002C20256420776F7264732C206D61784938
:10D9F000442025642C20636F6D70616374696F6EC1
:10DA0000206379636C657320256400526573746FBD
:10DA100072656420256420736372697074730053A7
:10DA200074617274656400726164696F0000000063
:10DA3000C0DA0000354F0000CDDA0000D1510000FF
:10DA4000DDDA000051510000EBDA00006553000000
:10DA5000F6DA00005D4F000006DB0000E54F000035
:10DA60001ADB0000CD4F000029DB00004755000005
:10DA700035DB0000C55400003EDB000069540000A7
:10DA800049DB0000B153000054DB0000ED530000FF
:10DA90005DDB00002154000066DB00006D4F0000DC
:10DAA00075DB00004D4F00007EDB00007D4F000065
:10DAB0006E6F6E65006F74686572007061697200E8
:10DAC00064697361626C65526164696F006D65734E
:10DAD000736167655265636569766564007061634B
:10DAE0006B657452656365697665007061636B652B
:10DAF0007453656E64007265636569766564496E2A
:10DB000074656765720072656365697665644D6505
:10DB100073736167655479706500726563656976D2
:10DB20006564537472696E670073656E64496E74E0
:10DB3000656765720073656E645061697200736534
:10DB40006E64537472696E67007365744368616EC6
:10DB50006E656C0073657447726F757000736574E1
:10DB6000506F776572007369676E616C537472658C
:10DB70006E677468006465766963654944006C612A
:10DB800073744D657373616765494400556E6B6EC0
:10DB90006F776E207072696D6974697665205B2598
:10DBA000733A25735D00000000000000963007778F
:10DBB0002C610EEEBA51099919C46D078FF46A7081
:10DBC00035A563E9A395649E3288DB0EA4B8DC79A1
:10DBD0001EE9D5E088D9D2972B4CB609BD7CB17E21
:10DBE000072DB8E7911DBF906410B71DF220B06AF1
:10DBF0004871B9F3DE41BE847DD4DA1AEBE4DD6D01
:10DC000051B5D4F4C785D38356986C13C0A86B6400
:10DC10007AF962FDECC9658A4F5C0114D96C066320
:10DC2000633D0FFAF50D088DC8206E3B5E10694C00
:10DC3000E44160D5727167A2D1E4033C47D4044B40
:10DC4000FD850DD26BB50AA5FAA8B5356C98B24220
:10DC5000D6C9BBDB40F9BCACE36CD832755CDF45A0
:10DC6000CF0DD6DC593DD1ABAC30D9263A00DE51D0
:10DC70008051D7C81661D0BFB5F4B42123C4B356C0
:10DC80009995BACF0FA5BDB89EB802280888055F40
:10DC9000B2D90CC624E90BB1877C6F2F114C6858A0
:10DCA000AB1D61C13D2D66B69041DC760671DB018E
:10DCB000BC20D2982A10D5EF8985B1711FB5B60660
:10DCC000A5E4BF9F33D4B8E8A2C9077834F9000FA0
:10DCD0008EA8099618980EE1BB0D6A7F2D3D6D0840
:10DCE000976C6491015C63E6F4516B6B62616C1C30
:10DCF000D83065854E0062F2ED95066C7BA5011B60
:10DD0000C1F4088257C40FF5C6D9B06550E9B712FF
:10DD1000EAB8BE8B7C88B9FCDF1DDD62492DDA15BF
:10DD2000F37CD38C654CD4FB5861B24DCE51B53ADF
:10DD30007400BCA3E230BBD441A5DF4AD795D83DDF
:10DD40006DC4D1A4FBF4D6D36AE96943FCD96E341F
:10DD5000468867ADD0B860DA732D0444E51D0333FF
:10DD60005F4C0AAAC97C0DDD3C710550AA4102270F
:10DD700010100BBE86200CC925B56857B3856F20DF
:10DD800009D466B99FE461CE0EF9DE5E98C9D9293F
:10DD90002298D0B0B4A8D7C7173DB359810DB42E7F
:10DDA0003B5CBDB7AD6CBAC02083B8EDB6B3BF9ACB
:10DDB0000CE2B6039AD2B1743947D5EAAF77D29D57
:10DDC0001526DB048316DC73120B63E3843B649437
:10DDD0003E6A6D0DA85A6A7A0BCF0EE49DFF099337
:10DDE00027AE000AB19E077D44930FF0D2A30887A7
:10DDF00068F2011EFEC206695D5762F7CB67658057
:10DE000071366C19E7066B6E761BD4FEE02BD38956
:10DE10005A7ADA10CC4ADD676FDFB9F9F9EFBE8EB6
:10DE200043BEB717D58EB060E8A3D6D67E93D1A1F6
:10DE3000C4C2D83852F2DF4FF167BBD16757BCA6D6
:10DE4000DD06B53F4B36B248DA2B0DD84C1B0AAF76
:10DE5000F64A0336607A0441C3EF60DF55DF67A8F6
:10DE6000EF8E6E3179BE69468CB361CB1A8366BC86
:10DE7000A0D26F2536E2685295770CCC03470BBBD6
:10DE8000B91602222F260555BE3BBAC5280BBDB2D6
:10DE9000925AB42B046AB35CA7FFD7C231CFD0B576
:10DEA0008B9ED92C1DAEDE5BB0C2649B26F263EC68
:10DEB0009CA36A750A936D02A906099C3F360EEB76
:10DEC0008567077213570005824ABF95147AB8E236
:10DED000AE2BB17B381BB60C9B8ED2920DBED5E516
:10DEE000B7EFDC7C21DFDB0BD4D2D38642E2D4F166
:10DEF000F8B3DD686E83DA1FCD16BE815B26B9F6F6
:10DF0000E177B06F7747B718E65A0888706A0FFF55
:10DF1000CA3B06665C0B0111FF9E658F69AE62F815
:10DF2000D3FF6B6145CF6C1678E20AA0EED20DD715
:10DF30005483044EC2B30339612667A7F71660D035
:10DF40004D476949DB776E3E4A6AD1AEDC5AD6D975
:10DF5000660BDF40F03BD83753AEBCA9C59EBBDE95
:10DF60007FCFB247E9FFB5301CF2BDBD8AC2BACA45
:10DF70003093B353A6A3B4240536D0BA9306D7CDB5
:10DF80002957DE54BF67D9232E7A66B3B84A61C4D5
:10DF9000021B685D942B6F2A37BE0BB4A18E0CC395
:10DFA0001BDF055A8DEF022D416C6C207461736B81
:10DFB000732073746F70706564007631303900209F
:10DFC0002573202573004D656D6F727920636C6534
:10DFD00061726564004E6F206672656520746173BE
:10DFE0006B20656E747269657300000044E0000088
:10DFF0006569000051E00000ED6400005DE0000094
:10E000003569000063E000004569000069E0000038
:10E01000556900006FE000002165000079E0000014
:10E02000C169000081E00000156700008AE000007F
:10E030007D65000092E000006966000073656E7304
:10E040006F727300616363656C65726174696F6E92
:10E050000074656D70657261747572650074696CC9
:10E0600074580074696C74590074696C745A007443
:10E070006F756368526561640069326352656164FB
:10E08000006932635772697465007265616444485F
:10E0900054006D6963726F70686F6E6500000000F8
:10E0A0001CE100004D6A00002AE100005D6A0000EA
:10E0B00037E10000516A000040E10000616A0000A1
:10E0C0004AE10000656A000053E10000696A00004F
:10E0D00058E100006D6A00005DE10000716A000017
:10E0E00069E10000756A000070E10000796A0000D3
:10E0F00079E100007D6A00007EE10000816A000095
:10E1000089E10000856A000093E10000556A000083
:10E110009DE10000596A000074667400656E6162DA
:10E120006C65446973706C617900736574426163F6
:10E130006B6C69676874006765745769647468001C
:10E1400067657448656967687400736574506978B9
:10E15000656C006C696E65007265637400726F7542
:10E160006E6465645265637400636972636C650014
:10E17000747269616E676C650074657874007466AA
:10E1800074546F756368656400746674546F756366
:10E19000685800746674546F7563685900746674C7
:10E1A000546F75636850726573737572650076613C
:10E1B00072730000D4E10000156F0000DEE1000082
:10E1C000F56E0000E7E10000D16E0000F3E1000011
:10E1D0005D6E0000766172457869737473007661D4
:10E1E000724E616D6564007365745661724E616D47
:10E1F0006564007661724E616D65466F72496E644A
:10E2000065780057656C636F6D6520746F204D698C
:10E2100063726F426C6F636B732100705F73706920
:10E2200020213D204E554C4C002F686F6D652F67A7
:10E2300069742F2E706C6174666F726D696F2F70C8
:10E2400061636B616765732F6672616D65776F726D
:10E250006B2D61726475696E6F6E6F726469636E47
:10E260007266352F6C69627261726965732F5350E3
:10E27000492F5350492E63707000535049436C61CD
:10E2800073733A3A535049436C617373284E524644
:10E290005F5350495F547970652A2C2075696E74FC
:10E2A000385F742C2075696E74385F742C20756922
:10E2B0006E74385F74290000000000000000000048
:10E2C00021710000DD700000037100000D7100007D
:10E2D000177100000171000003000000020000003F
:10E2E0000100000004000000050000001100000013
:10E2F0000C0000000B000000120000000A000000EB
:10E30000060000001A0000001400000017000000C2
:10E31000160000001500000010000000FFFFFFFFC6
:10E32000FFFFFFFF000000001E00000019000000BA
:10E3300018000000070000000800000009000000AD
:10E340000D0000000E0000000F0000001C00000087
:10E350001B0000001D000000130000000000000072
:10E36000000000000D750000417D00008D7500006B
:10E37000A17500009775000009750000FD7400008C
:10E38000AD75000029750000F97400000000000060
:10E39000000000000000304300000000000030C317
:10E3A0007371727400000000FB21F93FFB210940EA
:10E3B0007CD91240FB2119407A6A1F407CD9224047
:10E3C000BBFD2540FB2129403A462C407A6A2F406C
:10E3D0005C4731407CD932409C6B3440BBFD3540BA
:10E3E000DB8F3740FB2139401BB43A403A463C4072
:10E3F0005AD83D407A6A3F404C7E40405C4741409D
:10E400006C1042407CD942408CA243409C6B4440FB
:10E41000AC344540BBFD4540CBC64640DB8F474052
:10E42000EB584840FB21494083F9A200444E6E005E
:10E43000FC291500D1572700DD34F50062DBC00050
:10E440003C999500419043006351FE00BBDEAB0058
:10E45000B761C5003A6E2400D24D42004906E00083
:10E4600009EA2E001C92D100EB1DFE0029B11C0010
:10E47000E83EA700F535820044BB2E009CE98400ED
:10E48000B4267000417E5F00D69139005383390075
:10E490009CF439008B5F840028F9BD00F81F3B0015
:10E4A000DEFF97000F980500112FEF000A5A8B002E
:10E4B0006D1F6D00CF7E360009CB2700464FB70099
:10E4C0009E663F002DEA5F00BA277500E5EBC700A6
:10E4D0003D7BF100F739070092528A00FB6BEA009E
:10E4E0001FB15F00085D8D00300356007BFC4600C5
:10E4F000F0AB6B0020BCCF0036F49A00E3A91D00FE
:10E500005E619100081BE60085996500A0145F001C
:10E510008D40680080D8FF0027734D00060631004B
:10E52000CA561500C9A873007BE260006B8CC0005E
:10E5300000000040FB21F93F000000002D44743E24
:10E54000000000809846F83C0000006051CC783B09
:10E5500000000080831BF0390000004020257A383D
:10E56000000000802282E336000000001DF36935C0
:10E57000020000000300000004000000060000008C
:10E58000B89900006299000062990000909A00001A
:10E590005E9900005E990000869A0000909A000043
:10E5A0005E990000869A00005E990000909A000033
:10E5B000949A0000949A0000949A00009C9A00009B
:10E5C00094A4000006A300004AA30000AEA200002D
:10E5D0004AA300003AA400004AA30000AEA2000033
:10E5E00006A3000006A300003AA40000AEA20000AB
:10E5F000A6A20000A6A20000A6A2000048A4000057
:10E60000BCAB0000BEAA0000BEAA0000DCAD00004A
:10E61000B8AA0000B8AA0000C4AD0000DCAD00003C
:10E62000B8AA0000C4AD0000B8AA0000DCAD00002C
:10E63000D2AD0000D2AD0000D2AD0000E0AD0000D0
:10E640002C2066756E6374696F6E3A200061737377
:10E65000657274696F6E2022257322206661696C71
:10E6600065643A2066696C6520222573222C206C33
:10E67000696E65202564257325730A0088000020D3
:10E68000232D302B2000686C4C006566674546479B
:10E69000003031323334353637383941424344451E
:10E6A000460030313233343536373839616263648D
:10E6B000656600000000000000000000000000008F
:10E6C000000000000000000000000000000000004A
:10E6D000000000000000000000000000000000003A
:10E6E000000000000000000000000000000000002A
:10E6F000000000000000000000000000000000001A
:10E700000000000000000000000000000000000009
:10E7100000000000504F53495800002020202020C6
:10E7200020202020282828282820202020202020C1
:10E7300020202020202020202020208810101010B1
:10E740001010101010101010101010040404040405
:10E750000404040404101010101010104141414131
:10E760004141010101010101010101010101010119
:10E77000010101010101101010101010424242422B
:10E7800042420202020202020202020202020202E9
:10E79000020202020202101010102000000000000D
:10E7A0000000000000000000000000000000000069
:10E7B0000000000000000000000000000000000059
:10E7C0000000000000000000000000000000000049
:10E7D0000000000000000000000000000000000039
:10E7E0000000000000000000000000000000000029
:10E7F0000000000000000000000000000000000019
:10E800000000000000000000000000000000000008
:10E8100000000000000000000000000000000000F8
:08E82000E818FF7F0100000071
:10E82800FFFFFFFFE803000001000000E803DC052C
:10E83800DC05DC05DC050000FFFFFFFFFFFFFFFF35
:10E848001800000019FCFFFFFFFFFFFFFF0000009A
:10E858000024F4000200000003000000FFFFFFFF97
:10E86800000000000100000000000200010000009C
:10E87800FFFFFFFF0000000002000000000004008E
:10E8880002000000FFFFFFFF00000000030000007F
:10E8980000000800030000000A0000000800000053
:10E8A800010000008800002000000000D4E60000FD
:10E8B800F4E60000B4E600000000000000000000DC
:10E8C8000000000000000000000000000000000040
:10E8D8000000000000000000000000000000000030
:10E8E8000000000000000000000000000000000020
:10E8F8000000000000000000000000000000000010
:10E9080000000000000000004300000000000000BC
:10E9180000000000000000000000000000000000EF
:10E92800000000000000000043000000000000009C
:10E9380000000000000000000000000000000000CF
:10E94800000000000000000043000000000000007C
:10E9580000000000000000000000000000000000AF
:10E96800000000000000000043000000000000005C
:10E97800000000000000000000000000000000008F
:10E98800000000000000000043000000000000003C
:10E99800000000000000000000000000000000006F
:10E9A800000000000000000043000000000000001C
:10E9B800000000000000000000000000000000004F
:10E9C80000000000000000004300000000000000FC
:10E9D800000000000000000000000000000000002F
:10E9E8000000000000000000E9CC000001C70000A2
:10E9F800000000001AE7000032CF0000B8D3000082
:10EA0800B8D30000B8D30000B8D30000B8D30000D2
:10EA1800B8D30000B8D30000B8D30000B8D30000C2
:10EA2800FFFFFFFFFFFFFFFFFFFFFFFFFFFF0000EC
:10EA38000100415343494900000000000000000064
:10EA480000000000000000000000000000000000BE
:10EA58000000415343494900000000000000000045
:10EA6800000000000000000000000000000000009E
:10EA780000000000E9000000AD7000000174000013
:08EA880059780000C1000000F4
:040000030000749DE8
:00000001FF
